:100000004BC0000042C2000040C200003EC20000DF
:100010003CC200000C94D96238C2000036C2000015
:1000200034C2000032C200000C94CF620C94C5624E
:100030002CC200002AC2000028C2000026C2000014
:1000400024C2000022C2000020C200001EC2000024
:100050001CC200000C94A56318C2000016C2000068
:1000600014C2000012C2000010C200000EC2000044
:100070000CC200000AC2000008C2000006C2000054
:1000800004C2000002C2000000C20000FEC1000065
:10009000FCC10000FAC1000011241FBECFEFD0E266
:1000A000DEBFCDBF0E9400F0D7C10000076342361B
:1000B000B79BD8A71A39685618AEBAAB558C1D3CF9
:1000C000B7CC5763BD6DEDFD753EF6177231BF00BD
:1000D0000000803F05A84CCDB2D44EB93836A902F5
:1000E0000C50B9918688083CA6AAAA2ABE00000036
:1000F000803F08000000BE922449123EABAAAA2A03
:10010000BECDCCCC4C3E00000080BEABAAAAAA3E1D
:1001100000000000BF000000803F00000000000859
:100120004178D3BB4387D1133D190E3CC3BD4282F6
:10013000AD2B3E68EC8276BED98FE1A93E4C80EFB4
:10014000FFBE01C4FF7F3F0000000000FF004C8A9B
:1001500097509545406BA6D8E4B2282EAE90BF26A6
:10016000B14EE86FD0FBE0709A51862C379845323B
:10017000539D06840D971A8CE61E2E0DB41D401655
:100180009AC591F9F786A142660620AFAE19EE270F
:10019000C2BB0EBAB90AAA95CA45040444C1796A19
:1001A00091EE7D3E2E4C960BA96E5A6A9FF56D0519
:1001B000BB8F808DB4F54FC14AE99E674536394FF4
:1001C00075ADF44CB227A939D78036F7C49C7E6A46
:1001D000605F677992B4DD0E4786CD1A6DC6258AB9
:1001E000F464D953D154DB67F78B22BD5CFEA44D78
:1001F000F9A7590EC57E3BF9BA7D430AD39F6C3BE4
:100200000BDEB2875E3710ECC8A6856546290CF177
:10021000D6BCA38C755E4934200DFAE9D7C7B6A7C2
:10022000988A7C6E6155493D32271D1209FFF6EE12
:10023000E5DDD5CEC6BFB9B2ACA6A09A958F8A85AA
:10024000817C78736F6B6864605D5A56FF59E97DF5
:1002500015B150F39942EE9D4F04BC7632F1B2765F
:100260003B03CC98653405D8AC8259320CE7C4A264
:100270008161432509EDD3B9A089725C46321E0B1A
:10028000F8E6D5C4B4A596887A6D6053473C30260D
:100290001B1108FEF5EDE4DCD4CDC6BFB8B1ABA5AB
:1002A0009F99948F8A85807C77736F6B6763605D9D
:1002B000595653504D4A484543403E3C3A383634EF
:1002C00032302E2D2B2A282725242321201F1E1DC6
:1002D0001C1B1A19181716161514131312111110C6
:1002E0000F0F0E0E0D0D0C0C0B0B0B0A0A09090952
:1002F0000808080807070706060606060505050597
:1003000005040404040404030303030303030302B6
:1003100002020202020202020202010101010101C3
:1003200001010101010101010101010101000000C0
:1003300000000000000000000000000000000000BD
:10034000000000000000000000000000FF0C0B0B8C
:100350000B0A0A090909080808080707070606061C
:100360000606050505050504040404040403030347
:100370000303030303020202020202020202020258
:10038000010101010101010101010101010101015D
:10039000010101000000000000000000000000005A
:1003A000000000000000000000000000000000004D
:1003B000000000000000000000000000000000003D
:1003C000000000000000000000000000000000002D
:1003D000000000000000000000000000000000001D
:1003E000000000000000000000000000000000000D
:1003F00000000000000000000000000000000000FD
:1004000000000000000000000000000000000000EC
:1004100000000000000000000000000000000000DC
:1004200000000000000000000000000000000000CC
:1004300000000000000000000000000000000000BC
:1004400000000000000000000000000011241FBE9A
:10045000CFEFD0E2DEBFCDBF17E1ACE5B9E001C020
:100460001D92AF3EB107E1F719E0A0E0B1E0E2E58F
:10047000FFED00E00BBF02C007900D92AC35B10755
:10048000D9F70E94DE630C94A76FBACD2F923F92EA
:100490004F925F926F927F928F929F92AF92BF9294
:1004A000CF92DF92EF92FF920F931F93CF93DF9340
:1004B00000D000D01F92CDB7DEB78FE99DE00E943B
:1004C00046434090D00D5090D10D20915C0E20FFFE
:1004D00015C025FD02C00C944A0E420124FD0FC038
:1004E0008091B50D9091B60D95958795480E591E42
:1004F00021FD07C0C12CD12C76010BC0420121FF88
:10050000F9CFC090B50DD090B60DEE24D7FCE09495
:10051000FE2C00917C0E10917D0E20E030E01058F2
:10052000210931098091580E882311F40C94460E4C
:1005300080918E0E90918F0EA0E0B0E09058A109AE
:10054000B109B7FF02C00C949210B595A795979585
:1005500087959D838C832FB72983F89487EA9BE046
:100560000E94CF422090CB0B3090CC0BAA2497FC5A
:10057000A094BA2C662457FC6094762C8091E10DEF
:100580009091E20DB301A201480F591F611D711D29
:10059000DB01CA01009751E0A507B10524F08FEFF8
:1005A0009FEFA0E0B0E0B7FF02C00C945E0E0E9487
:1005B000FB1346EC41BB469A31E035B925E428B936
:1005C00050EF5BB992EA9EB987E881BB41BB469A7E
:1005D00035B928B960ED6BB99EB981BB00C000C0C8
:1005E00041BB469A35B928B95BB99EB981BB6C81CC
:1005F0007D819101AA27629FB12D7303C001369FAF
:10060000B00D811D9A1F72039A0BB00D811D9A1FA8
:100610001124AA2797FDA095BA2F880D991DAA1D10
:10062000BB1D2091D50D3091D60D820F931FA11DBA
:10063000B11D009731E0A307B10524F08FEF9FEFC4
:10064000A0E0B0E0B7FF02C00C94590E0E94FB136B
:1006500046EC41BB469A31E035B921E428B950EF68
:100660005BB990EA9EB987E881BB41BB469A35B930
:1006700028B960ED6BB99EB981BB00C000C041BB19
:10068000469A35B928B95BB99EB981BBA101AA27A1
:10069000049FB12D1503C001509FB00D811D9A1FFD
:1006A00014039A0BB00D811D9A1F1124AA2797FDE0
:1006B000A095BA2F8C0D9D1DAE1DBF1D2091ED0D77
:1006C0003091EE0D820F931FA11DB11D009751E0D7
:1006D000A507B10524F08FEF9FEFA0E0B0E0B7FFD2
:1006E00002C00C94540E0E94FB1326EC21BB469AC8
:1006F0002224239425B891E498B930EF3BB982EADB
:100700008EB9A7E83A2E31BA21BB469A25B898B9D6
:1007100040EE4BB98EB931BA00C000C021BB469A39
:1007200025B898B93BB98EB931BA83EA9CE02A83DF
:100730003B830E94CF428091C70C9091C80C0E94CD
:10074000FB132A8121BB469A25B895E498B93B81D1
:100750003BB980EA8EB931BA21BB469A25B898B91F
:1007600040EB4BB98EB931BA00C000C021BB469AEC
:1007700025B898B93BB98EB931BA69816FBF3FB717
:100780003983F8948091D50B9091D60BA091D70B1B
:10079000B091D80B8B2F9927AA27BB27892B8A2B9F
:1007A0008B2B21F081ED9BE00E947E428091FA0B21
:1007B000823011F40C94BC0C10F00C94B50C813008
:1007C00011F40C94C10D80E090E06091F30B7091F6
:1007D000F40B0E94871C2090F10B3090F20B280E36
:1007E000391E3092F60B2092F50B8091D10B90912F
:1007F000D20BA091D30BB091D40B4091D50B50915B
:10080000D60B6091D70B7091D80B840F951FA61F44
:10081000B71F8093D50B9093D60BA093D70BB093B3
:10082000D80B8091E30D9091E40DB301A201480F24
:10083000591F611D711D4115510581E06807710542
:1008400024F04FEF5FEF60E070E0DB01CA0177FF5B
:1008500002C00C940E0E0E94FB1366EC61BB469A1C
:1008600051E055B947E448B970EF7BB992EA9EB9B7
:1008700087E881BB61BB469A55B948B9E0EDEBB951
:100880009EB981BB00C000C061BB469A55B948B94A
:100890007BB99EB981BB2C813D81B101AA27269FDE
:1008A000B12D3703A001729FB00D411D5A1F3603B1
:1008B0005A0BB00D411D5A1F1124662757FD609534
:1008C000762F480D591D6A1D7B1D8091D70D909183
:1008D000D80D480F591F611D711D4115510581E04B
:1008E0006807710524F04FEF5FEF60E070E0DB0117
:1008F000CA0177FF02C00C94090E0E94FB1366EC3C
:1009000061BB469A51E055B943E448B970EF7BB9F1
:1009100090EA9EB987E881BB61BB469A55B948B950
:10092000E0EDEBB99EB981BB00C000C061BB469A47
:1009300055B948B97BB99EB981BB9101AA27029FDD
:10094000B12D1303A001309FB00D411D5A1F12039A
:100950005A0BB00D411D5A1F1124662757FD609593
:10096000762F4C0D5D1D6E1D7F1D8091EF0D9091BA
:10097000F00D480F591F611D711D4115510531E0E2
:100980006307710524F04FEF5FEF60E070E0DB017B
:10099000CA0177FF02C00C94040E0E94FB1346ECC0
:1009A00041BB469A31E035B923E428B950EF5BB931
:1009B00092EA9EB987E881BB41BB469A35B928B90E
:1009C00060EE6BB99EB981BB00C000C041BB469AC6
:1009D00035B928B95BB99EB981BB8091D10C909192
:1009E000D20CA091D30CB091D40C8B2F9927AA27AD
:1009F000BB27892B8A2B8B2B09F0D5C78091F60C4E
:100A0000823009F4A1C708F099C7813011F40C9421
:100A1000A00D80E090E06091EF0C7091F00C0E94CE
:100A2000871C2091ED0C3091EE0C280F391F30936C
:100A3000F20C2093F10C8091CD0C9091CE0CA091F2
:100A4000CF0CB091D00C4091D10C5091D20C609150
:100A5000D30C7091D40C840F951FA61FB71F8093E1
:100A6000D10C9093D20CA093D30CB093D40CC901A9
:100A70000E94FB1346EC41BB469A31E035B927E4AE
:100A800028B950EF5BB990EA9EB987E881BB41BBBA
:100A9000469A35B928B960EB6BB99EB981BB00C0E5
:100AA00000C041BB469A35B928B95BB99EB981BB34
:100AB00039813FBF3FB73983F8948091FF0B909104
:100AC000000CA091010CB091020C8B2F9927AA2742
:100AD000BB27892B8A2B8B2B09F060C78091240CB4
:100AE000823009F41AC708F012C7813011F40C944F
:100AF000900D80E090E060911D0C70911E0C0E94A2
:100B0000871C20901B0C30901C0C280E391E309234
:100B1000200C20921F0C8091FB0B9091FC0BA0915C
:100B2000FD0BB091FE0B4091FF0B5091000C6091BA
:100B3000010C7091020C840F951FA61FB71F8093A4
:100B4000FF0B9093000CA093010CB093020C8091CA
:100B5000E50D9091E60DB301A201480F591F611DEB
:100B6000711D4115510581E06807710524F04FEFB3
:100B70005FEF60E070E0DB01CA0177FF02C00C9418
:100B8000DF0D0E94FB1366EC61BB469A51E055B93C
:100B900041E448B970EF7BB990EA9EB987E881BB20
:100BA00061BB469A55B948B9E0EEEBB99EB981BB35
:100BB00000C000C061BB469A55B948B97BB99EB91F
:100BC00081BB2C813D81B101AA27269FB12D37031E
:100BD000A001729FB00D411D5A1F36035A0BB00D74
:100BE000411D5A1F1124662757FD6095762F480D29
:100BF000591D6A1D7B1D8091D90D9091DA0D480F0A
:100C0000591F611D711D4115510581E0680771056E
:100C100024F04FEF5FEF60E070E0DB01CA0177FF87
:100C200001C0C9C70E94FB1366EC61BB469A51E044
:100C300055B945E448B970EF7BB990EA9EB987E8A9
:100C400081BB61BB469A55B948B9E0EDEBB99EB995
:100C500081BB00C000C061BB469A55B948B97BB999
:100C60009EB981BB9101AA27029FB12D1303A00158
:100C7000309FB00D411D5A1F12035A0BB00D411D7C
:100C80005A1F1124662757FD6095762F4C0D5D1D68
:100C90006E1D7F1D8091F10D9091F20D480F591F2F
:100CA000611D711D4115510531E06307710524F087
:100CB0004FEF5FEF60E070E0DB01CA0177FF01C03A
:100CC0008FC70E94FB1346EC41BB469A31E035B911
:100CD00025E428B950EF5BB992EA9EB987E881BB59
:100CE00041BB469A35B928B960EE6BB99EB981BB54
:100CF00000C000C041BB469A35B928B95BB99EB95E
:100D000081BB8091FB0C9091FC0CA091FD0CB091EB
:100D1000FE0C8B2F9927AA27BB27892B8A2B8B2B7D
:100D200009F05AC68091200D823009F4DFC508F021
:100D3000D7C5813009F49AC680E090E06091190D22
:100D400070911A0D0E94871C2091170D3091180D7B
:100D5000280F391F30931C0D20931B0D8091F70C29
:100D60009091F80CA091F90CB091FA0C4091FB0C09
:100D70005091FC0C6091FD0C7091FE0C840F951F3E
:100D8000A61FB71F8093FB0C9093FC0CA093FD0C47
:100D9000B093FE0CC9010E94FB1346EC41BB469A7E
:100DA00031E035B921E428B950EF5BB992EA9EB938
:100DB00087E881BB41BB469A35B928B960EB6BB96E
:100DC0009EB981BB00C000C041BB469A35B928B965
:100DD0005BB99EB981BB39813FBF3FB73983F89476
:100DE0008091290C90912A0CA0912B0CB0912C0C85
:100DF0008B2F9927AA27BB27892B8A2B8B2B09F0AE
:100E0000E6C580914E0C823009F459C508F051C5F1
:100E1000813009F4FAC580E090E06091470C709150
:100E2000480C0E94871C2090450C3090460C280EE0
:100E3000391E30924A0C2092490C8091250C9091D9
:100E4000260CA091270CB091280C4091290C5091B0
:100E50002A0C60912B0C70912C0C840F951FA61FEF
:100E6000B71F8093290C90932A0CA0932B0CB0935E
:100E70002C0C8091E70D9091E80DB301A201480F71
:100E8000591F611D711D4115510581E068077105EC
:100E900024F04FEF5FEF60E070E0DB01CA0177FD07
:100EA00093C60E94FB1366EC61BB469A51E055B9AC
:100EB00043E448B970EF7BB990EA9EB987E881BBFB
:100EC00061BB469A55B948B9E0EEEBB99EB981BB12
:100ED00000C000C061BB469A55B948B97BB99EB9FC
:100EE00081BB2C813D81B101AA27269FB12D3703FB
:100EF000A001729FB00D411D5A1F36035A0BB00D51
:100F0000411D5A1F1124662757FD6095762F480D05
:100F1000591D6A1D7B1D8091DB0D9091DC0D480FE2
:100F2000591F611D711D4115510581E0680771054B
:100F300024F04FEF5FEF60E070E0DB01CA0177FD66
:100F40004BC60E94FB1366EC61BB469A51E055B953
:100F500047E448B970EF7BB990EA9EB987E881BB56
:100F600061BB469A55B948B9E0EDEBB99EB981BB72
:100F700000C000C061BB469A55B948B97BB99EB95B
:100F800081BB9101AA27029FB12D1303A001309FBD
:100F9000B00D411D5A1F12035A0BB00D411D5A1FAF
:100FA0001124662757FD6095762F4C0D5D1D6E1D33
:100FB0007F1D8091F30D9091F40D480F591F611D15
:100FC000711D4115510531E06307710524F04FEFA4
:100FD0005FEF60E070E0DB01CA0177FDF9C50E94B8
:100FE000FB1346EC41BB469A31E035B927E428B9FA
:100FF00050EF5BB992EA9EB987E881BB41BB469A44
:1010000035B928B960EE6BB99EB981BB00C000C08C
:1010100041BB469A35B928B95BB99EB981BB80916D
:10102000250D9091260DA091270DB091280D8B2FA5
:101030009927AA27BB27892B8A2B8B2B09F0D6C48B
:1010400080914A0D823009F421C408F019C481301E
:1010500009F436C580E090E06091430D7091440D35
:101060000E94871C2091410D3091420D280F391F9D
:101070003093460D2093450D8091210D9091220DC6
:10108000A091230DB091240D4091250D5091260D76
:101090006091270D7091280D840F951FA61FB71F13
:1010A0008093250D9093260DA093270DB093280DC6
:1010B000C9010E94FB1346EC41BB469A31E035B9A9
:1010C00023E428B950EF5BB992EA9EB987E881BB67
:1010D00041BB469A35B928B960EB6BB99EB981BB63
:1010E00000C000C041BB469A35B928B95BB99EB96A
:1010F00081BB39813FBF2FB72983F8948091530C6E
:101100009091540CA091550CB091560C8B2F9927AF
:10111000AA27BB27892B8A2B8B2B09F062C48091CD
:10112000780C823009F480C308F078C3813009F468
:10113000D6C480E090E06091710C7091720C0E94B6
:10114000871C20906F0C3090700C280E391E309246
:10115000740C2092730C80914F0C9091500CA091C4
:10116000510CB091520C4091530C5091540C609121
:10117000550C7091560C840F951FA61FB71F8093B6
:10118000530C9093540CA093550CB093560C809133
:10119000E90D9091EA0DB301A201480F591F611D9D
:1011A000711D4115510531E06307710524F04FEFC2
:1011B0005FEF60E070E0DB01CA0177FDF8C40E94D8
:1011C000FB1366EC61BB469A51E055B945E448B95A
:1011D00070EF7BB990EA9EB987E881BB61BB469A04
:1011E00055B948B9E0EEEBB99EB981BB00C000C06B
:1011F00061BB469A55B948B97BB99EB981BB6C8130
:101200007D819101AA27629FB12D7303A001369FB2
:10121000B00D411D5A1F72035A0BB00D411D5A1FCC
:101220001124662757FD6095762F480D591D6A1DBC
:101230007B1D8091DD0D9091DE0D480F591F611DC2
:10124000711D4115510531E06307710524F04FEF21
:101250005FEF60E070E0DB01CA0177FDA4C40E948B
:10126000FB1366EC61BB469A51E055B941E448B9BD
:1012700070EF7BB992EA9EB987E881BB61BB469A61
:1012800055B948B9E0EDEBB99EB981BB00C000C0CB
:1012900061BB469A55B948B97BB99EB981BBB101CA
:1012A000AA27069FB12D1703A001709FB00D411D05
:1012B0005A1F16035A0BB00D411D5A1F11246627E1
:1012C00057FD6095762F4C0D5D1D6E1D7F1D809125
:1012D000F50D9091F60D480F591F611D711D4115B7
:1012E000510581E06807710524F04FEF5FEF60E082
:1012F00070E0DB01CA0177FD77C40E94FB1346EC66
:1013000041BB469A31E035B921E428B950EF5BB9C9
:1013100090EA9EB987E881BB41BB469A35B928B9A6
:1013200060EB6BB99EB981BB00C000C041BB469A5F
:1013300035B928B95BB99EB981BB80914F0D9091A9
:10134000500DA091510DB091520D8B2F9927AA27C6
:10135000BB27892B8A2B8B2B09F02FC38091740D0F
:10136000823009F47AC208F072C2813009F468C38D
:1013700080E090E060916D0D70916E0D0E94871C71
:1013800020916B0D30916C0D280F391F3093700D2B
:1013900020936F0D80914B0D90914C0DA0914D0DB0
:1013A000B0914E0D40914F0D5091500D6091510DE7
:1013B0007091520D840F951FA61FB71F80934F0D7C
:1013C0009093500DA093510DB093520DC9010E94FE
:1013D000FB1346EC41BB469A31E035B925E428B908
:1013E00050EF5BB992EA9EB987E881BB41BB469A50
:1013F00035B928B960EB6BB99EB981BB00C000C09C
:1014000041BB469A35B928B95BB99EB981BB2981E0
:101410002FBF3FB73983F89480917D0C90917E0C5B
:10142000A0917F0CB091800C8B2F9927AA27BB2706
:10143000892B8A2B8B2B09F0BBC28091A20C8230A6
:1014400009F4D9C108F0D1C1813009F489C380E021
:1014500090E060919B0C70919C0C0E94871C2090E6
:10146000990C30909A0C280E391E30929E0C2092C6
:101470009D0C8091790C90917A0CA0917B0CB0918D
:101480007C0C40917D0C50917E0C60917F0C709192
:10149000800C840F951FA61FB71F80937D0C90931F
:1014A0007E0CA0937F0CB093800C8091EB0D9091FB
:1014B000EC0D480E591E611C711C4114510441E091
:1014C000640671042CF044244A94542C612C712C31
:1014D000D301C20177FC8CC30E94FB1366EC61BB95
:1014E000469A51E055B947E448B970EF7BB990EAA4
:1014F0009EB987E881BB61BB469A55B948B9E0EE11
:10150000EBB99EB981BB00C000C061BB469A55B91A
:1015100048B97BB99EB981BB6C817D819101AA27B5
:10152000629FB12D7303A001369FB00D411D5A1F5C
:1015300072035A0BB00D411D5A1F1124662757FD27
:101540006095762F480D591D6A1D7B1D8091DF0D1A
:101550009091E00D480F591F611D711D41155105F6
:1015600031E06307710524F04FEF5FEF60E070E05A
:10157000DB01CA0177FD44C30E94FB1366EC61BB2B
:10158000469A51E055B943E448B970EF7BB992EA05
:101590009EB987E881BB61BB469A55B948B9E0ED71
:1015A000EBB99EB981BB00C000C061BB469A55B97A
:1015B00048B97BB99EB981BBB101AA27069FB12D5D
:1015C0001703A001709FB00D411D5A1F16035A0B3F
:1015D000B00D411D5A1F1124662757FD6095762FC7
:1015E0004C0D5D1D6E1D7F1D8091F70D9091F80DC6
:1015F000480F591F611D711D4115510581E0680794
:10160000710524F04FEF5FEF60E070E0DB01CA018D
:1016100077FDF2C20E94FB1346EC41BB469A31E0D3
:1016200035B923E428B950EF5BB990EA9EB987E851
:1016300081BB41BB469A35B928B960EB6BB99EB9FD
:1016400081BB00C000C041BB469A35B928B95BB91F
:101650009EB981BB8091790D90917A0DA0917B0DFF
:10166000B0917C0D8B2F9927AA27BB27892B8A2B1A
:101670008B2B09F0A7C180919E0D823009F4A2C086
:1016800008F09AC0813009F400C280E090E06091D7
:10169000970D7091980D0E94871CE091950DF09127
:1016A000960DE80FF91FF0939A0DE093990D409174
:1016B000750D5091760D6091770D7091780D0091B8
:1016C000790D10917A0D20917B0D30917C0D400F9A
:1016D000511F621F731F4093790D50937A0D6093D1
:1016E0007B0D70937C0DCF010E94FB1346EC41BB38
:1016F000469A31E035B927E428B950EF5BB992EA50
:101700009EB987E881BB41BB469A35B928B960EBE1
:101710006BB99EB981BB00C000C041BB469A35B9C8
:1017200028B95BB99EB981BB29812FBF209160097F
:10173000922F9C7111E009F010E0922F937092307B
:1017400009F4E4C4933009F4D8C4913009F4BBC25D
:101750001111EDC40E94AD5180915C0990915D0919
:10176000A0915E09B0915F090196A11DB11D809302
:101770005C0990935D09A0935E09B0935F09209185
:1017800060092F5F209360090F900F900F900F90CA
:101790000F90DF91CF911F910F91FF90EF90DF900D
:1017A000CF90BF90AF909F908F907F906F905F9001
:1017B0004F903F902F900895833009F477C1843083
:1017C00009F063CF6091790D70917A0D80917B0D56
:1017D00090917C0D20919B0D21112FC2BB27A92F29
:1017E000982F872F8095909552CF833009F48EC122
:1017F000843009F02CCE60917D0C70917E0C80912C
:101800007F0C9091800C20919F0C211120C2BB274E
:10181000A92F982F872F809590951BCE833009F4A0
:1018200020C1843009F085CC6091530C7091540C28
:101830008091550C9091560C2091750C211111C27C
:10184000BB27A92F982F872F8095909574CC833034
:1018500009F431C1843009F08BCD60914F0D709146
:10186000500D8091510D9091520D2091710D2111CB
:10187000FDC1BB27A92F982F872F809590957ACDF2
:10188000833009F4B8C0843009F0E4CB6091250DB1
:101890007091260D8091270D9091280D2091470D74
:1018A0002111EFC1BB27A92F982F872F80959095E5
:1018B000D3CB833009F4A4C0843009F0ACCA609162
:1018C000290C70912A0C80912B0C90912C0C20915A
:1018D0004B0C44E851E00E945142809590959DCA7E
:1018E000833009F418C1843009F026CA6091FB0CDA
:1018F0007091FC0C8091FD0C9091FE0C20911D0DBF
:1019000044E851E00E9451428095909517CA833077
:1019100009F4F6C0843009F0ECC86091FF0B7091B7
:10192000000C8091010C9091020C2091210C44E854
:1019300051E00E94514280959095DDC8833009F4B2
:1019400073C0843009F065C86091D10C7091D20CDD
:101950008091D30C9091D40C2091F30C44E851E089
:101960000E9451428095909556C8833009F462C018
:10197000843011F00C94E3036091D50B7091D60B79
:101980008091D70B9091D80B2091F70B44E851E050
:101990000E945142809590950C94E5038BEF9BE05B
:1019A0000E947E429BC88DEC9CE00E947E4226C82D
:1019B00089E79CE00E947E4240CD8BE49DE00E943E
:1019C0007E42CCCC85E79DE00E947E4254CE85E2EB
:1019D0009CE00E947E4215CA87EF9CE00E947E42F6
:1019E000A1C98FE49CE00E947E4299CB81E29DE0F8
:1019F0000E947E4225CB8091350D9091360D2CCBE7
:101A00008091390C90913A0C08CA6091290C709120
:101A10002A0C80912B0C90912C0C20914B0C44E8BB
:101A200053E00E945142F9C98091E10C9091E20C7F
:101A30000C940B058091E50B9091E60B0C94E5035B
:101A400060914F0D7091500D8091510D9091520DFC
:101A50002091710D211100C1BB27A92F982F872F2D
:101A600089CC8091630C9091640C65CB6091FB0CE8
:101A70007091FC0C8091FD0C9091FE0C20911D0D3D
:101A800044E853E00E94514259C96091790D709128
:101A90007A0D80917B0D90917C0D20919B0D2111F1
:101AA000D1C0BB27A92F982F872FF1CD8091890D09
:101AB00090918A0DECCD80915F0D9091600D5ACC84
:101AC0006091250D7091260D8091270D9091280D24
:101AD0002091470D44E853E00E945142BDCA6091F5
:101AE000530C7091540C8091550C9091560C209190
:101AF000750C211198C0BB27A92F982F872F1BCBBE
:101B000080910F0C9091100C0C947B0580918D0CA2
:101B100090918E0C9ECC80910B0D90910C0D0EC966
:101B20006091FF0B7091000C8091010C9091020C60
:101B30002091210C44E853E00E9451420C947B0513
:101B40006091D10C7091D20C8091D30C9091D40CF7
:101B50002091F30C44E853E00E9451420C940B0591
:101B600060917D0C70917E0C80917F0C9091800C27
:101B700020919F0C21115CC0BB27A92F982F872F84
:101B800068CC6091D50B7091D60B8091D70B90915A
:101B9000D80B2091F70B21116EC0BB27A92F982FCE
:101BA000872F0C94E50380E090E0DC0158CB80E0C7
:101BB00090E0DC0104CB80E090E0DC0133C880E001
:101BC00090E0DC010C94C10580E090E0DC0169C983
:101BD00080E090E0DC0103CA80E090E0DC01B1C964
:101BE00080E090E0DC016DC880E090E0DC0185CB16
:101BF00080E090E0DC0170CC80E090E0DC010ACD78
:101C000080E090E0DC01B8CC80E090E0DC010C9456
:101C1000CD0480E090E0DC010C947D0480E090E055
:101C2000DC010C942B0444E853E00E94981C83CA06
:101C300044E853E00E94981C0CCC44E851E00E9418
:101C4000981CD0CD44E853E00E94981C20CD44E875
:101C500051E00E94981CDFCD44E853E00E94981C9C
:101C600089CB44E851E00E94981CEECD44E851E055
:101C70000E94981C02CE44E853E00E94981C0C94E9
:101C8000E50344E851E00E94981C10CE1D821C829E
:101C90000C94AB028090B50D9090B60D95948794FE
:101CA000840C951C0C946E0280E090E0DC010C9496
:101CB000730380E090E0DC010C94260380E090E068
:101CC000DC010C94D7020E949F298091A60B8823E7
:101CD00071F08091E10F882309F447C38091500E81
:101CE000882329F081508093500E0E94F92480911E
:101CF000490E882309F4FEC18091470E9091480E49
:101D00004091F90D5091FA0D2091D50D3091D60DDD
:101D10002417350708F4F9C24217530770F4B901C4
:101D2000641B750BAB018617970708F4AC01241BE5
:101D3000350B3093D60D2093D50D4091050E509163
:101D4000060E2091E10D3091E20D2417350708F4BD
:101D5000D0C24217530770F4F901E41BF50BAF0131
:101D60008E179F0708F4AC01241B350B3093E20D4E
:101D70002093E10D4091110E5091120E2091ED0D26
:101D80003091EE0D2417350708F4A7C24217530708
:101D900070F4B901641B750BAB018617970708F443
:101DA000AC01241B350B3093EE0D2093ED0D4091CB
:101DB000FB0D5091FC0D2091D70D3091D80D2417BB
:101DC000350708F47EC24217530770F4F901E41B8B
:101DD000F50BAF018E179F0708F4AC01241B350BE0
:101DE0003093D80D2093D70D4091070E5091080ED7
:101DF0002091E30D3091E40D2417350708F454C207
:101E00004217530770F4B901641B750BAB018617B9
:101E1000970708F4AC01241B350B3093E40D209395
:101E2000E30D4091130E5091140E2091EF0D30915F
:101E3000F00D2417350708F42AC24217530770F42F
:101E4000F901E41BF50BAF018E179F0708F4AC01F5
:101E5000241B350B3093F00D2093EF0D4091FD0DB9
:101E60005091FE0D2091D90D3091DA0D24173507D0
:101E700008F400C24217530770F4B901641B750BD4
:101E8000AB018617970708F4AC01241B350B309380
:101E9000DA0D2093D90D4091090E50910A0E209130
:101EA000E50D3091E60D2417350708F4D6C1421729
:101EB000530770F4F901E41BF50BAF018E179F0770
:101EC00008F4AC01241B350B3093E60D2093E50D8F
:101ED0004091150E5091160E2091F10D3091F20D9A
:101EE0002417350708F4ACC14217530770F4B90141
:101EF000641B750BAB018617970708F4AC01241B14
:101F0000350B3093F20D2093F10D4091FF0D509160
:101F1000000E2091DB0D3091DC0D2417350708F4FD
:101F200082C14217530770F4F901E41BF50BAF01AE
:101F30008E179F0708F4AC01241B350B3093DC0D82
:101F40002093DB0D40910B0E50910C0E2091E70D6C
:101F50003091E80D2417350708F458C1421753078C
:101F600070F4B901641B750BAB018617970708F471
:101F7000AC01241B350B3093E80D2093E70D409105
:101F8000170E5091180E2091F30D3091F40D241777
:101F9000350708F42EC14217530770F4F901E41B0A
:101FA000F50BAF018E179F0708F4AC01241B350B0E
:101FB0003093F40D2093F30D4091010E5091020ED9
:101FC0002091DD0D3091DE0D2417350708F404C192
:101FD0004217530770F4B901641B750BAB018617E8
:101FE000970708F4AC01241B350B3093DE0D2093CA
:101FF000DD0D40910D0E50910E0E2091E90D3091A6
:10200000EA0D2417350708F4DAC04217530770F4B5
:10201000F901E41BF50BAF018E179F0708F4AC0123
:10202000241B350B3093EA0D2093E90D4091190ED6
:1020300050911A0E2091F50D3091F60D24173507A9
:1020400008F4B0C04217530770F4B901641B750B54
:10205000AB018617970708F4AC01241B350B3093AE
:10206000F60D2093F50D4091030E5091040E209132
:10207000DF0D3091E00D2417350708F080C0421BBA
:10208000530B8417950708F46EC1420F531F5093EA
:10209000E00D4093DF0D40910F0E5091100E2091F6
:1020A000EB0D3091EC0D2417350708F055C0421B9D
:1020B000530B8417950708F454C1420F531F5093D4
:1020C000EC0D4093EB0D40911B0E50911C0E209196
:1020D000F70D3091F80D2417350760F5421B530BAF
:1020E0008417950708F43BC1420F531F5093F80D16
:1020F0004093F70D2091600944CB22FD42CB812F04
:102100000E94F34A812F0E944620F4CF8AEB9DE083
:102110000E94464380915C0E88700E942E2220917E
:1021200060092FCB0196A11DB11D0C94A5020E9440
:102130003B4D10CB42175307E8F6F901E41BF50BB2
:10214000AF018E179F0708F4AC01241B350B3093A9
:10215000F80D2093F70DCECF4217530708F0B3CFF9
:10216000B901641B750BAB018617970708F4AC0126
:10217000241B350B3093EC0D2093EB0DA4CF4217AD
:10218000530708F088CFF901E41BF50BAF018E1758
:102190009F0708F4AC01241B350B3093E00D20930E
:1021A000DF0D79CF421B530B8417950708F4D5C078
:1021B000420F531F5093F60D4093F50D54CF421B21
:1021C000530B8417950708F4C6C0420F531F509352
:1021D000EA0D4093E90D2ACF421B530B8417950754
:1021E00008F4B7C0420F531F5093DE0D4093DD0D2E
:1021F00000CF421B530B8417950708F4A8C0420F69
:10220000531F5093F40D4093F30DD6CE421B530B46
:102210008417950708F499C0420F531F5093E80D97
:102220004093E70DACCE421B530B8417950708F47F
:102230008AC0420F531F5093DC0D4093DB0D82CEBA
:10224000421B530B8417950708F47BC0420F531FA2
:102250005093F20D4093F10D58CE421B530B84174F
:10226000950708F46CC0420F531F5093E60D40933E
:10227000E50D2ECE421B530B8417950708F45DC065
:10228000420F531F5093DA0D4093D90D04CE421BD9
:10229000530B8417950708F44EC0420F531F5093F9
:1022A000F00D4093EF0DDACD421B530B84179507C9
:1022B00008F43FC0420F531F5093E40D4093E30DC9
:1022C000B0CD421B530B8417950788F1420F531F63
:1022D0005093D80D4093D70D87CD421B530B8417D5
:1022E000950718F1420F531F5093EE0D4093ED0DDB
:1022F0005ECD421B530B84179507A8F0420F531F66
:102300005093E20D4093E10D35CD421B530B8417E2
:10231000950738F0420F531F5093D60D4093D50DBB
:102320000CCDAC01F7CFAC01E9CFAC01DBCFAC01F8
:10233000CDCFAC01BFCFAC01B0CFAC01A1CFAC01D0
:1023400092CFAC0183CFAC0174CFAC0165CFAC01AF
:1023500056CFAC0147CFAC0138CFAC0129CFAC018F
:10236000C3CEAC01AACEAC0190CE8091500E882392
:1023700009F4BBCCB7CCE82FF0E0EE0FFF1FE75419
:10238000F14F8081918108958038910538F4FC01E6
:10239000E050FF4F208130E0C90108952FEF3FEF5B
:1023A000FBCFCF93DF93CFEFD4E1E881F98185EACA
:1023B00096E1A1E6B0E081939193A193B193F98363
:1023C000E883DF91CF9108958091E10F813009F08A
:1023D0000895683F59F06A3FD9F78FEF9FE79093D0
:1023E000A20B8093A10B1092500E08958091500E75
:1023F0008F5F8093500E0895AFEFB4E1ED91FC91A3
:1024000011978191ED93FC930895AFEFB4E1ED91B5
:10241000FC9111978191ED93FC930895AFEFB4E196
:10242000ED91FC911197808191813296ED93FC930F
:102430000895AFEFB4E1ED91FC9111976081718146
:10244000828193813496ED93FC930895E82FE6956D
:10245000E695E695F0E0EE5DF54F9081992351F019
:102460008770E82FF0E0E454F94F2081292381E0C0
:1024700009F0089580E00895FC01A18DBB27A19586
:102480000CF4B095AA0FBB1F1196208531854285AB
:1024900053850E94586F648775878687978708954C
:1024A000CF92DF92EF92FF92CF93603E710581054C
:1024B0009105F8F4DC01CB019F5FAF4FBF4FCC24F7
:1024C000D82EE92EFA2EA0E0B0E020E030E0EBBEFE
:1024D000F601C791A40FB51FCC932F5F3F4FD901D1
:1024E0008FEFC81AD80AE80AF80A211581E03807E0
:1024F00071F7CF91FF90EF90DF90CF90089596EC19
:1025000091BB469A982F9695969596958295880FA9
:10251000807E95B990E498B91BB88EB987E881BBE5
:1025200085E08A95F1F70000089555E05A95F1F796
:10253000000036EC31BB469A80EE87B997E09AB935
:102540008DB915B880E488B91BB880E28EB987E4EC
:1025500081BB82E08A95F1F700C026B199B18CB1B8
:1025600031BB479A37EE37B937EF3AB932EE3DB95A
:10257000422F4695437050E8259F90011124422B2D
:10258000292F2071422B292F269526952870422B22
:1025900096959076492B90E0880F991F8470992723
:1025A000842B0895CF93DF93BC0180E090E04FEF40
:1025B00052E176DFCFEFD2E1D0930015C093FF1444
:1025C0001092011536DF653A76418146910551F04A
:1025D00080E092E0FE019C01119221503040E1F731
:1025E00080E004C012DF8093011581E0DF91CF917C
:1025F0000895AF92BF92CF92DF92EF92FF920F9326
:102600001F93CF93DF935C01C12CD12C7601C0E0E6
:10261000D0E0062F10E00EC0A60141505D4EBE0175
:102620006A0D7B1D80E090E03BDF21962FEFD21AF0
:10263000E20AF20AC017D10778F3CFEFD2E1D093C4
:102640000015C093FF1410920115F3DE653A764130
:102650008146910551F080E092E0FE019C011192CB
:1026600021503040E1F780E004C0CFDE80930115B7
:1026700081E0DF91CF911F910F91FF90EF90DF905C
:10268000CF90BF90AF9008956095EDEEFFE0908100
:10269000982B6923608386EC81BB469A362F330FD3
:1026A000962F9695262F221F2227221F832F867072
:1026B000282B20646071832F880F8072862B307CDA
:1026C000832B9270906C31E035B928B98BB99EB9E3
:1026D00087E881BB85E08A95F1F70000ECEEFFE02A
:1026E00080818F5F808308953091ED0F832F886004
:1026F0008E7F8093ED0F96EC91BB469A282F220F88
:10270000982F9695881F8827881F422F4670842B04
:102710008064207C30713062232B9270906C31E0A9
:1027200035B988B92BB99EB987E881BB85E08A9510
:10273000F1F700008091EC0F8F5F8093EC0F08950C
:102740004091ED0F242F22602093ED0F86EC81BB8A
:10275000469A322F330F922F9695221F2227221F3F
:10276000832F8670282B2064832F880F80724071FE
:10277000842B307C832B9270906C31E035B928B972
:102780008BB99EB987E881BB85E08A95F1F7000097
:102790008091EC0F8F5F8093EC0F089590911D0B4B
:1027A0009E7F8111916090931D0B4FB7F89480919B
:1027B0001D0B96EC91BB469A382F330F982F9695A8
:1027C000232F26702064582F551F5527551F252B62
:1027D000582F5071832F880F8072852B307C832B6C
:1027E0009270906631E035B928B98BB99EB987E807
:1027F00081BB4FBF08959C01232F33272695269533
:10280000722F66EC61BB469A522F550F452F4670CA
:102810004068207133272260352F330F3072322BFE
:10282000507C352B272F26952270206215B848B989
:102830003BB92EB957E851BB9695879596958795E4
:10284000282F61BB469A482F440F382F3695221FF8
:102850002227221F642F6670262B206880719927FB
:102860008260942F990F9072982B407C942B327039
:1028700015B828B99BB93EB951BB0895EF92FF92A4
:102880000F931F93CF93DF937C01EB01142F40FF35
:1028900009C02091E60F3091E70F282739272C7FB8
:1028A000232B71F511FF0AC08091E80F9091E90F79
:1028B0008C279D2788279E7F892B39F4DF91CF9124
:1028C0001F910F91FF90EF9008950D2F0695409165
:1028D000DF0F4F70406BE0910217F091031721E07A
:1028E00063E070E082E097E10995D093E90FC0932F
:1028F000E80FDF91CF911F910F91FF90EF90089516
:1029000090589C013595279535952795092F069563
:102910002F7733274091DF0F4F70406EE091021701
:10292000F091031763E070E082E097E10995F0927F
:10293000E70FE092E60FB6CF0F931F93072F069590
:1029400010E00F771127282F285E2F774091DF0F97
:102950004F704069E0910217F091031763E070E057
:1029600082E097E109951F910F9108950F93262F0B
:102970004F772F778F708068E0910217F0910317DF
:10298000042F482F63E070E082E097E109950F91F2
:102990000895EF92FF920F931F93CF93DF93EC0173
:1029A000162FF42EE22E80912717843071F1C23059
:1029B000D10509F453C0C330D10571F1C130D1053F
:1029C000F9F1C430D105C8F5E0911E17F0911F1739
:1029D000309739F00E2D2F2D412FBE0182E097E167
:1029E0000995E0912017F0912117309739F00E2DBD
:1029F0002F2D412FBE0182E097E10995DF91CF9104
:102A00001F910F91FF90EF900895E0911C17F091A6
:102A10001D173097F9F6D8CF862F807F803A09F4BA
:102A20008DC008F041C0803809F456C0803961F685
:102A3000E0910617F091071742C0C0E0D0E0C4CF84
:102A4000683F50F1E0911817F0911917309709F489
:102A5000BBCF612F82E097E10995C3CF862F807F9E
:102A6000803D09F455C0803F09F440C0803C09F026
:102A7000ABCFE0911017F0911117309709F4A4CF64
:102A8000133F09F43FC0113FE9F1612F6F704F2DE3
:102A900082E097E10995A5CF663F09F095CFE091D7
:102AA0001A17F0911B17D2CF803ED9F0803FA9F1C1
:102AB000803B09F089CFE0910417F091051730971A
:102AC00009F482CF123F99F1612F6F702E2D4F2D97
:102AD00082E097E1099585CFE0910817F0910917F9
:102AE000EECFE0910C17F0910D17E9CF633F59F14C
:102AF000613F09F069CFE0911617F09117173097F1
:102B000009F462CF4F2D612F82E097E1099569CFDB
:102B1000E0911217F0911317B0CF623F09F054CF34
:102B2000E0910E17F0910F17309709F44DCF2E2D2D
:102B30004F2D62EF82E097E1099553CFE0910A179C
:102B4000F0910B17BCCFE0911417F0911517309747
:102B5000C9F63ACFCF93DF93E8DCC82FD0E0E5DCAD
:102B6000382F20E0C22BD32B81E0C9DC81E0C7DC09
:102B700086EC81BB469A15B882E488B91BB880E41C
:102B80008EB987E881BB85E08A95F1F7000082E085
:102B9000B6DCC095D095CE01DF91CF910895EF922C
:102BA000FF920F931F93CF93DF93F82EE62EABEA9D
:102BB0008A9FA12D1124A695A695A6951A2F1F5F71
:102BC00050E0A83008F06AC08A2F90E0880F991F63
:102BD000FC01EE0FFF1FEE0FFF1FEE0FFF1FE80FB0
:102BE000F91FE40FF51FEE0FFF1FE754F14FC081EF
:102BF000D181183008F476C0FA01EE0FFF1FEB54B4
:102C0000F04F0190F081E02DDA01AA0FBB1FAF5603
:102C1000B04F8D919C919F01281B390BA12FB0E0E3
:102C200017970E94C66A6E0F7F1F811D911D611547
:102C3000710521E08207910508F06AC08B010C1B29
:102C40001D0B3E2D20E09BEAF99E912D11249695B7
:102C500096959695892F880F890F880F880F6F2D6D
:102C6000681B862F90E0A0E0B0E077276627620F10
:102C7000731F811D911D2CE030E040E050E00E9468
:102C8000856FD8010E944E6FC80FD91FCE01DF910A
:102C9000CF911F910F91FF90EF900895FA01EE0FE1
:102CA000FF1FEB54F04F0190F081E02DEA01CC0FB3
:102CB000DD1FCF56D04F888199819F01281B390B8A
:102CC000B0E017970E94C66A6E0F7F1F811D911D8D
:102CD0006115710521E082079105F8F4EB011830C8
:102CE00008F08ACF812F90E0880F991FFC01EE0F2A
:102CF000FF1FEE0FFF1FEE0FFF1FE80FF91FE40F7E
:102D0000F51FEE0FFF1FE754F14F6081718196CFE1
:102D10006FEF7FEF80E090E091CF6FEF7FEF80E08B
:102D200090E0EB01DCCFFF920F931F93CF93DF93E3
:102D3000F82EABEA8A9FA12D1124A695A695A695FB
:102D40001A2F1F5F462F50E0A83008F063C08A2F6B
:102D500090E0880F991FFC01EE0FFF1FEE0FFF1F81
:102D6000EE0FFF1FE80FF91FE40FF51FEE0FFF1F17
:102D7000E754F14FC081D181183008F46FC0FA01D7
:102D8000EE0FFF1FEB54F04F0190F081E02DDA01C0
:102D9000AA0FBB1FAF56B04F8D919C919F01281B6E
:102DA000390BA12FB0E017970E94C66A6E0F7F1FE4
:102DB000811D911D6115710521E08207910508F0C3
:102DC00063C08B010C1B1D0B9BEAF99E912D1124F6
:102DD000969596959695892F880F890F880F880F5D
:102DE0006F2D681B862F90E0A0E0B0E07727662764
:102DF0002CE030E040E050E00E94856FD8010E9456
:102E00004E6FC80FD91FCE01DF91CF911F910F9147
:102E1000FF900895FA01EE0FFF1FEB54F04F019061
:102E2000F081E02DEA01CC0FDD1FCF56D04F888115
:102E300099819F01281B390BB0E017970E94C66A41
:102E40006E0F7F1F811D911D6115710521E08207A5
:102E50009105F8F4EB01183008F091CF812F90E044
:102E6000880F991FFC01EE0FFF1FEE0FFF1FEE0FE3
:102E7000FF1FE80FF91FE40FF51FEE0FFF1FE754C8
:102E8000F14F608171819DCF6FEF7FEF80E090E027
:102E900098CF6FEF7FEF80E090E0EB01DCCFAF9257
:102EA000BF92CF92DF92EF92FF920F931F93CF9337
:102EB000DF93E1E2FEE0119211928EE0E534F80733
:102EC000D1F71092460E1092450E8091650E823019
:102ED00009F421C1833009F40AC1813059F0DF912E
:102EE000CF911F910F91FF90EF90DF90CF90BF9007
:102EF000AF900895C0911F0ED091200E1091640ED6
:102F0000110F60E0812F0FDF7C0180E034DA970140
:102F1000281B390BDE010E94C66ACC24CA94DC2C23
:102F2000E12CF12CA70196010E945E6F3093220ED6
:102F30002093210E61E0812FF6DE5C0181E01BDA37
:102F40009501281B390BDE010E94C66AA701960174
:102F50000E945E6F3093240E2093230E62E0812F37
:102F6000E2DE5C0182E007DA9501281B390BDE0105
:102F70000E94C66AA70196010E945E6F3093260EDA
:102F80002093250E63E0812FCEDE5C0183E0F3D930
:102F90009501281B390BDE010E94C66AA701960124
:102FA0000E945E6F3093280E2093270E64E0812FDD
:102FB000BADE5C0184E0DFD99501281B390BDE0104
:102FC0000E94C66AA70196010E945E6F30932A0E86
:102FD0002093290E65E0812FA6DE5C0185E0CBD928
:102FE0009501281B390BDE010E94C66AA7019601D4
:102FF0000E945E6F30932C0E20932B0E66E0812F83
:1030000092DE5C0186E0B7D99501281B390BDE0101
:103010000E94C66AA70196010E945E6F30932E0E31
:1030200020932D0E67E0812F7EDE5C0187E0A3D91F
:103030009501281B390BDE010E94C66AA701960183
:103040000E945E6F3093300E20932F0E68E0812F28
:103050006ADE5C0188E08FD99501281B390BDE01FF
:103060000E94C66AA70196010E945E6F3093320EDD
:103070002093310E69E0812F56DE5C0189E07BD917
:103080009501281B390BDE010E94C66AA701960133
:103090000E945E6F3093340E2093330E6AE0812FCE
:1030A00042DE5C018AE067D99501281B390BDE01FD
:1030B0000E94C66AA70196010E945E6F3093360E89
:1030C0002093350E6BE0812F2EDE8C018BE053D9DF
:1030D0009801281B390BDE010E94C66AA7019601E0
:1030E0000E945E6F3093380E2093370EF8CE2091F9
:1030F000640EA0911F0EB091200E30E00E94C66AAF
:103100002CE030E040E050E00E945E6F3093460ECD
:103110002093450EE4CE2091640EA0911F0EB09135
:10312000200E30E00E94C66A2CE030E040E050E023
:103130000E945E6F30933A0E2093390E30933C0E0E
:1031400020933B0E30933E0E20933D0E3093400E65
:1031500020933F0E3093420E2093410E3093440E45
:103160002093430EBCCE21E030E002C0220F331F7B
:103170008A95E2F7D901A095B095E091E109F09127
:10318000E209EA23FB23F093E209E093E10980914D
:10319000E3099091E4098A239B239093E4098093A7
:1031A000E309662331F0E22BF32BF093E209E0937D
:1031B000E109442331F0282B392B3093E409209383
:1031C000E309089521E030E002C0220F331F8A9501
:1031D000E2F7F901E095F0958091E1099091E2091B
:1031E0008E239F239093E2098093E1094091E309A4
:1031F0005091E4094E235F235093E4094093E3097F
:10320000662331F0282B392B3093E2092093E10912
:103210000895E1EEF9E080819181A3EEB9E02D916E
:103220003C9111973E7F2D933C93916091838083D5
:103230000895CF93DF931F92CDB7DEB790E06983F7
:10324000A3D88093E5096981862F90E09DD880936B
:10325000E6090F90DF91CF91089524E630E040E039
:1032600050E00E945E6F2AE030E040E050E00E94B3
:103270005E6F605D822F805DDCCF21E02093EB09E3
:10328000009721F48FEF8093EA0908951092EA09DC
:10329000BC0181EF99E00E94F06E6CE978E080EF6C
:1032A00099E00C94E56E10923A0A8FEF8093390AF8
:1032B0008093380A1092320A1092330A1092340A1C
:1032C0001092350A1092430A8093420A8093410A71
:1032D00010923B0A10923C0A10923D0A10923E0A4C
:1032E00010924C0A80934B0A80934A0A1092440A27
:1032F0001092450A1092460A1092470A1092550AF7
:103300008093540A8093530A10924D0A10924E0AE9
:1033100010924F0A1092500A10925E0A80935D0A32
:1033200080935C0A1092560A1092570A1092580A1B
:103330001092590A1092670A8093660A8093650A70
:1033400010925F0A1092600A1092610A1092620A4B
:1033500008951F93CF93DF93D82FC92F162F8091F5
:10336000700A68130AC046E050E068E67AE08D2FE4
:103370000E94B76E009711F424C095DF1093700A75
:1033800046E050E06FEF70E088E69AE00E94DE6E63
:10339000ED2FFC2FA8E6BAE080E091919F3F19F451
:1033A000882341F004C09D938F5F8630B1F710925F
:1033B000680A07C086E0E8E6FAE0DF011D928A9518
:1033C000E9F7DF91CF911F910895CF93DF9300D05C
:1033D00000D000D0CDB7DEB786E0E6EBF6E0DE0148
:1033E000119601900D928A95E1F760E0CE01019669
:1033F000B0DF26960FB6F894DEBF0FBECDBFDF91CB
:10340000CF910895EF92FF920F931F93CF93DF9385
:1034100000D000D000D0CDB7DEB746E050E06FEF6F
:1034200070E08E010F5F1F4FC8010E94DE6EF12C0D
:10343000E12C8F2D0BD88823A9F0F801EE0DF11D9A
:10344000E7FCFA95F082EE2021F089819F2D981BF0
:103450009083E39485E08E152CF461E0CE01019613
:1034600078DF05C0F39490E8F912E3CFF6CF269603
:103470000FB6F894DEBF0FBECDBFDF91CF911F9185
:103480000F91FF90EF90089586E0E8E6FAE0A6EA53
:10349000BEE001900D928A95E1F708951092730AAB
:1034A0001092740A1092750A1092760A8FEF809328
:1034B000D80A8093AF0E8FEF9FEFDC018093B00EA0
:1034C0009093B10EA093B20EB093B30E0895CF9324
:1034D000DF93CDB7DEB728970FB6F894DEBF0FBEE7
:1034E000CDBF92E09D8393E09E8325E02F833CE057
:1034F000388729839A8391E09B831C82823081F1F3
:1035000034F4882361F0813009F061C013C0843045
:1035100009F450C0D4F1853009F059C052C0440FAD
:10352000551F661F771F80915A0E8170842B8093E0
:103530005A0E4DC080915C0E8F7C41305105610563
:10354000710521F4806180935C0E41C042305105C9
:103550006105710509F001C0806280935C0E37C07F
:10356000DB01CA0181709927AA27BB2721E08227A6
:103570008093600E4270552766277727759567956B
:10358000579547954093610E22C0DB01CA018170B7
:103590009927AA27BB2721E0822780935E0E4270DD
:1035A00055276627772775956795579547954093D3
:1035B0005F0E0DC0FE01E40FF51F85818093640E40
:1035C00006C0FE01E40FF51F81818093660E2896E8
:1035D0000FB6F894DEBF0FBECDBFDF91CF91089537
:1035E000BF92CF92DF92EF92FF920F931F93CF93F0
:1035F000DF93CDB7DEB764970FB6F894DEBF0FBE8A
:10360000CDBF0091B80E8CE00802800111240C5748
:103610001A4F44DFD80112966D917C911397CE0119
:1036200001960E94F06E6AE978E0CE0101960E9450
:10363000E56EF80180818130B9F020F0823009F028
:103640005AC025C0E181EE0FFF0BEF5AF14F818D7B
:10365000928DA0E0B0E08093B00E9093B10EA09355
:10366000B20EB093B30E47C0E181FF27E7FDF0959E
:10367000EF5AF14F8081F801E80FF11DE80FF11DBD
:1036800064817581CE0101960E94E56E34C089E1A6
:10369000E1E5FEE0A2E0B5E101900D928A95E1F747
:1036A000C12CD12C7601B701A601F80181810FDF71
:1036B00049E150E061E57EE082E095E10E94B76E6D
:1036C000009771F4F8018C2D92E08902E00DF11D54
:1036D000112464817581CE0101960E94E56E0BC0B4
:1036E000AFEFCA1ADA0AEA0AFA0AB4E0CB16D10432
:1036F000E104F104C1F6CE010196BFDD64960FB678
:10370000F894DEBF0FBECDBFDF91CF911F910F9117
:10371000FF90EF90DF90CF90BF9008958F929F928F
:10372000AF92BF92CF92DF92EF92FF920F931F93CF
:103730004A015B0168017901BC0180E090E00E94D0
:10374000206C9058A50194010E945B6B0E94C86B8D
:10375000A70196010E94806D0E94F46BCB011F911E
:103760000F91FF90EF90DF90CF90BF90AF909F9020
:103770008F9008950F931F9380919C0E90919D0EB2
:1037800000E010E42CE135E440E050E86BE376E43F
:1037900080959095C3DF90934F0E80934E0E1F91AE
:1037A0000F9108958091220A9091230A892B90917C
:1037B000240A892B9091250A892B9091260A892B1E
:1037C0009091270A892B9091280A892B9091290A98
:1037D000892B90912A0A892B90912B0A892B909101
:1037E0002C0A892B90912D0A892B90912E0A892BD6
:1037F00090912F0A892B9091300A892B9091310A50
:10380000982B21E009F420E080914C0A9091430A22
:10381000892B9091550A892B90915E0A892B909162
:103820003A0A892B9091670A892B59F48FEF9FEF01
:10383000DC0180934A0E90934B0EA0934C0EB093F4
:103840004D0E2223A1F08091EB0F811110C08091C9
:103850005C0990915D09A0915E09B0915F09809328
:103860004A0E90934B0EA0934C0EB0934D0E2093A6
:10387000EB0F08950F931F93CF93DF93EC018A8989
:103880009B8900E01FEF2FE737E440E050E26BE454
:1038900076E48095909542DFAC0160E070E0088CA2
:1038A00004C0440F551F661F771F0A94D2F748873C
:1038B00059876A877B87DF91CF911F910F91089578
:1038C000CF93DF93EC01888D681741F0688FCE01AC
:1038D000D1DFCE01DF91CF910C943C12DF91CF91DB
:1038E0000895CF93DF93EC01598B488B8A899B898C
:1038F0006817790749F07B8B6A8BCE01BBDFCE015D
:10390000DF91CF910C943C12DF91CF910895AC01DF
:10391000AA27469FB12D579F9001749FB00D211D7E
:103920003A1F569FB00D211D3A1F1124C901089559
:10393000A72F8F3FF9F0282F2F5F30E0220F331F82
:10394000E82FF0E0EE0FFF1FE40FF51F608171819B
:10395000FA01E20FF31F80819181861B970B892F5B
:103960009927A89F9001A99F300D1124260F371F7A
:10397000C90108952EEF31E0E3CF8FBF0895F89489
:1039800081E008958FBF0895EFEFF4E1A081B18148
:103990008C93808191810196918380830895EFEFCC
:1039A000F4E1A081B1818C93808191810196918312
:1039B00080830895CF93DF93EFEFF2E180E092E010
:1039C000DF019C011D9221503040E1F7F09300157A
:1039D000E093FF14C1E0D5E184E088830E94D11117
:1039E0008881DF91CF91DBCFAFEFB4E1ED91FC9116
:1039F000119781939193ED93FC930895F89481E04E
:103A00000895CF92DF92EF92FF920F931F93CF937F
:103A1000DF931F92CDB7DEB7F82E8B01EFB69983F7
:103A2000EDDF99818823F1F08F2D0E94D212EFEF04
:103A3000F3E16F018FEF92E1C81AD90A82918823CE
:103A4000C1F3F092021523E035E1EFEFF2E1A601B8
:103A5000BF01C9010E94C46E9FEFC91AD90AF801BB
:103A6000D182C0828E2D0F90DF91CF911F910F9147
:103A7000FF90EF90DF90CF9085CF1F93CF93DF9390
:103A8000EC011FB7BBDF811104C0812F7BDFC1E0D8
:103A90005AC0CE010E94D212882309F451C010925C
:103AA000630E1092A60E9FEF9093A70E9093A80E10
:103AB0009093A90E9093AA0E9093AB0E809101154E
:103AC000811102C0C1E03DC0C0E00E940E12EC2F87
:103AD000F0E0EE0FFF1FEF5AF14F928F818FCF5F13
:103AE000C93199F7D0E00E940512ED2FF0E0EF5AAE
:103AF000F14F8083DF5FD731B1F7809101158230BC
:103B000008F30E940E12EC2FF0E0EE0FFF1FEF5AA9
:103B1000F14F928F818FCF5FCE3199F70E940512BE
:103B20008093680E0E9405128093690EC6EADEE05B
:103B30000E94051289938EE0CC3AD807C9F7A5CF29
:103B4000C0E0812F1FDF8C2FDF91CF911F9108954F
:103B50001F93CF93DF93182FDFB750DF882309F42B
:103B600048C08BE5E1E5FEE0DF011D928A95E9F7AB
:103B70002FEF3FE730936F0E20936E0E3093750E4C
:103B80002093740E4FEF5FEF5093790E4093780EB1
:103B900030937D0E20937C0E5093890E4093880EB7
:103BA00050936D0E40936C0E3093990E2093980EA7
:103BB0003093A50E2093A40E30939F0E20939E0E5B
:103BC00085E08093640EC1E0C093650EC0935E0EE5
:103BD000C093600EC093660E82E08093670E46E04D
:103BE00050E06FEF70E086EA9EE00E94DE6E1111F9
:103BF00005C08D2FDF91CF911F91C4CEC093510E80
:103C0000F8CFFF920F931F93CF93DF93FFB6F6DEAB
:103C1000811104C08F2DB6DEC1E064C062E08CED7E
:103C200090E00E94F912882309F459C08FE3809331
:103C3000E00F1092E20F80910115882319F0C9EB73
:103C4000DEE013C0C1E04CC00E940E12FE01E00F86
:103C5000F11F918380830E5F1F4F04321105A1F77E
:103C6000A4968FE0C93DD80719F000E010E0ECCF32
:103C70000E940E129093DC0F8093DB0F0E940E12B5
:103C80009093DA0F8093D90F0E9405128093DD0F75
:103C90000E94FC118093DE0F80910115823090F21A
:103CA0000E9405128093E00F0E94FC118093DF0FA9
:103CB00080910115833030F20E9405128093E10F4C
:103CC00080910115843008F4BDCF0E94FC118093CF
:103CD000E20F80910115853008F09CCFB3CFC0E092
:103CE0008F2D50DE8C2FDF91CF911F910F91FF9080
:103CF0000895BF92CF92DF92EF92FF920F931F939E
:103D0000CF93DF931092EF0FC0E0D0E0B4E2BB2E70
:103D10000CC00193119313870287778B668B8150B8
:103D2000C1F72196C830D10591F16C2F772767FD37
:103D30007095872F972F0E94226C6B017C012CE8D5
:103D40003EE24AEB55E40E94806D20E030E44CE90D
:103D500055E40E94F46A0E94F46B8B012CE83EE269
:103D60004AE355E4C701B6010E94806D20E030E4CB
:103D70004CE156E40E94F46A0E94F46BBC9EF00190
:103D8000BD9EF00D1124E754F14F86E0C2CFDF91C4
:103D9000CF911F910F91FF90EF90DF90CF90BF9048
:103DA0000895CF93CFB72ADE8823B1F02AE231E01D
:103DB000E9EBFEE0DF01C9011D920197E9F72FEF62
:103DC0003FE73093DA0F2093D90F8FEF8093DE0F08
:103DD0008FE38093E00F8DDF8C2FCF91D3CD8FBFFA
:103DE0000895EEEEFFE080818F5F80830895F89460
:103DF00081E00895CF93DF93EC016A8F88819981E8
:103E0000AA81BB81892B8A2B8B2B51F460915C0991
:103E100070915D0980915E0990915F090E94456FE4
:103E20000E94426F688379838A839B83DF91CF915D
:103E300008958091A50B08958091A60B08950F9386
:103E40001F93CF93DF93FC018BE1DF011D928A95D5
:103E5000E9F700EF1FE060E070E080E89FEBC0E072
:103E6000D0E01BC0BE01882777FD8095982F0E9467
:103E7000226C21E830E840E85BE30E94806D20E09E
:103E800030E040E85FE30E94F46A2BED3FE049E454
:103E900050E40E94806D0E94586B20E030E040E8C2
:103EA0005FE30E94F46A20E03FEF4FEF56E40E9488
:103EB000806D0E94F46BF801619371938F012196DC
:103EC000C115F1E0DF0771F6DF91CF911F910F91DE
:103ED00008950F931F93082F10E0F801E45BFE4F45
:103EE0008491F801E45BFD4F9491F801E45BFC4F91
:103EF000049110E020E030E0980111270027192BF1
:103F0000082BB801C9011F910F9108951092E5097E
:103F10001092E6091092E2091092E1091092E40968
:103F20001092E3091092EB09089536EC20EE97E029
:103F3000A0E8F7E4E7EE77EF62EE5FB7F89431BB05
:103F4000469A27B99AB92DB915B8A8B99BB91EB820
:103F5000F1BB42E04A95F1F700C046B1B9B1BCB13E
:103F600031BB479AE7B97AB96DB95FBF55E05A9549
:103F7000F1F7000042FFE1CF5FB7F89496EC91BBF8
:103F8000469A382F330F982F9695232F2670206846
:103F9000482F441F4427441F242B80718360432FE4
:103FA000440F4072842B307C832B9270906215B842
:103FB00028B98BB99EB987E881BB85E08A95F1F76E
:103FC00000005FBF0895EF92FF920F93CF93DF93AE
:103FD0001F92CDB7DEB77B016115710539F40F90E3
:103FE000DF91CF910F91FF90EF900895842F298357
:103FF0009CDF298182E0E816F10488F3822F95DFA7
:10400000E2E0EE16F10459F3802F0F90DF91CF918B
:104010000F91FF90EF9089CF26EC90EE87E0F0E8CB
:10402000E7E477EE67EF52EE4FB7F89421BB469A7C
:1040300097B98AB99DB915B8F8B98BB91EB8E1BB63
:1040400032E03A95F1F700C036B1A9B1ACB121BB6D
:10405000479A77B96AB95DB94FBF45E04A95F1F71C
:10406000000032FFE1CF9FB7F89486EC81BB469AFF
:1040700015B887E888B923ED2BB922E22EB981BBA8
:1040800085E08A95F1F700009FBF0895CF938823BC
:1040900039F18091E7098F5F8093E709853148F016
:1040A00081E09091E8099111CDC08093E8091092C8
:1040B000E709C091EB09C11179C05091E5099091D0
:1040C000E609E091EC09E13009F4DEC008F4AFC084
:1040D000E23009F4C4C020E0F0E0EF51F64F24874D
:1040E000AFB7F89456EC51BB469A41E045B980E42D
:1040F00088B91BB880E28EB937E831BB00C000C078
:1041000080E190E00090EC0902C0880F991F0A94AA
:10411000E2F7282F51BB469A782F770F682F6695C4
:10412000221F2227221F972F9670292B206480712F
:10413000972F990F9072982B707C972B627045B9CE
:1041400028B99BB96EB931BB00C000C0E091EC0941
:10415000F0E0EF51F64F848551BB469A582F550F2A
:10416000982F9695252F26702064682F661F662746
:10417000661F262B682F6071852F880F8072862B13
:10418000507C852B9270906245B928B98BB99EB945
:1041900031BBAFBF8091EC0990E0019663E070E025
:1041A0000E94CC6A8093EC09CF9108954091E9096F
:1041B0004F5F4093E909E0EFF9E001900020E9F753
:1041C000E15FF9402091EA09332727FD3095C901C5
:1041D00001966E2F772767FD70950E94CC6AF901D2
:1041E000EF51F64F278530E02038310588F15FEF39
:1041F000E82FFF27E7FDF095EF51F64F278530E0D8
:104200002038310550F5F901E050FF4F90814031E1
:1042100008F457CF8093EA091092E909811151CF30
:104220001C160CF04ECFC150C093EB094ACF209121
:10423000E1098091E809882309F44ECF8091E309D0
:1042400028274ACF80E08093E8091092E70931CF10
:10425000F901E050FF4F5081CBCF9FEFD8CF292FEE
:104260002F778091E1099091E20990FD206880917B
:10427000E3099091E40990FF2FCF8091E80988230A
:1042800009F42ACF205828CF252F2F778091E109D4
:104290009091E20991FD20688091E3099091E409F1
:1042A00091FF1ACFEACF86EC81BB469A15B896E803
:1042B00098B993E09BB91EB897E891BBEFE9FFE08E
:1042C0003197F1F700C0000081BB469A15B823E88A
:1042D00028B923E12BB922E02EB991BBFAE0FA9577
:1042E000F1F700C081BB469A20EE27B997E09AB952
:1042F0002DB915B820E828B99BB91EB897E491BB31
:1043000092E09A95F1F700C096B199B19CB181BB4A
:10431000479A87EE87B987EF8AB982EE8DB9EAE0CE
:10432000EA95F1F700C0089526EC90EE87E0F0E8FA
:10433000E7E477EE67EF52EE4FB7F89421BB469A69
:1043400097B98AB99DB915B8F8B98BB91EB8E1BB50
:1043500032E03A95F1F700C036B1A9B1ACB121BB5A
:10436000479A77B96AB95DB94FBF45E04A95F1F709
:10437000000032FFE1CF8FB7F89496EC91BB469ADC
:1043800015B891E898B993ED9BB990E29EB997E87A
:1043900091BB95E09A95F1F700008FBF0895CF92F9
:1043A000DF92EF92FF928091B70A9091B80AA0E055
:1043B000B0E0E091D90FF091DA0F6F01E12CF12C10
:1043C0008C159D05AE05BF05E4F4A7019601281BD9
:1043D000390B4A0B5B0BA0E0B0E80E945A6FA701B3
:1043E00096010E945E6F2F3F8FE738074105510508
:1043F000FCF02FEF3FE7C901FF90EF90DF90CF90E7
:1044000008959C01AD012C193D094E095F09AFEFDC
:10441000BFE70E944E6F9F012095309540E050E02D
:104420000E945E6F2F3F8FE73807410551050CF75B
:10443000DA01C901811520E892072FEFA207B20720
:104440003CF09C01C901FF90EF90DF90CF90089560
:1044500080E090E8AFEFBFEF9C01F4CF0F931F9384
:10446000382F2091530EE091560E222309F403C1F8
:1044700040916E0E50916F0E60E070E0EE2309F4F3
:10448000F5C08091740E9091750EA0E0B0E03323DA
:10449000A1F0222381F020915C0E25FD0CC000913B
:1044A000B50D1091B60D222717FD2095322F400F24
:1044B000511F621F731FE111E3C02FB7F89441151C
:1044C000510531E06307710524F04FEF5FEF60E0C5
:1044D00070E077FDEAC0BA01672F77276695669589
:1044E000062FE6ECE1BB469A162F110FF12FF6705E
:1044F000F068607177276260312F330F3072362B8E
:10450000107C312B602F66956270606215B8F8B927
:104510003BB96EB967E861BB569547955695479587
:10452000742FE1BB469A142F110FF42FF695771FC5
:104530007727771F312F3670732B7068407155279E
:104540004260312F330F3072342B107C312BF270DC
:1045500015B878B93BB9FEB961BBE1BB469A51E0E9
:1045600055B941E448B970EF7BB932EA3EB961BB55
:10457000E1BB469A55B948B9F0E7FBB93EB961BB12
:1045800000C000C0E1BB469A55B948B97BB93EB9F5
:1045900061BB009731E0A307B10524F08FEF9FEFD7
:1045A000A0E0B0E0B7FD7DC0AC01452F5527469592
:1045B0004695F42F66EC61BB469AE42FEE0F7E2FF2
:1045C000767070684071552742603E2F330F30720D
:1045D000342BE07C3E2B4F2F46954270406215B83D
:1045E00078B93BB94EB937E831BB96958795969522
:1045F0008795482F61BB469A782F770F582F56958D
:10460000441F4427441FE72FE6704E2B40688071FB
:1046100099278260972F990F9072982B707C972B17
:10462000527015B848B99BB95EB931BB61BB469AA7
:1046300041E045B997E498B950EF5BB982EA8EB989
:1046400031BB61BB469A45B998B970E77BB98EB961
:1046500031BB00C000C061BB469A45B998B95BB98F
:104660008EB931BB2FBF1F910F9108958FEF9FEF30
:10467000A0E0B0E00CCF4FEF5FEF60E070E0FECE67
:1046800020915C0E24FD19CF0091B50D1091B60D4F
:10469000222717FD2095322F800F911FA21FB31FD5
:1046A0000CCF80E090E0DC017FCF40E050E0BA0129
:1046B00012CF96EC91BB469A482F440F282F26958F
:1046C000342F36703064982F991F9927991F392BF2
:1046D0008071942F990F9072982B407C942B2270AC
:1046E000206615B838B99BB92EB987E881BB85E03B
:1046F0008A95F1F70000089580959091ED0F892338
:104700008093ED0F96EC91BB469A482F440F282FCB
:104710002695382F331F3327331F942F9670392B4C
:1047200030648071942F990F9072982B407C942B59
:104730002270206C81E085B938B99BB92EB987E821
:1047400081BB85E08A95F1F700008091EC0F8F5FC7
:104750008093EC0F08958091ED0F80618093ED0FB1
:1047600096EC91BB469A382F330F982F9695282FA9
:10477000221F2227221F832F8670282B2064832F3D
:10478000880F80728061307C832B9270906C31E056
:1047900035B928B98BB99EB987E881BB85E08A9580
:1047A000F1F700008091EC0F8F5F8093EC0F08957C
:1047B0008091ED0F81608F7E8093ED0F96EC91BB21
:1047C000469A382F330F982F9695881F8827881F71
:1047D000232F2670822B8064232F220F2072307C9F
:1047E000232B9270906C31E035B988B92BB99EB902
:1047F00087E881BB85E08A95F1F700008091EC0F96
:104800008F5F8093EC0F08952091DE0F27FD09C084
:104810006F7070E0332727FD30956217730709F03A
:104820000895842F90E0489797FD04C040E050E041
:1048300060E012C780E090E0F9CFE091DE0FE7FD85
:1048400009C06F7070E0FF27E7FDF0956E177F07D6
:1048500009F00895842F90E04897422F50E0542F9C
:104860004427550F41505E4F61E0211101C060E0C7
:1048700097FFF2C680E090E0FCCF603E71058105B5
:10488000910508F00895DC01CB019F5FAF4FBF4F4A
:104890006627782F892F9A2F0C9400F88091FF14A7
:1048A000909100158F5F92418130924070F44FEFEC
:1048B00052E16CED70E080E090E0DFDF4FEF53E11C
:1048C0006DED70E080E090E0D8CF089560FD05C008
:1048D0009093120B8093110B0895EFB7F8949C01FD
:1048E000232F332726952695722F46EC41BB469AF7
:1048F000622F660F562F5670506820713327226042
:10490000362F330F3072322B607C362B272F2695B3
:104910002270206215B858B93BB92EB927E821BBDF
:104920009695879596958795382F41BB469A682F1F
:10493000660F582F5695331F3327331F762F767007
:10494000372B3068807199278260962F990F90726B
:10495000982B607C962B527015B838B99BB95EB90C
:1049600021BB41BB469A31E035B995E498B950EF87
:104970005BB980EA8EB921BB65E06A95F1F700006A
:1049800041BB469A35B998B960E76BB98EB921BB7E
:104990006AE06A95F1F700C041BB469A35B998B90B
:1049A0005BB98EB921BB8AE08A95F1F700C0EFBFF1
:1049B000089510921C0B10921B0B08951092160B69
:1049C0001092150B0895CF938091A00B8F3F79F033
:1049D000C82FCF7740E050E060E08C2F3DD66C2FA1
:1049E000685E40E08091DF0FCF910C94B614CF91B8
:1049F00008953F924F925F926F927F928F929F9213
:104A0000AF92BF92CF92DF92EF92FF920F931F93DC
:104A1000CF93DF938091A60B882339F18091A10B6E
:104A20009091A20B01969093A20B8093A10B2091E1
:104A3000A30B3091A40B82179307B8F01092A20B2E
:104A40001092A10BEEE1FBE004C08BE0EE39F80719
:104A500061F081918F3FC9F3B6DF8091A60B823060
:104A600061F1833099F1813089F1DF91CF911F910C
:104A70000F91FF90EF90DF90CF90BF90AF909F90FD
:104A80008F907F906F905F904F903F90089561500E
:104A900071098109910960687F6F8F6F9F6F6F5FE8
:104AA0007F4F8F4F9F4FFB0170939F0B60939E0B27
:104AB000E25EF44F80818F3F21F50E94426F6F7755
:104AC00077278827907897FFEECFE1CF20919E0B34
:104AD00030919F0B07C09C01FC01E25EF44F4081C6
:104AE0004F3F59F4C90101968F77907897FFF3CF24
:104AF000019780689F6F0196EECF80939E0B9093F5
:104B00009F0BA081CFE75C2E5A22E52DE695E69516
:104B1000E695F0E0EE5DF54FA770B0E0A454B94F14
:104B200080819C91892B8083C0905C09D0905D0925
:104B3000E0905E09F0905F098091700A8111A5C133
:104B4000E0916F0ACE2FC170E0FF4CC280913A0A0B
:104B50008111B7C24091320A5091330A6091340AF0
:104B60007091350A4F3FFFEF5F076F077F0709F42A
:104B70003CC290E0AE2FA270E1FF14C08091430AC6
:104B800000913B0A10913C0A20913D0A30913E0A67
:104B900081118BC2041715072607370718F4B901CE
:104BA000A80191E03E2F3470E2FF14C080914C0ABE
:104BB0008090440A9090450AA090460AB090470A17
:104BC000811193C284169506A606B70618F4B5019E
:104BD000A40192E02E2F2870E3FF14C08091550AA3
:104BE00080904D0A90904E0AA0904F0AB090500AC3
:104BF000811187C284169506A606B70618F4B5017A
:104C0000A40193E08E2F8071E4FF14C0F0915E0A3E
:104C10008090560A9090570AA090580AB090590A6E
:104C2000F11137C284169506A606B70618F4B50129
:104C3000A40194E0BE2FB072E5FF17C0E091670AAF
:104C4000EE2309F416C240915F0A5091600A609108
:104C5000610A7091620A4C155D056E057F0528F4A6
:104C60004091660A541609F402C29F3F09F0B1C090
:104C7000CC2309F4C5C15091380AE52FE695E69595
:104C8000E695F0E0EE5DF54F40814111B0C14091F5
:104C9000320A5091330A6091340A7091350A4F3FBD
:104CA000EFEF5E076E077E0709F090E0AA23E1F0C0
:104CB0001091410AE12FE695E695E695F0E0EE5D6C
:104CC000F54FD081D11139C280903B0A90903C0AB7
:104CD000A0903D0AB0903E0A84169506A606B70637
:104CE00018F4B501A40191E03323E1F010914A0AD0
:104CF000E12FE695E695E695F0E0EE5DF54FD08183
:104D0000D11125C28090440A9090450AA090460A8D
:104D1000B090470A84169506A606B70618F4B501A2
:104D2000A40192E02223E1F01091530AE12FE695CD
:104D3000E695E695F0E0EE5DF54FD081D11111C218
:104D400080904D0A90904E0AA0904F0AB090500A61
:104D500084169506A606B70618F4B501A40193E0DB
:104D60008823E1F010915C0AE12FE695E695E6953F
:104D7000F0E0EE5DF54FD081D111FDC18090560A73
:104D80009090570AA090580AB090590A8416950638
:104D9000A606B70618F4B501A40194E0BB23B1F050
:104DA0001091650AE12FE695E695E695F0E0EE5D57
:104DB000F54FD081DD2309F4B0C1E12FE770F0E0B9
:104DC000E454F94FE081ED2309F4A7C19F3F09F4B2
:104DD00089C0312CB8E68B2EBAE09B2E4424439434
:104DE000AA24AA94BA2C052D10E0C6E0D0E0F40164
:104DF00081914F018F3FD1F1692E772467FC709428
:104E0000F301EE0FFF1FEE0FFF1FEE0FFF1FE60D6A
:104E1000F71DEE5DF54F408EB58AA48A568A98013B
:104E2000280F311D278BC08AD18AE28AF38A432D4D
:104E30006FEF7FEF892F72D340916F0A04C0692E04
:104E4000772467FC7094C3010196BE010E94CC6A6E
:104E50009C01982FF901E454F94F8081842379F360
:104E6000FEE68F16FAE09F0609F0C1CF6FEF7FEFE5
:104E7000852D0E949C14E0919E0BF0919F0BE25EA9
:104E8000F44F80818093A00BF0CD80916E0A88232F
:104E900009F4BAC0252D30E0312C823009F426C245
:104EA000813009F4FEC180E090E082179307A1F001
:104EB000E82FE695E695E695F0E0EE5DF54F40814A
:104EC000442351F0FC01E770FF27E454F94F50816F
:104ED000542311F03324339401968038910529F737
:104EE00090E078CFF0916E0ACC2309F44EC1F130F6
:104EF00009F4C6C108F076C14091320A5091330AD4
:104F00006091340A7091350A4F3FEFEF5E076E07EC
:104F10007E0709F090E0AA2309F40FC24A015B0161
:104F200040913B0A50913C0A60913D0A70913E0AC3
:104F3000481559056A057B0508F4A0C1B501A4010F
:104F4000E52D332309F430C18090440A9090450A3E
:104F5000A090460AB090470A84169506A606B706A2
:104F600018F4B501A40192E0222309F467C000916E
:104F70004D0A10914E0A20914F0A3091500A0417A1
:104F800015072607370708F488C18A019B01B90174
:104F9000A801882309F45CC00091560A1091570AB1
:104FA0002091580A3091590A041715072607370728
:104FB00008F49AC18A019B01BB2381F0B901A801C1
:104FC00000915F0A1091600A2091610A3091620A93
:104FD000041715072607370708F449C09F3F09F44F
:104FE00045CFF7CE4FEF5FEFBA019FEFC3CD5770BC
:104FF000E52FF0E0E454F94F5081542309F447CEF3
:105000004FEF5FEFBA0152CE312C90E0E3CEE52DA9
:105010004FEF5FEFBA01332309F4C6C0F13009F452
:105020000BC108F491CFF23009F0BEC030914B0AA9
:105030003E1710F4E32F92E02111C1C0882341F004
:10504000F13009F40BC108F4A7CFF23009F4C0C065
:10505000BB2321F2F13009F40AC108F4B1CFF230D8
:1050600009F0BCCF8091660A8E1708F0B7CF95E0A3
:10507000B0CE80905F0A9090600AA090610AB090D4
:10508000620A84169506A606B70608F0EECD95E0EE
:10509000A0CE8C149D04AE04BF0408F0CBCDF091DB
:1050A0005D0A5F12C7CD94E094CE0C151D052E0548
:1050B0003F0508F077CD8091420A581273CD91E0F8
:1050C00088CE8091320A9091330AA091340AB0912F
:1050D000350A8C159D05AE05BF0508F083CF80917C
:1050E000390A58127FCF90E074CE8C149D04AE0420
:1050F000BF0408F06FCD80914B0A58126BCD92E03F
:1051000068CE8C149D04AE04BF0408F07BCD809162
:10511000540A581277CD93E05CCE80905F0A90904D
:10512000600AA090610AB090620A84169506A606ED
:10513000B70608F04BCE95E04CCEE12FE770F0E0DB
:10514000E454F94FE081ED2309F0CECDBDCDE12F40
:10515000E770F0E0E454F94FE081ED2309F0E2CD8F
:10516000D1CDE12FE770F0E0E454F94FE081ED2379
:1051700009F0F6CDE5CDE12FE770F0E0E454F94F0A
:10518000E081ED2309F00ACEF9CDAA2309F43FCF3F
:10519000F13009F444C0F0F588248A94982C540125
:1051A000BFCE4FEF5FEFBA01222309F447CFF130B2
:1051B00009F44BC008F4DBCEF23009F03FCF209168
:1051C000540A2E1710F4E22F93E0882309F440CFFD
:1051D00080915D0A8E1710F4E82F94E0BB2309F448
:1051E000FDCE40CFF23089F6E091390AE51508F49A
:1051F000A2C0E52DAA2309F44AC04E2FE091420A2D
:10520000E41708F496C0E42F332359F24FEF5FEF11
:10521000BA010CCFF23009F0FACE452DEFCFE52DD3
:105220004091420AE417B8F14E2FE42F332309F4DA
:10523000B8CF4FEF5FEFBA0130914B0AE31710F48C
:10524000E32F92E0222309F4F9CE2091540AE217C9
:1052500010F4E22F93E0882309F4FACE80915D0ADE
:10526000E81710F4E82F94E0BB2309F4B7CE80913F
:10527000660AE81708F0B2CE95E0ABCD91E060CEBB
:10528000E091390A5E1658F0E52DA111C9CF4FEF14
:105290005FEFBA01C0CE91E0C8CF93E078CE90E046
:1052A000F4CF80E090E082179307C1F0E82FE695F5
:1052B000E695E695F0E0EE5DF54F4081442371F010
:1052C000FC01E770FF27E454F94F5081542331F07B
:1052D000821793070CF4CACD332433940196803897
:1052E000910509F790E076CD94E066CE80E090E0FD
:1052F00082179307C1F0E82FE695E695E695F0E072
:10530000EE5DF54F4081442371F0FC01E770FF270B
:10531000E454F94F5081542331F0281739070CF425
:10532000A5CD3324339401968038910509F790E098
:1053300051CD91E069CF90E05DCFE52D6CCECF935C
:105340004FB7F89436EC31BB469A80EE87B997E0B8
:105350009AB98DB981E085B980E488B91BB880E23B
:105360008EB987E481BB52E05A95F1F700C026B1AF
:1053700099B18CB131BB479AC22FC695C37050E822
:10538000259F90011124C22B292F2071C22B292F78
:10539000269526952870C22B96959076C92B90E07D
:1053A000880F991F84709927C82B87EE87B987EFDC
:1053B0008AB982EE8DB94FBF8091620E882331F099
:1053C000C5FD04C08091EA0F85FD45C08091A60B04
:1053D000882351F18091EA0F8C2785FF25C0C5FFF6
:1053E00013C08091A50B882309F441C0EEE1FBE0D6
:1053F0009FEF05C031965BE0EE39F507C1F1808182
:1054000087FFF8CF9083F6CF8091A50B823049F0CB
:10541000EEE1FBE08081806881938BE0EE39F80754
:10542000C9F782E08093A50B8091E10F823021F0D3
:10543000C093EA0FCF910895C0FFFACF8091EA0F91
:1054400080FDF6CF8091500E8F5F8093500EC093F9
:10545000EA0FCF9108950E94021A86E0E8E6FAE08A
:10546000A6EABEE001900D928A95E1F7DDCF80E0DB
:10547000D9CFCF93DF93D82FC62F8091A60B8D174E
:10548000C1F0A1DA2FEF3FEF30939F0B20939E0BDB
:105490008FEF8093A00B40E850E06FEF70E08EE15B
:1054A0009BE00E94DE6E0E9453198091E10F8111F2
:1054B0002EC08091A50B8C17A1F0EEE1FBE0C1118D
:1054C00017C02FEF05C031968BE0EE39F80749F091
:1054D000908197FFF8CF208331968BE0EE39F80763
:1054E000B9F7D093A60BC093A50BDF91CF91089588
:1054F0009081906891938BE0EE39F80791F3908159
:10550000906891938BE0EE39F80791F7EACF2FEF8F
:105510003FE73093A20B2093A10BCBCFAF92BF926A
:10552000CF92DF92EF92FF920F931F93CF93DF936F
:105530001F92CDB7DEB7D82E7B0149830E94D21BC4
:105540006D2D81E00E94EC534981442329F0809124
:10555000A60B882309F471C08D2D9AE2890280017F
:10556000112487EAA82E8BE0B82EA00EB11EF501FB
:10557000148215821682178264A175A1CB01A0E066
:10558000B0E0772766272689378940E050E00E94FF
:10559000856FF501378F268FCC24C394C1A6C50132
:1055A0000E940B4DF501C7A233EAA32E3CE0B32EB7
:1055B000A00EB11EF501148215821682178206898B
:1055C000178964A175A1CB01A0E0B0E07727662719
:1055D000980140E050E00E94856FB901F501378FD6
:1055E000268FC1A6AA27209FB12D319FC001129FEF
:1055F000B00D811D9A1F309FB00D811D9A1F11247F
:1056000080A391A360957095AA27609FB12D719F8B
:10561000C001169FB00D811D9A1F709FB00D811D96
:105620009A1F112482A393A380859185A285B385B7
:1056300080839183A283B383C7A2B7018D2D0F907E
:10564000DF91CF911F910F91FF90EF90DF90CF905E
:10565000BF90AF900C94A53B2F923F924F925F92D8
:105660006F927F928F929F92AF92BF92CF92DF9272
:10567000EF92FF920F931F93CF93DF9300D000D050
:10568000CDB7DEB7782E642E552E869586958695F5
:1056900090E0E72DE770F0E0E454F94F2081FC0141
:1056A000EE5DF54F662309F440C08081822B808334
:1056B00090E0C0905C09D0905D09E0905E09F090A8
:1056C0005F098091700A882309F48FC080916E0A67
:1056D000882309F431C2272D30E0392E823009F4B5
:1056E000B0C7813011F40C94753380E090E0632DE5
:1056F0008217930799F0E82FE695E695E695F0E096
:10570000EE5DF54F4081442349F0FC01E770FF272F
:10571000E454F94F5081542309F061E00196803838
:10572000910531F7362E90E0A4C120958081282381
:105730002083D0903A0AC090380A8C2C912C00918A
:10574000430A6090410AE62CF12CE0914C0A5090FB
:105750004A0A252D30E02090550A4090530A642DC6
:1057600070E0B0915E0A30905C0A432D50E01091D9
:10577000670A8091650A8983A82EB12C80916E0AF0
:10578000823009F47FC280E090E0D110D8C11111BD
:10579000E1C3011107C5EE2EA82FE82FE695E69587
:1057A000E695F0E0EE5DF54FF080FF2009F494C33C
:1057B000FC01E770FF27E454F94FE081EF2109F481
:1057C0008BC3EE2021F02817390709F485C3222066
:1057D00021F06817790709F47FC3BB2321F048172C
:1057E000590709F479C3EE2DE0C1E0916F0AAE2F9D
:1057F000A170E0FF17C080913A0A882309F42DC3F5
:105800004091320A5091330A6091340A7091350AFE
:105810004C155D056E057F0528F48091390A7816D0
:1058200009F4AFC70FEF1FEF98019FEF4E2F4270A3
:10583000E1FF17C08091430A80903B0A90903C0A98
:10584000A0903D0AB0903E0A882309F4FCC28C1453
:105850009D04AE04BF0428F48091420A781609F42E
:1058600092C78E2F8470E2FF17C050914C0A80902F
:10587000440A9090450AA090460AB090470A5523E2
:1058800009F406C38C149D04AE04BF0428F450919F
:105890004B0A751609F473C75E2F5870E3FF17C0E3
:1058A0006091550A80904D0A90904E0AA0904F0A40
:1058B000B090500A662309F4E1C28C149D04AE0432
:1058C000BF0428F46091540A761609F456C76E2F67
:1058D0006071E4FF17C070915E0A8090560A909044
:1058E000570AA090580AB090590A772309F4DAC2EF
:1058F0008C149D04AE04BF0428F470915D0A7716E1
:1059000009F439C77E2F7072E5FF17C0E091670A6E
:10591000EE2309F4D1C200915F0A1091600A209130
:10592000610A3091620A0C151D052E053F0528F409
:105930002091660A721609F4CDC29F3F09F098C003
:10594000A11183C10FEF1FEF98014423E1F0B09044
:10595000410AEB2DE695E695E695F0E0EE5DF54F14
:10596000B081B11126C380903B0A90903C0AA09070
:105970003D0AB0903E0A80169106A206B30618F4BE
:105980009501840191E08823E1F0B0904A0AEB2D63
:10599000E695E695E695F0E0EE5DF54FB081B11144
:1059A0002CC38090440A9090450AA090460AB0907B
:1059B000470A80169106A206B30618F495018401E1
:1059C00092E05523E1F0B090530AEB2DE695E69571
:1059D000E695F0E0EE5DF54FB081B11122C3809005
:1059E0004D0A90904E0AA0904F0AB090500A80162F
:1059F0009106A206B30618F49501840193E066238C
:105A0000E1F0B0905C0AEB2DE695E695E695F0E0C6
:105A1000EE5DF54FB081B111D6C28090560A9090DC
:105A2000570AA090580AB090590A80169106A2060B
:105A3000B30618F49501840194E07723B1F0B09097
:105A4000650AEB2DE695E695E695F0E0EE5DF54FFF
:105A5000B081BB2309F4C1C2EB2DE770F0E0E45440
:105A6000F94FE081EB2309F4B8C29F3F09F4C5C3A5
:105A7000312C28E63AE044244394A72CB12C76E05C
:105A8000872E912C3C832B83592FEB81FC818191B4
:105A9000FC83EB838F3FC9F1052F112707FD10957C
:105AA000F801EE0FFF1FEE0FFF1FEE0FFF1FE00FBD
:105AB000F11FEE5DF54F408E648A558A768A950116
:105AC000280F311D278BC08AD18AE28AF38A432DA1
:105AD000662D752D852F22DD20916F0A04C0082FB9
:105AE000112707FD1095C8010196B4010E94CC6AE8
:105AF000582FFC01E454F94F3081322381F38B811C
:105B00009C818E569A4009F0C0CF0F900F900F9055
:105B10000F90DF91CF911F910F91FF90EF90DF9049
:105B2000CF90BF90AF909F908F907F906F905F903D
:105B30004F903F902F900895392E90E09ACF011109
:105B4000D7C1EE2E111157C0A82FE82FE695E69584
:105B5000E695F0E0EE5DF54FF080FF2009F4C2C15C
:105B6000FC01E770FF27E454F94FE081EF2109F4CD
:105B7000B9C18816990609F4B5C1EE2021F028179D
:105B8000390709F4AFC1222021F06817790709F419
:105B9000A9C1BB2321F04817590709F4A3C1EE2D71
:105BA000DD2019F0C71409F492C28FEF9FEF002394
:105BB00019F0671409F477C2EE2319F0571409F4A9
:105BC00077C2222019F0471409F477C2BB2319F0D9
:105BD000371409F477C2112321F02981271509F41C
:105BE0005DC2682E592E7A2E91E063CD01968038E1
:105BF000910509F485C0A82FE82FE695E695E6956E
:105C0000F0E0EE5DF54FF080FF2081F3FC01E770DE
:105C1000FF27E454F94FE081EF2141F388169906FC
:105C200029F3EE2019F02817390701F3222019F083
:105C300068177907D9F2BB2319F048175907B1F251
:105C4000A816B90609F0ABCFD1CF3091380AE32FAF
:105C5000E695E695E695F0E0EE5DF54F20812111A1
:105C6000D6C10091320A1091330A2091340A309142
:105C7000350A0F3FEFEF1E072E073E0709F465CEEA
:105C800090E063CE8FE790E0222009F4D4C1EE23A8
:105C900009F417C30111F5C3EE2EA82FE82FE695DE
:105CA000E695E695F0E0EE5DF54FF080FF2009F413
:105CB00068C3FC01E770FF27E454F94FE081EF214E
:105CC00009F45FC3DD2021F08816990609F459C351
:105CD0002817390709F455C36817790709F451C320
:105CE000BB2321F04817590709F44BC3112321F0B6
:105CF000A816B90609F445C3EE2DAF3F09F050CF01
:105D0000DD20A1F0C71012C00E94D21B60E081E02C
:105D10000E94EC5360E087EA9BE00E94354460E01B
:105D200083EA9CE00E9435440091430A0023A1F0DD
:105D30008091410A871110C00E94D21B61E081E06E
:105D40000E94EC5360E081ED9BE00E94354460E0EE
:105D50008DEC9CE00E94354480914C0A8823A1F090
:105D600080914A0A871110C00E94D21B62E081E034
:105D70000E94EC5360E08BEF9BE00E94354460E0B2
:105D800087EF9CE00E9435448091550A8823A1F05A
:105D90008091530A871110C00E94D21B63E081E0FA
:105DA0000E94EC5360E085E29CE00E94354460E094
:105DB00081E29DE00E94354480915E0A8823A1F033
:105DC00080915C0A871110C00E94D21B64E081E0C0
:105DD0000E94EC5360E08FE49CE00E94354460E058
:105DE0008BE49DE00E9435448091670A882309F482
:105DF0008CCE8091650A871188CE0E94D21B65E007
:105E000081E00E94EC5360E089E79CE00E94354409
:105E100060E085E79DE00F900F900F900F90DF916D
:105E2000CF911F910F91FF90EF90DF90CF90BF9097
:105E3000AF909F908F907F906F905F904F903F902A
:105E40002F900C94354480169106A206B30608F0F4
:105E500008CD9501840191E004CD0091320A1091A2
:105E6000330A2091340A3091350A0F3F6FEF16073D
:105E70002607360709F4D9CC90E0D8CC80169106D5
:105E8000A206B30608F023CD9501840193E01FCD4F
:105E900080169106A206B30608F0FECC9501840197
:105EA00092E0FACC80169106A206B30608F02ACD3D
:105EB0009501840194E026CD80905F0A9090600A5D
:105EC000A090610AB090620A80169106A206B306FD
:105ED00008F033CD95E0CCCD01968038910509F0DE
:105EE0005BCC24CF01968038910509F02DCE08CFE8
:105EF000E111F2C0EA83A82FE82FE695E695E69532
:105F0000F0E0EE5DF54F20812223F9F0FC01E7700F
:105F1000FF27E454F94F30813223B9F088169906EF
:105F2000A1F0E816F90689F0222019F06817790720
:105F300061F0BB2319F04817590739F0112319F004
:105F4000A816B90611F0EA812BCE0196803891058A
:105F500091F6D6CEB111F6C0DE2EA82FE82FE69529
:105F6000E695E695F0E0EE5DF54F40814423E1F0E3
:105F7000FC01E770FF27E454F94F50815423A1F04E
:105F8000002319F0E816F90679F0DD2019F028173A
:105F9000390751F0211005C0A816B90629F0ED2DDA
:105FA00004CE68177907C1F7019680389105A9F6E4
:105FB000BDCEEB2DE770F0E0E454F94FE081EB2328
:105FC00009F0E1CCD0CCEB2DE770F0E0E454F94FD0
:105FD000E081EB2309F031CD20CD80905F0A9090D5
:105FE000600AA090610AB090620A80169106A2062B
:105FF000B30608F03ACD95E03BCDEB2DE770F0E02D
:10600000E454F94FE081EB2309F0DBCCCACC3770C4
:10601000E32FF0E0E454F94F3081322309F092CCC1
:1060200020CEEB2DE770F0E0E454F94FE081EB2354
:1060300009F0E5CCD4CCDD2009F471C10111F2C125
:10604000FE2EA82FE82FE695E695E695F0E0EE5DAA
:10605000F54F6081662309F48CC1FC01E770FF27CE
:10606000E454F94F7081762309F483C188169906A8
:1060700009F47FC1FF2021F02817390709F479C1FD
:10608000BB2321F04817590709F473C1112321F0EC
:10609000A816B90609F46DC1EF2D2FCE8091630AC1
:1060A0009091640A9ECD80913F0A9091400A84CDE0
:1060B0008091480A9091490A84CD8091510A90912B
:1060C000520A84CD80915A0A90915B0A84CD8091C6
:1060D000360A9091370A6BCDEB832A82A82FE82FDE
:1060E000E695E695E695F0E0EE5DF54F20802220FE
:1060F00021F1FC01E770FF27E454F94FE081E22130
:10610000E1F088159905C9F08E159F05B1F0821749
:10611000930799F0FA81FF2319F08617970769F022
:10612000BB2319F08417950741F0112319F08A1544
:106130009B0519F0EB812A8033CD019680389105BB
:1061400069F6DECDCE2EA82FE82FE695E695E695EA
:10615000F0E0EE5DF54FD080DD20F9F0FC01E77056
:10616000FF27E454F94FE081ED21B9F0002319F045
:106170008E159F0591F0CC2019F08217930769F0D6
:10618000222019F08617970741F08417950729F008
:106190008A159B0511F0EC2D08CD019680389105EC
:1061A00091F6C4CDCE2EA82FE82FE695E695E6957C
:1061B000F0E0EE5DF54FD080DD20D1F0FC01E7701E
:1061C000FF27E454F94FE081ED2191F0E816F9063C
:1061D00079F0CC2019F02817390751F0222019F056
:1061E0006817790729F0BB23B1F24817590799F6C8
:1061F000019680389105B9F699CDE0916E0AAA23EF
:1062000009F4C3C0E13009F494C208F000C200915F
:10621000320A1091330A2091340A3091350A0F3F27
:10622000FFEF1F072F073F0709F090E04111B8C0AB
:10623000F72D882309F4C9C0E13009F42CC208F015
:10624000C3C18090440A9090450AA090460AB0903D
:10625000470A80169106A206B30618F49501840138
:1062600092E0552309F4BBC080904D0A90904E0AED
:10627000A0904F0AB090500A80169106A206B3066D
:1062800008F403C2480159016111B3C095018401AA
:10629000772399F0E13009F419C208F0B4C14091B4
:1062A0005F0A5091600A6091610A7091620A40171A
:1062B00051076207730708F40DCE9F3F09F425CC00
:1062C000D7CBD1103DC19E2EA82FE82FE695E6959D
:1062D000E695F0E0EE5DF54F2081222309F44DC0F4
:1062E000FC01E770FF27E454F94F3081322309F4B1
:1062F00044C0002321F0E816F90609F43EC06817EF
:10630000790709F43AC0BB2319F048175907A9F1D6
:10631000112319F0A816B90681F1E92DEECC11115F
:10632000E3C0BE2EA82FE82FE695E695E695F0E0AF
:10633000EE5DF54F60816623C9F0FC01E770FF2731
:10634000E454F94F7081762389F0002319F0E816A0
:10635000F90661F0BB2019F02817390739F0BB2383
:1063600019F04817590711F0EB2DC7CC0197D0F65B
:10637000DDCC019708F065CEC3CC019708F0A4CF1F
:10638000D5CC019708F089CCBBCC442309F445C097
:10639000E13009F4E3C108F02FC10FEF1FEF9801BE
:1063A00080903B0A90903C0AA0903D0AB0903E0A33
:1063B00080169106A206B30608F493C1480159015C
:1063C00095018401F72D81113CCF552341F0E13037
:1063D00009F46AC108F448CFE23009F402C1662327
:1063E00009F456CFE13009F468C108F0D9C048017A
:1063F00059010091560A1091570A2091580A30917C
:10640000590A081519052A053B0508F4A9C1950183
:106410008401772309F451CF42CFF72D0FEF1FEFFF
:10642000980107CFEA83A82FE82FE695E695E69531
:10643000F0E0EE5DF54F6081662301F1FC01E7704D
:10644000FF27E454F94F70817623C1F0881699062E
:10645000A9F0E816F90691F06A81662319F0281769
:10646000390761F0BB2319F04817590739F0112398
:1064700019F0A816B90611F0EA813FCC019798F6F9
:106480003FCCEB832A82A82FE82FE695E695E69588
:10649000F0E0EE5DF54F2080222019F1FC01E7705D
:1064A000FF27E454F94FE081E221D9F0DD2019F013
:1064B00088159905B1F08E159F0599F082179307FD
:1064C00081F08617970769F0BB2319F084179507A9
:1064D00041F0112319F08A159B0519F0EB812A80F0
:1064E0000CCC019780F60CCC9E2E03C0019708F4CB
:1064F0001DCCA82FE82FE695E695E695F0E0EE5D39
:10650000F54F6081662391F3FC01E770FF27E454A7
:10651000F94F7081762351F3002319F0E816F9063C
:1065200029F3992019F02817390701F3BB2319F033
:1065300048175907D9F2A816B906C1F2E92DDDCBE3
:10654000EA8307C0A816B90609F096CF019708F4A8
:10655000D7CBA82FE82FE695E695E695F0E0EE5D1F
:10656000F54F2081222391F3FC01E770FF27E454CB
:10657000F94F3081322351F38816990639F30023FD
:1065800019F0E816F90611F368177907F9F2BB2339
:1065900019F048175907D1F21111D4CFEA81ADCBC8
:1065A000E23009F075CE80915D0A8F1708F46FC054
:1065B0008F2F772309F481CEF82F8091660A8F17E9
:1065C00008F07BCE95E054CAE23009F0FECE4F2FA2
:1065D000F0914B0AF41708F45CC0F42F552309F42A
:1065E000FECE8091540A8F1708F47DC08F2FF82FAC
:1065F000662309F44DCED7CFF72DE23091F00FEF9F
:106600001FEF980116CEE23009F057CED6CFE23018
:1066100009F0BBCEF091390AF71578F0F72D442335
:1066200071F34091420A4F1750F04F2F882309F41D
:106630009DC00FEF1FEF9801CBCF90E0F0CF91E01E
:10664000F5CF80E090E0632D06C061E001968038D0
:10665000910509F467C882179307C1F3E82FE695FF
:10666000E695E695F0E0EE5DF54F4081442371F349
:10667000FC01E770FF27E454F94F5081542331F3B4
:10668000281739070CF441CAE0CF93E0FDCD94E020
:1066900090CF92E0A3CF8F2FF0914B0A8F17F8F095
:1066A000F82F552309F49BCE8091540AF81710F463
:1066B000F82F93E0662309F4EBCD80915D0AF8177B
:1066C00060F08F2F772309F4F8CDF82F8091660AB8
:1066D000F81708F0F2CD95E0CBC994E0F3CF92E043
:1066E000E0CF91E06DCE93E082CF80E090E0632D2B
:1066F00006C061E001968038910509F413C882173D
:106700009307C1F3E82FE695E695E695F0E0EE5D98
:10671000F54F4081442371F3FC01E770FF27E454F7
:10672000F94F5081542331F3821793070CF4EDC9CC
:10673000E0CFF091390A7F16B8F0F72D442309F421
:106740005ECF2F2FF091420A2F1760F0F22F88238F
:1067500071F08F2F0FEF1FEF98019ECF272DF2CFF3
:1067600094E057CE91E0F3CF90E0E8CFF42F0FEF15
:106770001FEF98012ACE94E07BC993E079C992E09B
:1067800077C990E075C991E073C990911D0B977F0F
:106790008111986090931D0B4FB7F89480911D0B59
:1067A00096EC91BB469A382F330F982F9695232F4E
:1067B00026702064582F551F5527551F252B582FFD
:1067C0005071832F880F8072852B307C832B9270C1
:1067D000906631E035B928B98BB99EB987E881BB9D
:1067E0004FBF089590911D0B9D7F811192609093F2
:1067F0001D0B4FB7F89480911D0B96EC91BB469AF8
:10680000382F330F982F9695232F26702064582FFA
:10681000551F5527551F252B582F5071832F880F33
:106820008072852B307C832B9270906631E035B975
:1068300028B98BB99EB987E881BB4FBF0895809175
:106840001D0B8E7F9091510E9111816080931D0BD5
:106850004FB7F89480911D0B96EC91BB469A382F58
:10686000330F982F9695232F26702064582F551F8D
:106870005527551F252B582F5071832F880F807255
:10688000852B307C832B9270906631E035B928B926
:106890008BB99EB987E881BB4FBF80911D0B877F65
:1068A0009091540E9111886080931D0B4FB7F8940E
:1068B00080911D0B96EC91BB469A382F330F982F81
:1068C0009695232F26702064582F551F5527551F46
:1068D000252B582F5071832F880F8072852B307C89
:1068E000832B9270906631E035B928B98BB99EB987
:1068F00087E881BB4FBF80911D0B8D7F9091520E19
:106900009111826080931D0B4FB7F89480911D0BFD
:1069100096EC91BB469A382F330F982F9695232FDC
:1069200026702064582F551F5527551F252B582F8B
:106930005071832F880F8072852B307C832B92704F
:10694000906631E035B928B98BB99EB987E881BB2B
:106950004FBF80911D0B8F7E9091550E91118061DC
:1069600080931D0B4FB7F89480911D0B96EC91BB53
:10697000469A382F330F982F9695232F2670206430
:10698000582F551F5527551F252B582F5071832FD2
:10699000880F8072852B307C832B9270906631E05B
:1069A00035B928B98BB99EB987E881BB4FBF8091B3
:1069B0001D0B8B7F9091570E9111846080931D0B5E
:1069C0004FB7F89480911D0B96EC91BB469A382FE7
:1069D000330F982F9695232F26702064582F551F1C
:1069E0005527551F252B582F5071832F880F8072E4
:1069F000852B307C832B9270906631E035B928B9B5
:106A00008BB99EB987E881BB4FBF80911D0B8F7DED
:106A10009091580E9111806280931D0B4FB7F8949E
:106A200080911D0B96EC91BB469A382F330F982F0F
:106A30009695232F26702064582F551F5527551FD4
:106A4000252B582F5071832F880F8072852B307C17
:106A5000832B9270906631E035B928B98BB99EB915
:106A600087E881BB4FBF80911D0B8F7B9091590EA2
:106A70009111806480931D0B4FB7F89480911D0B8A
:106A800096EC91BB469A382F330F982F9695232F6B
:106A900026702064582F551F5527551F252B582F1A
:106AA0005071832F880F8072852B307C832B9270DE
:106AB000906631E035B928B98BB99EB987E881BBBA
:106AC0004FBF08958091220A9091230A892B9091BB
:106AD000240A892B9091250A892B9091260A892BCB
:106AE0009091270A892B9091280A892B9091290A45
:106AF000892B90912A0A892B90912B0A892B9091AE
:106B00002C0A892B90912D0A892B90912E0A892B82
:106B100090912F0A892B9091300A892B9091310AFC
:106B2000982B21E009F420E080914C0A9091430ACF
:106B3000892B9091550A892B90915E0A892B90910F
:106B40003A0A892B9091670A892B59F48FEF9FEFAE
:106B5000DC0180934A0E90934B0EA0934C0EB093A1
:106B60004D0E222329F08091EB0F882309F4D2C027
:106B70002093EB0F0E94BA1B62DE8091620E81119E
:106B8000DAC00E94E5199091E00F80916F0A981782
:106B900009F457C010923A0A8FEF8093390A809314
:106BA000380A1092320A1092330A1092340A109264
:106BB000350A1092430A8093420A8093410A109248
:106BC0003B0A10923C0A10923D0A10923E0A109223
:106BD0004C0A80934B0A80934A0A1092440A1092FE
:106BE000450A1092460A1092470A1092550A80935D
:106BF000540A8093530A10924D0A10924E0A109232
:106C00004F0A1092500A10925E0A80935D0A809398
:106C10005C0A1092560A1092570A1092580A109263
:106C2000590A1092670A8093660A8093650A109247
:106C30005F0A1092600A1092610A1092620A9093A1
:106C40006F0A9091630E80916E0A981709F459C0EB
:106C500010923A0A8FEF8093390A8093380A109283
:106C6000320A1092330A1092340A1092350A1092A6
:106C7000430A8093420A8093410A10923B0A109281
:106C80003C0A10923D0A10923E0A10924C0A8093E0
:106C90004B0A80934A0A1092440A1092450A1092B5
:106CA000460A1092470A1092550A8093540A80931C
:106CB000530A10924D0A10924E0A10924F0A1092E7
:106CC000500A10925E0A80935D0A80935C0A1092CB
:106CD000560A1092570A1092580A1092590A1092A6
:106CE000670A8093660A8093650A10925F0A109281
:106CF000600A1092610A1092620A933048F49093ED
:106D00006E0A0E94A14462D50E944F170C946F4FE7
:106D100090E0F5CF80915C0990915D09A0915E09AA
:106D2000B0915F0980934A0E90934B0EA0934C0E46
:106D3000B0934D0E1DCF61E086EA9EE00E94A91936
:106D400022CFE82FF0E0EF59F64F9081917080321A
:106D500009F456C078F0843209F44CC0A0F18632B0
:106D600009F445C008F058C09093580E81E0809314
:106D7000AE0EA8CE8C31C8F08C3109F444C080919D
:106D80007E09817090915C0E9073892B90917F09A0
:106D900090FD47C090E0892B9091800990FF45C0FD
:106DA00092E0892B80935C0EE1CF8A31A8F080912C
:106DB0007C09817090917B0990FD35C090E0892B12
:106DC00080935D0ED3CF8232C1F018F09093540EB1
:106DD000CDCF9093520ECACF883131F0893109F06E
:106DE00008959093560EC2CF9093530EBFCF9093B9
:106DF000590EBCCF9093550EB9CF9093570EB6CF86
:106E00009093510EB3CF90917D0980915A0E90FBD3
:106E100080F980935A0EAACF873211F79093620EB1
:106E2000A5CF98E0B8CF92E0CACF90E0BACFCF9389
:106E3000C8E18C2F86DFCF5FC832D9F7CF91089594
:106E40008091DD0F8823C9F08091DB0F9091DC0FDA
:106E50000E943D1D8823B9F08091DD0F8823D1F079
:106E60000E944E1A1092AE0E81E09091DD0F9111AA
:106E700001C080E08093AC0E08958BED90E00E94FD
:106E80003D1D8111E9CF81E00E94A81D8091DD0F99
:106E90008111E6CFCCDF8091AE0E20E0E22FF0E052
:106EA000DF01AC58B94FAC91AF3F69F0EE0FFF1F57
:106EB000EF5AF14FAA0FBB0BA956B54F8D919C917C
:106EC000928F818F81E02F5F2E3141F78093AE0E3C
:106ED000C7CF90911D0B9B7F8111946090931D0BE8
:106EE0004FB7F89480911D0B96EC91BB469A382FC2
:106EF000330F982F9695232F26702064582F551FF7
:106F00005527551F252B582F5071832F880F8072BE
:106F1000852B307C832B9270906631E035B928B98F
:106F20008BB99EB987E881BB4FBF0895FC012689C4
:106F300037892617370721F0778B668B0C94D4415D
:106F4000089590911D0B9F7B8111906490931D0B70
:106F50004FB7F89480911D0B96EC91BB469A382F51
:106F6000330F982F9695232F26702064582F551F86
:106F70005527551F252B582F5071832F880F80724E
:106F8000852B307C832B9270906631E035B928B91F
:106F90008BB99EB987E881BB4FBF089590911D0BB7
:106FA0009F7D8111906290931D0B4FB7F894809153
:106FB0001D0B96EC91BB469A382F330F982F969560
:106FC000232F26702064582F551F5527551F252B1A
:106FD000582F5071832F880F8072852B307C832B24
:106FE0009270906631E035B928B98BB99EB987E8BF
:106FF00081BB4FBF089590911D0B9F7E81119061C1
:1070000090931D0B4FB7F89480911D0B96EC91BB9C
:10701000469A382F330F982F9695232F2670206489
:10702000582F551F5527551F252B582F5071832F2B
:10703000880F8072852B307C832B9270906631E0B4
:1070400035B928B98BB99EB987E881BB4FBF089580
:10705000DF92EF92FF920F931F93CF93DF93EDEDAB
:10706000FAE0D0E048E050E0C6ECB7E811E000EF0D
:10707000819191917D2F786F2D2F269526952695BC
:107080007A0102C0EE0CFF1C2A95E2F76E2D609586
:107090006723FFB6F8949C01232F33272695269566
:1070A000D22EC1BB469AE22EEE0CAE2DA670A06881
:1070B0002071332722603E2D330F3072322B2E2D5C
:1070C000207C322B2D2D26952270206215B8A8B970
:1070D0003BB92EB9B1BB9695879596958795282F84
:1070E000C1BB469AA82FAA0F382F3695221F2227F8
:1070F000221F0F2EF6E0EF2EF02DEA222E29206817
:107100008071992782609A2F990F9072982BA07C9A
:107110009A2B327015B828B99BB93EB9B1BBC1BB27
:10712000469A372F330F36703164972F96959270A9
:10713000906A15B938B90BB99EB9B1BB85E08A958B
:10714000F1F70000C1BB469A262F220F762F7695C5
:10715000A62FAA1FAA27AA1F822F8670A82BA06479
:107160006071822F880F8072862B207C822B727038
:10717000706A15B9A8B98BB97EB9B1BB8AE08A9596
:10718000F1F700C0C1BB469A15B938B90BB99EB921
:10719000B1BB8AE08A95F1F700C0FFBEDF5FD03255
:1071A00009F066CF4FB7F89480911D0B96EC91BB18
:1071B000469A382F330F982F9695232F26702064E8
:1071C000582F551F5527551F252B582F5071832F8A
:1071D000880F8072852B307C832B9270906631E013
:1071E00035B928B98BB99EB987E881BB4FBFDF910C
:1071F000CF911F910F91FF90EF90DF9008956091D4
:10720000EF0F663028F46F5C81E60E9419190BC0FD
:107210006C3028F4655D82E60E94191904C06B5D2C
:1072200086E60E94191981E00E94462011CF9F92A4
:10723000AF92BF92CF92DF92EF92FF920F931F9384
:10724000CF93DF93D82FCEE1DADFC150E9F7109268
:10725000ED0F1092EC0F6AE081E10E9444130E944E
:10726000AA15C12CD12C7601DD2309F4E4C016EC5B
:10727000C0EE87E0982EAA24A39490E4B92E00E2F1
:107280000E94A0130E94741380E492E4AFE0B0E087
:1072900067E457EE47EF32EE05C00097A105B10550
:1072A00009F4DAC011BB469AC7B99AB8CDB9A5B8E6
:1072B000B8B81BB80EB961BB22E02A95F1F700C03F
:1072C00026B179B17CB111BB479A57B94AB93DB9DA
:1072D0000197A109B10922FDE0CF892B8A2B8B2BC5
:1072E00009F4BAC00E94D82340E452E46FE070E091
:1072F000E7E437EE27EF92EE06C041155105610530
:10730000710509F4ACC011BB469AC7B99AB8CDB99A
:10731000A5B8B8B81BB80EB9E1BB82E08A95F1F701
:1073200000C086B1F9B1FCB111BB479A37B92AB98F
:107330009DB9415051096109710982FFDECF452B8A
:10734000462B472B09F48BC00E94AB2340E452E448
:107350006FE070E0E7E437EE27EF92EE06C04115EC
:1073600051056105710509F47DC011BB469AC7B985
:107370009AB8CDB9A5B8B8B81BB80EB9E1BB82E0D0
:107380008A95F1F700C086B189B18CB111BB479ADB
:1073900037B92AB99DB9415051096109710981FD77
:1073A000DECF452B462B472B09F45CC080E10E94C1
:1073B0007C230E94AB2340E452E46FE070E0E7E4FA
:1073C00037EE27EF92EE06C04115510561057105B4
:1073D00009F43FC011BB469AC7B99AB8CDB9A5B850
:1073E000B8B81BB80EB9E1BB82E08A95F1F700C0CE
:1073F00086B189B18CB111BB479A37B92AB99DB909
:10740000415051096109710981FFDECF452B462B9F
:10741000472BF9F08AE00E947C23D1500E94AA15E4
:10742000C80ED91EE11CF11CEADE8091EE0F8530FA
:10743000E0F4D11125CFB601C701DF91CF911F91A3
:107440000F91FF90EF90DF90CF90BF90AF909F9003
:1074500008950E94F11EDECF0E94F11E43CF0E94CC
:10746000F11E72CF0E94F11EA1CFCC24CA94DC2C55
:107470007601E1CF2F923F924F925F926F927F926F
:107480008F929F92AF92BF92CF92DF92EF92FF9234
:107490000F931F93CF93DF93CDB7DEB729970FB626
:1074A000F894DEBF0FBECDBF782E662E4A831092B1
:1074B000EE0F70E080E090E00E94206C9B01AC0138
:1074C00060E070E080E090E40E94E36D24EA30ED3B
:1074D00042E851E40E94806D9B01AC0160E074E2DF
:1074E00084EF99E40E945B6B6B837C838D839E8326
:1074F000262D235081E090E0022E01C0880F0A94CF
:10750000EAF789834EE0542E00E010E88FEF9FEFFA
:1075100099878887E22FFF27E1950CF4F0954F01BA
:10752000AA2497FCA094BA2C672D8A810E949316F6
:10753000288539858217930760F5B901872D0E9448
:10754000E945898174DE6B017C016F3F3FEF730772
:107550008307930709F44FC0C501B4010E94226C50
:107560009B01AC0160E070E080E090E40E94E36D7C
:107570001B01482E9F83C701B6010E94206C9B010E
:10758000AC01FF80622D732D842D9F2D0E94806D94
:1075900004C06FEF7FEF8FE79FE7BB81AC81ED8188
:1075A000FE802B2F3A2F4E2F5F2D0E940C6D181648
:1075B0003CF488859985800F911F9987888706C03C
:1075C000E885F985E01BF10BF987E88716950795A3
:1075D0005A9409F0A9CF22E1629EF0011124E70D2F
:1075E000F11DEE0FFF1FE754F14F888599859183B8
:1075F000808380E001C08FEF29960FB6F894DEBF3C
:107600000FBECDBFDF91CF911F910F91FF90EF90F3
:10761000DF90CF90BF90AF909F908F907F906F90B2
:107620005F904F903F902F9008950F931F93CF93AB
:10763000DF93D82F062F8093EF0F862F0E94FB45F4
:10764000DC3008F057C013E04CE0612F8D2F12DFC3
:10765000811103C01F5F1730B9F7ED2FF0E0DF0194
:10766000AA0FBB1FAB5DB04F8D919C919C01220F67
:10767000331FDF01AA0FBB1FA75BB04F4D915C9179
:10768000241B350BDF01AA0FBB1FAF5FB04F2D933B
:107690003C93A901440F551F481B590BDF01AA0F4A
:1076A000BB1FA352B14F4D935C93440F551FDF0195
:1076B000AA0FBB1FA754B14F421B530B4D935C93B2
:1076C000DF01AA0FBB1FAB54B04FCF01880F991F2A
:1076D0008F56904FEC0128813981220F331FEE0F16
:1076E000FF1FE359F04F80819181281B390B2D93A7
:1076F0003C9323C014E044E2612F8D2FBBDE88232E
:1077000041F0ED2FF0E0EE0FFF1FE75BF04F44E09C
:1077100004C01F5F183079F7F4CFDF019497208100
:107720003181220F331F84A195A1281B390B11969B
:107730003C932E934150FD0181F7802F0E94F2452A
:10774000DF91CF911F910F9183CC0F931F93CF9314
:10775000DF938B0140919A0E50919B0EAA27049FB4
:10776000B12D159FB001509FB00D611D7A1F149F60
:10777000B00D611D7A1F112440955095640F751F3F
:107780009AE28902E0011124CE018955944FCEDBA3
:107790004091980E5091990EAA27049FB12D159FE4
:1077A000B001509FB00D611D7A1F149FB00D611D77
:1077B0007A1F112440955095640F751FCE018D5589
:1077C000934FDF91CF911F910F91B0CB2F923F92AA
:1077D0004F925F926F927F928F929F92AF92BF92E1
:1077E000CF92DF92EF92FF920F931F93CF93DF938D
:1077F000CDB7DEB72C970FB6F894DEBF0FBECDBF66
:10780000E090880EF090890E2090800E3090810ECE
:107810008091600E8093C90C80915E0E8093CD0B99
:107820008091610E882309F4D2C463E083EA9CE06E
:1078300035D680915F0E882309F4C7C463E087EAD8
:107840009BE02CD68091E20F882309F4BAC480E033
:1078500091E0A0E0B0E020918C0E30918D0E2C01D3
:107860003D01420E531E611C711C20918A0E309105
:107870008B0EAC01BD01420F531F611D711D209184
:10788000860E3091870E5C016D01A20EB31EC11CE5
:10789000D11CA982BA82CB82DC822091840E3091E5
:1078A000850E5C016D01A20EB31EC11CD11CAD8200
:1078B000BE82CF82D8862091820E3091830E5C01E9
:1078C0006D01A20EB31EC11CD11CA986BA86CB863F
:1078D000DC8620917E0E30917F0E4C015D01820E80
:1078E000931EA11CB11C09811A812B813C810115B9
:1078F000110581E02807310524F00FEF1FEF20E08C
:1079000030E041155105E1E06E07710524F04FEFBD
:107910005FEF60E070E041145104F1E06F06710424
:107920002CF044244A94542C612C712C9701B20100
:1079300083EA9CE085D5950184018114910441E09E
:10794000A406B10424F00FEF1FEF20E030E04984DB
:107950005A846B847C844114510481E0680671046C
:107960002CF044244A94542C612C712C6D817E811E
:107970008F81988561157105E1E08E07910524F0EE
:107980006FEF7FEF80E090E09101A20187EA9BE03A
:1079900057D58091600E8093F30C80915E0E80939A
:1079A000F70B8091610E882309F409C463E08DEC24
:1079B0009CE074D580915F0E882309F4FEC363E0D8
:1079C00081ED9BE06BD58091E20F882309F4F1C330
:1079D00080E09FEFAFEFBFEF20918C0E30918D0EC6
:1079E0002C013D01420E531E611C711C77FCF1C33A
:1079F00020918A0E30918B0EAC01BD01420F531FB6
:107A0000611D711D77FD2FC42091860E3091870E68
:107A10005C016D01A20EB31EC11CD11C9601850133
:107A2000D7FC1DC48090840E9090850E5C016D0182
:107A3000A80CB91CC11CD11CA982BA82CB82DC82E1
:107A4000D7FC08C48090820E9090830E5C016D017B
:107A5000A80CB91CC11CD11CAD82BE82CF82D886B5
:107A6000D7FCF3C3E0917E0EF0917F0E4C015D01D7
:107A70008E0E9F1EA11CB11CB7FCE3C3011511059E
:107A800081E02807310524F00FEF1FEF20E030E000
:107A900041155105E1E06E07710524F04FEF5FEFEE
:107AA00060E070E041145104F1E06F0671042CF0C5
:107AB00044244A94542C612C712C9701B2018DEC12
:107AC0009CE0BED4950184018114910441E0A40698
:107AD000B10424F00FEF1FEF20E030E04D805E8016
:107AE0006F8078844114510481E0680671042CF0A1
:107AF00044244A94542C612C712C69817A818B81A5
:107B00009C8161157105E1E08E07910524F06FEF0E
:107B10007FEF80E090E09101A20181ED9BE090D4A5
:107B20008091600E80931D0D80915E0E8093210CDC
:107B30008091610E882309F43AC363E087EF9CE0EB
:107B4000ADD480915F0E882309F42FC363E08BEFDF
:107B50009BE0A4D48091E20F882309F422C380E043
:107B600092E0A0E0B0E020918C0E30918D0E2C01BF
:107B70003D01420E531E611C711C20918A0E3091F2
:107B80008B0EAC01BD01420F531F611D711D209171
:107B9000860E3091870E5C016D01A20EB31EC11CD2
:107BA000D11CA982BA82CB82DC822091840E3091D2
:107BB000850E5C016D01A20EB31EC11CD11CAD82ED
:107BC000BE82CF82D8862091820E3091830E5C01D6
:107BD0006D01A20EB31EC11CD11CA986BA86CB862C
:107BE000DC8620917E0E30917F0E4C015D01820E6D
:107BF000931EA11CB11C09811A812B813C810115A6
:107C0000110581E02807310524F00FEF1FEF20E078
:107C100030E041155105E1E06E07710524F04FEFAA
:107C20005FEF60E070E041145104F1E06F06710411
:107C30002CF044244A94542C612C712C9701B201ED
:107C400087EF9CE0FDD3950184018114910441E00C
:107C5000A406B10424F00FEF1FEF20E030E04984C8
:107C60005A846B847C844114510481E06806710459
:107C70002CF044244A94542C612C712C6D817E810B
:107C80008F81988561157105E1E08E07910524F0DB
:107C90006FEF7FEF80E090E09101A2018BEF9BE01E
:107CA000CFD38091600E8093470D80915E0E8093BC
:107CB0004B0C8091610E882309F471C263E081E26C
:107CC0009DE0ECD380915F0E882309F466C263E0E7
:107CD00085E29CE0E3D38091E20F882309F459C246
:107CE00080E09EEFAFEFBFEF20918C0E30918D0EB4
:107CF0002C013D01420E531E611C711C77FC9DC27C
:107D000020918A0E30918B0EAC01BD01420F531FA2
:107D1000611D711D77FD8DC22091860E3091870EF9
:107D20005C016D01A20EB31EC11CD11C9601850120
:107D3000D7FC7BC28090840E9090850E5C016D0113
:107D4000A80CB91CC11CD11CA982BA82CB82DC82CE
:107D5000D7FC66C28090820E9090830E5C016D010C
:107D6000A80CB91CC11CD11CAD82BE82CF82D886A2
:107D7000D7FC51C2E0917E0EF0917F0E4C015D0167
:107D80008E0E9F1EA11CB11CB7FC41C2011511052E
:107D900081E02807310524F00FEF1FEF20E030E0ED
:107DA00041155105E1E06E07710524F04FEF5FEFDB
:107DB00060E070E041145104F1E06F0671042CF0B2
:107DC00044244A94542C612C712C9701B20181E215
:107DD0009DE036D3950184018114910441E0A4060D
:107DE000B10424F00FEF1FEF20E030E04D805E8003
:107DF0006F8078844114510481E0680671042CF08E
:107E000044244A94542C612C712C69817A818B8191
:107E10009C8161157105E1E08E07910524F06FEFFB
:107E20007FEF80E090E09101A20185E29CE008D321
:107E30008091600E8093710D80915E0E8093750C21
:107E40008091610E882309F4A2C163E08BE49DE078
:107E500025D380915F0E882309F497C163E08FE4F6
:107E60009CE01CD38091E20F882309F48AC180E052
:107E700093E0A0E0B0E020918C0E30918D0E2C01AB
:107E80003D01420E531E611C711C20918A0E3091DF
:107E90008B0EAC01BD01420F531F611D711D20915E
:107EA000860E3091870E5C016D01A20EB31EC11CBF
:107EB000D11CA982BA82CB82DC822091840E3091BF
:107EC000850E5C016D01A20EB31EC11CD11CAD82DA
:107ED000BE82CF82D8862091820E3091830E5C01C3
:107EE0006D01A20EB31EC11CD11CA986BA86CB8619
:107EF000DC8620917E0E30917F0E4C015D01820E5A
:107F0000931EA11CB11C09811A812B813C81011592
:107F1000110581E02807310524F00FEF1FEF20E065
:107F200030E041155105E1E06E07710524F04FEF97
:107F30005FEF60E070E041145104F1E06F067104FE
:107F40002CF044244A94542C612C712C9701B201DA
:107F50008BE49DE075D2950184018114910441E088
:107F6000A406B10424F00FEF1FEF20E030E04984B5
:107F70005A846B847C844114510481E06806710446
:107F80002CF044244A94542C612C712C6D817E81F8
:107F90008F81988561157105E1E08E07910524F0C8
:107FA0006FEF7FEF80E090E09101A2018FE49CE011
:107FB00047D28091600E80939B0D80915E0E8093DE
:107FC0009F0C8091610E882309F4D9C063E085E796
:107FD0009DE064D280915F0E882309F4CEC063E0F7
:107FE00089E79CE05BD28091E20F882309F4C1C04D
:107FF00080E09DEFAFEFBFEF20918C0E30918D0EA2
:108000002C013D01420E531E611C711C77FCFBC00C
:1080100020918A0E30918B0EAC01BD01420F531F8F
:10802000611D711D77FDEBC02091860E3091870E8A
:108030005C016D01A20EB31EC11CD11C960185010D
:10804000D7FCD9C08090840E9090850E5C016D01A4
:10805000A80CB91CC11CD11CA982BA82CB82DC82BB
:10806000D7FCC4C08090820E9090830E5C016D019D
:10807000A80CB91CC11CD11CAD82BE82CF82D8868F
:10808000D7FCAFC0E0917E0EF0917F0E4C015D01F8
:108090008E0E9F1EA11CB11CB7FC9FC001151105BF
:1080A00081E02807310524F00FEF1FEF20E030E0DA
:1080B00041155105E1E06E07710524F04FEF5FEFC8
:1080C00060E070E041145104F1E06F0671042CF09F
:1080D00044244A94542C612C712C9701B20185E7F9
:1080E0009DE0AED1950184018114910441E0A40684
:1080F000B10424F00FEF1FEF20E030E04D805E80F0
:108100006F8078844114510481E0680671042CF07A
:1081100044244A94542C612C712C69817A818B817E
:108120009C8161157105E1E08E07910524F06FEFE8
:108130007FEF80E090E09101A20189E79CE080D18F
:108140002C960FB6F894DEBF0FBECDBFDF91CF9156
:108150001F910F91FF90EF90DF90CF90BF90AF9065
:108160009F908F907F906F905F904F903F902F9057
:10817000089580E090E0DC013FCF61E031CF61E025
:1081800026CF80E090E0DC0176CE61E068CE61E051
:108190005DCE80E090E0DC01A7CD61E099CD61E0AB
:1081A0008ECD80E090E0DC01DECC61E0D0CC61E0FF
:1081B000C5CC80E090E0DC010FCC61E001CC61E057
:1081C000F6CB80E090E0DC0146CB61E038CB61E0AB
:1081D0002DCB412C512C32010BCC812C912C5401F4
:1081E0005DCF1D821E821F8218864CCF19821A8293
:1081F0001B821C8237CF00E010E0980123CF40E0C3
:1082000050E0BA0111CF412C512C320101CF812C09
:10821000912C5401BBCD1D821E821F821886AACDCF
:1082200019821A821B821C8295CD00E010E0980111
:1082300081CD40E050E0BA016FCD412C512C32018C
:108240005FCD812C912C540119CC1D821E821F827E
:10825000188608CC19821A821B821C82F3CB00E09C
:1082600010E09801DFCB40E050E0BA01CDCBFC013B
:10827000623009F43BC018F1633069F1643011F5E4
:1082800011A210A2268D378D46895789AA27249FCF
:10829000B12D359FC001529FB00D811D9A1F349F93
:1082A000B00D811D9A1F112482A393A34089518987
:1082B0006289738940835183628373830895613037
:1082C00009F443C011A210A213A212A210821182BB
:1082D00012821382089511A210A28689978993A30E
:1082E00082A310821182128213820895268937890F
:1082F00044895589AA27429FB12D539FC001349FBD
:10830000B00D811D9A1F529FB00D811D9A1F11241F
:1083100080A391A340955095AA27429FB12D539FCA
:10832000C001349FB00D811D9A1F529FB00D811D59
:108330009A1F112482A393A344855585668577856A
:108340004083518362837383089526893789468DDC
:10835000578DAA27429FB12D539FC001349FB00D66
:10836000811D9A1F529FB00D811D9A1F112480A359
:1083700091A340955095AA27429FB12D539FC001CC
:10838000349FB00D811D9A1F529FB00D811D9A1F01
:10839000112482A393A34085518562857385408310
:1083A00051836283738308951F93CF93DF93EC010E
:1083B000898D0E94691F18A5012E04C09695879586
:1083C000779567950A94D2F724E0660F771F881F88
:1083D000991F2A95D1F7688779878A879B878B8D24
:1083E0000E94691F012E04C0969587957795679521
:1083F0000A94D2F734E0660F771F881F991F3A95C9
:10840000D1F76C877D878E879F878D8D0E94691F2E
:1084100004C096958795779567951A95D2F744E0AD
:10842000660F771F881F991F4A95D1F7688B798B44
:108430008A8B9B8B69A5CE01DF91CF911F9117CFBE
:108440000F931F93FC01808D918D8617970721F064
:10845000718F608F61E001C060E0828D938D841721
:10846000950719F0538F428F61E0848995898217AF
:10847000930719F0358B248B61E0848D958D8017DF
:10848000910719F0158F048F02C0662321F0CF01E8
:108490001F910F9189CF1F910F910895FC0160A743
:1084A00083CF211107C0BB27A92F982F872FBC018D
:1084B000CB010895A72FE82F8F3FE9F08F5F90E061
:1084C000880F991FF0E0EE0FFF1FE40FF51F2081CA
:1084D0003181FA01E80FF91F80819181821B930B92
:1084E000892F9927A89FB001A99F700D1124620FB1
:1084F000731FCB0108958EEF91E0E4CFFC0114824D
:10850000158216821782108211821282138281A52F
:108510008F5F81A7833009F43BC0853009F434C0F4
:10852000823009F008952689378935A324A3448928
:108530005589AA27429FB12D539FC001349FB00D8A
:10854000811D9A1F529FB00D811D9A1F112480A377
:1085500091A340955095AA27429FB12D539FC001EA
:10856000349FB00D811D9A1F529FB00D811D9A1F1F
:10857000112482A393A3448555856685778540831E
:10858000518362837383089511A615A214A20895DE
:1085900011A210A28689978993A382A30895CF92EE
:1085A000DF92EF92FF92CF93DF93EC01CC80DD80DE
:1085B000EE80FF808F2D9927AA27BB27892B8A2B36
:1085C0008B2B09F042C089A5823009F433C070F5C5
:1085D000813009F444C040E050E02AA13BA1AA2721
:1085E000429FB12D539FC001349FB00D811D9A1F32
:1085F000529FB00D811D9A1F112428A139A1820F0D
:10860000931F9DA38CA3488159816A817B814C0D66
:108610005D1D6E1D7F1D4C835D836E837F83DF91A7
:10862000CF91FF90EF90DF90CF9008958330A1F02D
:10863000843089F68EA1811122C0BB27AF2D9E2DDB
:108640008D2DAC0140955095C8CFCE0157DFCC8021
:10865000DD80EE80FF80B7CF4C895D89BECF8EA1D3
:10866000811105C077276F2D5E2D4D2DB6CF44E8C3
:1086700053E0C701B6010E94981CAC01AECF44E89C
:1086800051E0C701B6010E94981CDBCFCF92DF9268
:10869000EF92FF920F931F93CF93DF93EC01CC8067
:1086A000DD80EE80FF808F2D9927AA27BB27892B9D
:1086B0008A2B8B2B09F04AC02A8D6C857D858E858F
:1086C0009F85233009F467C040F5213009F4ABC021
:1086D000EC89FD89C60ED71EE81EF91ECC82DD820C
:1086E000EE82FF829F0140E050E03058410951097D
:1086F000A889B9890E944E6F2FEF3FEF40E050E00C
:108700000E945E6F3F8B2E8BDF91CF911F910F9157
:10871000FF90EF90DF90CF900895243009F45FC070
:108720002530B1F69701860149E0369527951795D2
:1087300007954A95D1F7F8011D8B0C8B298D2223C3
:1087400049F2E095F095FD8BEC8BC4CFE1E0898D8B
:10875000E81BE98FE1116FC0C12CD12C7601CC82CE
:10876000DD82EE82FF82FF27E1950CF4F095DF01B8
:10877000AA0FBB1F1196288539854A855B850E9403
:10878000586F6C877D878E879F872A8D211159C0EE
:10879000FD8BEC8B9DCFAD2DEE2DEF3F09F462C02C
:1087A0002E2D2F5F30E0220F331FF0E0EE0FFF1F62
:1087B000E051F04F40815181F901E051F04F2081AB
:1087C0003181241B350B232F3327A29FF001A39F58
:1087D000F00D1124E40FF51FFD8BEC8B7BCFAB89E3
:1087E000A295AF70088119812A813B81F32F000F78
:1087F000111F221F331FEF2FEE1FEE27EE1FBF2F7B
:10880000B295B695B770EB27EF27F695EF27E17095
:108810000E2BA15058F7088319832A833B83F80154
:108820001D8B0C8B57CF33272F2D1E2D0D2DF801AF
:108830001D8B0C8B4FCFCC24CA94DC2CEC2CF12C50
:108840008ECF223009F03DCF0E94426F7D8B6C8B22
:108850002A8D6C857D858E859F85CC80DD80EE8020
:10886000FF802FCF2EEF31E0A0CFFF920F931F9309
:10887000CF93DF93EC01F62E1C821D821E821F8295
:108880000E891F896CA17DA1CB01A0E0B0E0772704
:108890006627980140E050E00E94856F3F8F2E8F41
:1088A000F11023C084E089A719A218A2AA27209F4B
:1088B000B12D319FC001129FB00D811D9A1F309FB5
:1088C000B00D811D9A1F11248AA39BA388899989C1
:1088D000AA89BB8988839983AA83BB83FFA2DF917E
:1088E000CF911F910F91FF90089581E089A7CE014C
:1088F0000E940B4DFFA2DF91CF911F910F91FF902E
:108900000895FC0111A210A2268D378D4689578942
:10891000AA27249FB12D359FC001529FB00D811D04
:108920009A1F349FB00D811D9A1F112482A393A317
:10893000408951896289738940835183628373833B
:108940000895CF92DF92EF92FF920F931F93CF93F0
:10895000DF9380915B0EC82FCC0FC80FCF5F609163
:108960005A0E8FE99DE00E94FA1E6C2F8FE99DE060
:108970000E94601C80914A0E90914B0EA0914C0E6B
:10898000B0914D0E8F3F2FEF9207A207B20709F467
:108990009CC020919C0E30919D0E2115324008F014
:1089A0005DC0CFEFDFEFE0901D0EF0901E0E009047
:1089B000660E02C0F694E7940A94E2F74091940E92
:1089C0005091950E411582E0580708F4ACC09A0109
:1089D00032508091A00E9091A10E96958795969514
:1089E0008795811542E0940708F472C08C011250FB
:1089F0008091680E882309F471C0AE01AA27249FD4
:108A0000B12D359FC001529FB00D811D9A1F349F1B
:108A1000B00D811D9A1F11246091920E7091930EDA
:108A2000AC018FE99DE00E94711CC8018095909572
:108A30008E159F0508F07AC04FEF5FEF60919E0E94
:108A400070919F0E8AEB9DE0DF91CF911F910F9166
:108A5000FF90EF90DF90CF900C94711C20914E0E00
:108A600030914F0E40E050E0820F931FA41FB51FBE
:108A7000C0905C09D0905D09E0905E09F0905F09BC
:108A8000C816D906EA06FB0600F1C0905C09D09032
:108A90005D09E0905E09F0905F09C81AD90AEA0AF8
:108AA000FB0AC216D306E406F50608F07ACF9E2D1F
:108AB0008D2D7C2D66270E94856FF901EE0FFF1F1B
:108AC000EC57FC4FC081D1816ECFC0E0D0E06BCFBE
:108AD00000E010E08091680E81118FCFC901809570
:108AE00090958E159F0530F54FEF5FEF6091920ED8
:108AF0007091930E8FE99DE00E94711C9E01AA2740
:108B0000029FB12D139FC001309FB00D811D9A1F90
:108B1000129FB00D811D9A1F112460919E0E7091BD
:108B20009F0EAC018FCF20E030E053CFA8014E0D57
:108B30005F1D84CFA9014E0D5F1DD8CF8091DE0F40
:108B400087FD09C06F7070E0992787FD90956817C1
:108B5000790709F0089580E8289F90011124242BBB
:108B60003052220F331F220F331F3093200E2093D9
:108B70001F0E0E944F176FEF81E00C94EC530F9380
:108B80001F93CF93DF931F92CDB7DEB78B0140FDCC
:108B900008C041FD14C00F90DF91CF911F910F913C
:108BA00008959093200E80931F0E49830E944F17C3
:108BB0006FEF81E00E94EC53498141FFECCF1093AD
:108BC0001E0E00931D0E0F90DF91CF911F910F91FC
:108BD000B8CEE82FF0E0EE0FFF1FE352F54F7183A0
:108BE00060830895E82FF0E0EE0FFF1FE352F54F8A
:108BF000118210820895E82FF0E0EE0FFF1FE3527C
:108C0000F54F8FEF9FEF91838083089560FD05C03E
:108C100090931A0B8093190B0895BC018EE168C6DE
:108C200060FD05C09093100B80930F0B0895BC015D
:108C300089E15EC660FD05C09093180B8093170B09
:108C40000895BC018DE154C660FD05C090930E0BE4
:108C500080930D0B0895BC0188E14AC660FD05C0F4
:108C60009093140B8093130B0895BC018BE140C6C5
:108C7000FF920F931F93CF93DF93FFB60E94FE1CCA
:108C8000882309F43FC00E94DA1CC9EBDEE011C062
:108C9000FE01E00FF11F808191810E94F41C0E5FA4
:108CA0001F4F04321105A1F7A4968FE0C93DD807E4
:108CB00019F000E010E0ECCF8091DB0F9091DC0F19
:108CC0000E94F41C8091D90F9091DA0F0E94F41C3D
:108CD0008091DD0F0E94CF1C8091DE0F0E94C41C8A
:108CE0008091E00F0E94CF1C8091DF0F0E94C41C76
:108CF0008091E10F0E94CF1C8091E20F0E94C41C62
:108D00000E944E248F2DDF91CF911F910F91FF90E4
:108D10000C94C21C0F931F93CF93DF93CDB7DEB794
:108D2000E6970FB6F894DEBF0FBECDBF92E2E4EC3B
:108D3000F6E0DE01119601900D929A95E1F78130EF
:108D400011F58091DE0F992787FD9095029661E1DC
:108D500070E00E94CC6A81508093DE0F89DF8091A1
:108D6000DE0FE1E0F0E0EC0FFD1F92E08902E00D84
:108D7000F11D112462817381CE0183960E94F06EF1
:108D80006EE978E022C0823049F58091DF0F9927A3
:108D900087FD9095019660E170E00E94CC6A809317
:108DA000DF0F66DF8091DF0FE1E0F0E0EC0FFD1FE9
:108DB00092E08902E00DF11D112462817381CE01E0
:108DC00083960E94F06E64EA78E0CE0183960E945A
:108DD000E56ECE0183960E943D19C9C08330A1F48F
:108DE0008091B70A9091B80A9093DA0F8093D90FC7
:108DF0003FDF0E94CF2141E060E070E0C0DE8AEA00
:108E000098E00E943D19B3C08430D1F48091F011F4
:108E1000992787FD9095019666E070E00E94CC6AE4
:108E2000182F8093F0116CEB78E0CE0183960E94AE
:108E3000F06E1F5C1DA3CE0183960E943D1997C062
:108E40008530E1F51091E00F0091F011212F30E015
:108E5000002E02C0359527950A94E2F720FF12C034
:108E600060EC78E0CE0183960E94F06E21E030E065
:108E7000002E01C0220F0A94EAF7209521232093A7
:108E8000E00F10C068EC78E0CE0183960E94F06E8F
:108E900081E090E0002E01C0880F0A94EAF7812B50
:108EA0008093E00FE5DE8091F0118F5C8DA3CE0101
:108EB00083960E943D190E94623559C0863059F44C
:108EC0000E94895D8FEC98E00E943D190E94203736
:108ED0000E9462354CC0873031F481E00E94A81DA9
:108EE0000E94623544C0883021F58091E10F9927B6
:108EF00087FD9095019663E070E00E94CC6A8093B4
:108F0000E10FB6DE8091E10F813049F0823061F0EF
:108F100081112BC08EED98E00E943D1926C087EE8E
:108F200098E00E943D1921C081EF98E00E943D1910
:108F30001CC08930E1F48091E20F992787FD90955C
:108F4000019662E070E00E94CC6A8093E20F90DEAE
:108F50008091E20F882329F08BEF98E00E943D1961
:108F600004C085E099E00E943D190E946235E696B2
:108F70000FB6F894DEBF0FBECDBFDF91CF911F912A
:108F80000F910895CF93DF932091DE0F27FD0BC043
:108F90006F7070E0332727FD30956217730719F063
:108FA000DF91CF9108958091DD0F8823C9F3443676
:108FB000B8F7C42FD0E08091DB0F9091DC0FC81779
:108FC000D90771F3CE010E943D1D882349F3D09348
:108FD000DC0FC093DB0F1092AE0E4ADEDF91CF9113
:108FE0000C946235CF93DF9300D0CDB7DEB780917C
:108FF000DE0F87FD0DC06F7070E0992787FD90959B
:109000006817790729F00F900F90DF91CF9108959D
:1090100041111DC03091DD0F223008F454C03323BC
:1090200091F3842F80518E31A0F1842F80558E31A1
:10903000A0F0842F8053893108F46BC08091AE0E6C
:10904000811121C00F900F90DF91CF910895413091
:1090500009F451C03091DD0FE2CFE42FF0E0EE0FC4
:10906000FF1FEF54F24F818D928D88279E7F30E055
:10907000220F331F220F331F822B932B928F818F4E
:1090800081E08093AE0E0F900F90DF91CF910C9402
:109090006235E42FF0E0EE0FFF1FEF5CF14F818DA2
:1090A000928D8C7F9170522F550F40E0842B952B21
:1090B000928F818F81E08093AE0E0F900F90DF91A1
:1090C000CF910C946235632F772767FD7095822FBF
:1090D00090E06817790709F4A2CF2093DD0F2A8367
:1090E0004983C6DD0E9420370E9462353091DD0F32
:1090F0002A81498194CF822F880F10921D0E809370
:109100001E0E2A8349831DDC3091DD0F49812A819F
:1091100086CFE42FF0E0F097DF01AF5AB14F30E097
:10912000EA51F94F408187E090E0841B910902C029
:10913000359527958A95E2F72C9381E08093AE0EC2
:10914000A2CF2091FF14309100152F5F32412130C2
:10915000324038F4BC0180E090E04FEF52E10C94D3
:109160003D240895FF920F931F93CF93DF938C01BB
:10917000FFB60E94FE1C8823D9F10E94DA1CC0E0D1
:10918000EC2FF0E0EE0FFF1FEF5AF14F818D928D23
:109190000E94F41CCF5FC93199F7D0E0ED2FF0E0C9
:1091A000EF5AF14F80810E94CF1CDF5FD731B1F7BA
:1091B000EC2FF0E0EE0FFF1FEF5AF14F818D928DF3
:1091C0000E94F41CCF5FCE3199F78091680E0E9407
:1091D000CF1C8091690E0E94CF1CC6EADEE0899107
:1091E0000E94CF1C8EE0CC3AD807C9F7C801A9DF8E
:1091F0008F2DDF91CF911F910F91FF900C94C21C86
:109200006091B80E8A3030F5681305C0862F865FEE
:109210008093B80E14C0462F552747FD5095282F30
:10922000332727FD3095265F3F4F4217530729F418
:10923000862F8A508093B80E02C08093B80E8FEFAD
:109240009FEFDC018093B40E9093B50EA093B60E01
:10925000B093B70E8091B80E861749F00E94F01AAD
:109260008091DD0F811103C08BED90E07BCF0895DD
:10927000CF93DF93DFB70E94F71E882309F49DC0C8
:109280000E94791E0E94861F0E94091960E080E0FA
:1092900090E0E4DC80E00E94CE1380E00E94F23394
:1092A00080E00E94C53380E00E94FB3780E00E948E
:1092B000CE3780E00E94A13780E00E94693760E0ED
:1092C00080E090E0A3DC0E94DE240E94D92460E0CC
:1092D00080E090E0B9DC60E080E090E0ABDC80E32F
:1092E0000E94592380E70E94592382EB0E94592350
:1092F00060E080E090E08ADCC2E18C2F73DC8C2F90
:10930000865079DCCF5FC831C1F781E00E94CE136F
:1093100060E08FEF9FEF84DC60E080E090E00E94EF
:109320006624C0E06C2F6E5E8C2F0E94153BCF5FD1
:10933000C630C1F780E00E94CE1381E00E94C533A1
:1093400060E080E090E06CDC60E08FEF9FEF0E94D7
:1093500066246C2F645F8C2F0E94153BCF5FCC304E
:10936000C1F780E00E94C53360E080E090E058DC07
:1093700060E080E090E00E94662460E08FEF9FEF65
:1093800045DC8C2F2FDCCF5FC231D9F7CCE06C2FBE
:109390006A5F8C2F0E94153BCF5FC231C1F760E03E
:1093A00080E090E033DC8C2F1DDCCF5FC831D9F733
:1093B0000E9428380E94861F5BDC8D2FDF91CF91A1
:1093C0000C94EF1EEF92FF920F931F93CF93DF93B6
:1093D0001F92CDB7DEB7182F7B010E94A136E11492
:1093E000F10409F0ECC0123171F542DF2CC00E948B
:1093F000191F89830E941C1F91E06981813009F443
:1094000090E0892F0E94392A1EC01B30E1F40E948F
:109410001C1F823091F018F08330A9F407C00E941D
:10942000191F682F83E00E94392A0DC00E94191F5E
:10943000682F82E00E94392A06C00E94191F682FF7
:1094400080E00E94392A0E941C1F082F8823B1F057
:10945000E114F10409F4C0C01D3009F0B9C00E9444
:10946000191F61E0811160E0802F0F90DF91CF9193
:109470001F910F91FF90EF900C94392A173291F4BD
:10948000E114F10419F00E94021A02C00E94E519C9
:109490000E94441A8091DD0F8111A1C08BED90E0F4
:1094A00061DE9DC0EF2809F481C01E3009F08BC039
:1094B0008091DD0F882309F486C08091AC0E88234B
:1094C00019F01092AC0E7FC081E08093AC0E7BC08F
:1094D000812F20DC6BC01C30A1F48091DD0F811145
:1094E00003C08BED90E03EDE81E09091DD0F9111A5
:1094F00080E08093DD0FBCDB0E9420370E94623544
:1095000055C09091AC0E1D3069F4923039F481E071
:109510009091DD0F911120C080E01EC082E0809309
:10952000AC0E44C0911103C0812F6ADE3FC01A30D7
:1095300008F03CC0923069F018F49130B9F503C0DE
:109540009530A0F50CC01093AD0E83E08093AC0E67
:109550002DC01093AD0E84E08093AC0E27C0809197
:10956000AD0E2AE0829F100D1124812F1093AD0EB5
:10957000943021F4992787FD9095F4DD8091AD0E0C
:10958000992787FD90950E943D1D882351F0809179
:10959000AD0E992787FD90959093DC0F8093DB0F9C
:1095A00067DB8FEF8093AD0E0E9420370F90DF9125
:1095B000CF911F910F91FF90EF900C9462351A306C
:1095C00009F023CF14CF8091700980FF84CF80CF22
:1095D000173209F06ACF57CF173241F757CFEF282C
:1095E00091F7E4CFEFCE4F925F926F927F928F927E
:1095F0009F92AF92BF92CF92DF92EF92FF920F9322
:109600001F93CF93DF9300D000D0CDB7DEB78FB6D6
:10961000F894882309F438C1C12CBC2CBB0CBB0CBA
:10962000BB0C36EC77247A940FE710E0BEE94B2EA2
:10963000BBE05B2EEE24EA948FE7F82E31BB469A0E
:109640009C2D990F292F26702064892F880F8072F6
:10965000907C892B9C2D9695927041E045B928B954
:109660008BB99EB987E881BB2DE02A95F1F7000000
:1096700031BB469A80EE87B997E09AB98DB945B962
:1096800080E488B91BB88EB987E481BB82E08A95F3
:10969000F1F700C066B189B14CB131BB479A962F42
:1096A00096959370E0E86E9FB0011124962B282FB9
:1096B0002071922B282F269526952870922B86951F
:1096C0008076982B50E0440F551F44705527942BFB
:1096D00087EE87B987EF8AB982EE8DB9DB2C20E05F
:1096E000F0ECAF2EAB0CA8ED9A2E9B0C07C082506D
:1096F000808396952F5FD394283021F1ED2DF0E0F3
:10970000EF59F64F8081482F4E7F89F7792F71707E
:109710008170781771F3872F8A608083FFE3FD15CE
:1097200070F1672F772767FD70958D2D2B833C8314
:109730009A8358DF2B813C819A8196952F5FD39431
:109740002830E1F6C394E8E0BE0EFFE0FC1508F017
:1097500075CF8FBE0F900F900F900F90DF91CF912C
:109760001F910F91FF90EF90DF90CF90BF90AF903F
:109770009F908F907F906F905F904F9008956A2C8C
:10978000620E4091A60B4423B1F1772309F451C036
:10979000EEE1FBE0DF0105C08BE0AE39B80709F46C
:1097A00091C08D918F3FC1F3413009F479C0AEE192
:1097B000BBE040E050E005C04F5F5F4F40385105CF
:1097C00039F08D918F3FC1F7DA01A25EB44F6C92F0
:1097D0008091A50B813009F08CCF808180688193C6
:1097E0004E165F0609F485CF8081806881934E16FE
:1097F0005F0699F77ECF4FEF5FEF672F862D2B83A4
:109800003C8379839A830E942C2B79812B813C8124
:109810009A8171113CC0692D620F4FE78091DF0F73
:109820002B833C839A830E94B6142B813C819A81BE
:1098300060CF8091A50B81115CCF413009F44BC002
:10984000EEE1FBE040E050E005C04F5F5F4F403885
:10985000510539F081918611F8CFFA01E25EF44F9B
:109860007082EEE1FBE081918F3F09F042CF8BE007
:10987000EE39F807C1F72B833C839A830E94E324D7
:109880002B813C819A8135CF98E0C92EC6CE6FEFEF
:109890007FEF862D0E949C142B813C819A8129CFD9
:1098A000462D50E0DA01A25EB44F6C92D801A41BA1
:1098B000B50BA25EB44F6C928091A50B813009F07C
:1098C00018CF8BCF8091E10F81116ECFF092A20B58
:1098D000E092A10B69CF462D50E0FA01E25EF44F11
:1098E0007082F801E41BF50BE25EF44F7082B9CF91
:1098F000E82FE86F86958695869528E030E001C0D0
:10990000220F8A95EAF720952E23AFB7F894CB0162
:10991000892F992786958695F82F56EC51BB469A44
:10992000482F440F342F3670306880719927826039
:10993000942F990F9072982B407C942B8F2F8695A3
:109940008270806215B838B99BB98EB947E841BBBF
:109950007695679576956795362F51BB469AF62F83
:10996000FF0F962F9695331F3327331F8F2F867047
:10997000382B30686071772762608F2F880F807274
:10998000862BF07C8F2B927015B838B98BB99EB9A5
:1099900041BB51BB469A3E2F330F367031649E2F28
:1099A00096959270906AE1E0E5B938B9B0EFBBB92D
:1099B0009EB941BB85E08A95F1F7000051BB469AFC
:1099C000F22FFF0F622F6695722F771F7727771F71
:1099D0008F2F8670782B706420718F2F880F807284
:1099E000822BF07C8F2B6270606AE5B978B98BB9F5
:1099F0006EB941BB8AE08A95F1F700C051BB469A27
:109A0000E5B938B9BBB99EB941BB8AE08A95F1F78F
:109A100000C0AFBF0895FC0126893789468D578D58
:109A2000AA27429FB12D539FC001349FB00D811DC5
:109A30009A1F529FB00D811D9A1F112480A391A3DC
:109A400040955095AA27429FB12D539FC001349F46
:109A5000B00D811D9A1F529FB00D811D9A1F1124B8
:109A600082A393A34085518562857385408351838A
:109A70006283738308959091390A8091380A209106
:109A80003A0A211131C02091CC0C2111DFC1209163
:109A9000430A211162C02091F60C211145C1209189
:109AA0004C0A21114EC02091200D2111ABC02091F4
:109AB000550A21113AC020914A0D21117EC12091F1
:109AC0005E0A211126C02091740D2111E4C020915D
:109AD000670A211112C020919E0D21114AC0909356
:109AE000390A8093380A08952091CC0C2111CFCFE8
:109AF00010923A0A8FEF9FEFCACF20919E0D21114D
:109B0000EECF1092670A2FEF2093660A2093650A22
:109B1000E6CF2091740D2111DACF10925E0A2FEF5B
:109B200020935D0A20935C0AD2CF20914A0D211127
:109B3000C6CF1092550A2FEF2093540A2093530A50
:109B4000BECF2091200D2111B2CF10924C0A2FEFE1
:109B500020934B0A20934A0AAACF2091F60C211198
:109B60009ECF1092430A2FEF2093420A2093410A7E
:109B700096CF10929C0D10929A0D1092990D109202
:109B8000790D10927A0D10927B0D10927C0D10922F
:109B9000940D1092930D10929E0D1092960D1092AE
:109BA000950D1092980D1092970D1092750D1092C0
:109BB000760D1092770D1092780D1092A00C1092E5
:109BC0009E0C10929D0C10927D0C10927E0C1092A7
:109BD0007F0C1092800C1092980C1092970C10929F
:109BE000A20C10929A0C1092990C10929C0C10924C
:109BF0009B0C1092790C10927A0C10927B0C1092A4
:109C00007C0C6DCF10921E0D10921C0D10921B0D2E
:109C10001092FB0C1092FC0C1092FD0C1092FE0C9A
:109C20001092160D1092150D1092200D1092180D15
:109C30001092170D10921A0D1092190D1092F70C28
:109C40001092F80C1092F90C1092FA0C1092220C4F
:109C50001092200C10921F0C1092FF0B1092000C0F
:109C60001092010C1092020C10921A0C1092190C06
:109C70001092240C10921C0C10921B0C10921E0CB3
:109C800010921D0C1092FB0B1092FC0B1092FD0B0E
:109C90001092FE0B0CCF1092720D1092700D10925C
:109CA0006F0D10924F0D1092500D1092510D109299
:109CB000520D10926A0D1092690D1092740D10924F
:109CC0006C0D10926B0D10926E0D10926D0D109226
:109CD0004B0D10924C0D10924D0D10924E0D109296
:109CE000760C1092740C1092730C1092530C10920C
:109CF000540C1092550C1092560C10926E0C10923F
:109D00006D0C1092780C1092700C10926F0C1092D7
:109D1000720C1092710C10924F0C1092500C109209
:109D2000510C1092520CD3CE1092F40C1092F20CF3
:109D30001092F10C1092D10C1092D20C1092D30C04
:109D40001092D40C1092EC0C1092EB0C1092F60CBA
:109D50001092EE0C1092ED0C1092F00C1092EF0C91
:109D60001092CD0C1092CE0C1092CF0C1092D00C01
:109D70001092F80B1092F60B1092F50B1092D50B77
:109D80001092D60B1092D70B1092D80B1092F00BAA
:109D90001092EF0B1092FA0B1092F20B1092F10B43
:109DA0001092F40B1092F30B1092D10B1092D20B75
:109DB0001092D30B1092D40B72CE1092480D1092C9
:109DC000460D1092450D1092250D1092260D109201
:109DD000270D1092280D1092400D10923F0D1092F9
:109DE0004A0D1092420D1092410D1092440D1092A6
:109DF000430D1092210D1092220D1092230D1092FE
:109E0000240D10924C0C10924A0C1092490C109296
:109E1000290C10922A0C10922B0C10922C0C1092E0
:109E2000440C1092430C10924E0C1092460C10925F
:109E3000450C1092480C1092470C1092250C109271
:109E4000260C1092270C1092280C39CE1092CA0CB6
:109E50001092C80C1092C70C1092A70C1092A80C6C
:109E60001092A90C1092AA0C1092C20C1092C10C64
:109E70001092CC0C1092C40C1092C30C1092C60C11
:109E80001092C50C1092A30C1092A40C1092A50C69
:109E90001092A60C1092CE0B1092CC0B1092CB0B02
:109EA0001092AB0B1092AC0B1092AD0B1092AE0B4C
:109EB0001092C60B1092C50B1092D00B1092C80BCB
:109EC0001092C70B1092CA0B1092C90B1092A70BDD
:109ED0001092A80B1092A90B1092AA0BD8CDCF927A
:109EE000DF92EF92FF92CF93DF938091AC0E8823A5
:109EF00009F471C0813009F4BBC08091AD0E87FDBB
:109F000044C060E2805D0E9419196091DD0F84E019
:109F10000E94E2188091AC0E811135C061E0809101
:109F2000DD0F882381F186E00E94E21860917009BC
:109F3000617087E00E94E2188091A60B81112AC00F
:109F400061E08091AC0E823009F060E0462F85E040
:109F50000E94B3188091E3099091E4092091E109EE
:109F60003091E209237F3093E2092093E109837F56
:109F70009093E4098093E309DF91CF91FF90EF90F4
:109F8000DF90CF90089560E0CECF60E280E20E9443
:109F90001919BBCF6091A50B85E00E94E21861E022
:109FA0008091A60B813009F060E082E00E94E21807
:109FB0008091A60B41E0823009F040E061E0813001
:109FC00009F454C083E0DF91CF91FF90EF90DF90D0
:109FD000CF900C94B3188091E1099091E2099D7F94
:109FE0009093E2098093E1098091E3099091E4095B
:109FF0009D7F9093E4098093E309C090B00ED090C8
:10A00000B10EE090B20EF090B30EF7FCBECFC701D8
:10A01000B60120E932E040E050E00E945E6FE901C5
:10A020008091AF0E833081F0893171F08F3161F012
:10A030008F3051F0803141F0BE01882777FD809547
:10A04000982F0E942D1961CF9E012253310937FDAF
:10A050001DC0E90161E0C11480E8D806E104F10403
:10A060000CF060E089E00E94E218E6CF60E0AACF41
:10A070006091DB0F7091DC0F80E090E00E942D1961
:10A080006091AE0E89E00E94E2183FCF3195219594
:10A090003109DFCF2F923F924F925F926F927F9262
:10A0A0008F929F92AF92BF92CF92DF92EF92FF92E8
:10A0B0000F931F93CF93DF9300D0CDB7DEB7382E29
:10A0C0004FB6F894282F259525952595259580E25E
:10A0D00090E002C0959587952A95E2F7932D9F70A1
:10A0E000982B86EC81BB469A492F440F292F269541
:10A0F000392F331F3327331F842F8670382B30645A
:10A100009071842F880F8072892B407C842B227061
:10A11000206491E095B938B98BB92EB987E881BB35
:10A1200025E02A95F1F70000832D992787FD90956A
:10A130009A838983FC01E150F94FE081F0E080E1EE
:10A1400090E08E1B9F0B66246A94762C082E02C02A
:10A15000769467940A94E2F702C0660C771C8A959D
:10A16000E2F740E050E020E030E88FEF9FEF66EC50
:10A17000262E17E877E0972EAA24A394A0E4BA2EFF
:10A18000B0E2CB2E07E4D02E67EEE62E77EFF72E67
:10A19000A2EE5A2E0AC0820F931F369527954F5F65
:10A1A0005F4FE417F5070CF46BC0BC01672F7727EE
:10A1B00066956695062F21BA469AB62FBB0FAB2F30
:10A1C000A670A0686071772762607B2F770F70722E
:10A1D000762BB07C7B2B602F66956270606215B821
:10A1E000A8B97BB96EB911BBBC0176956795769518
:10A1F0006795A62F21BA469A062F000FB62FB6955F
:10A20000AA1FAA27AA1F0F2EF6E08F2EF02D80225C
:10A21000A829A068607177276260702F770F70722D
:10A22000762B007C702BB27015B8A8B97BB9BEB97B
:10A2300011BBA2E0AA95F1F700C021BA469AB0EE90
:10A24000B7B99AB8BDB9A5B8B8B81BB8CEB8D1BA25
:10A2500062E06A95F1F700C066B169B17CB121BADC
:10A26000479AE7B8FAB85DB865FD95CF821B930BA6
:10A27000369527954F5F5F4FE417F5070CF095CFA4
:10A2800026EC21BB469A21E025B927E428B920EF26
:10A290002BB922E42EB927E821BBA5E0AA95F1F756
:10A2A000000086219721E981FA81EE0FFF1FE95610
:10A2B000F54F91838083892F9927A981BA81AD5861
:10A2C000B54F14962C91149730E0281B390B37FDAD
:10A2D00019C025303105E4F44FBE0F900F90DF9187
:10A2E000CF911F910F91FF90EF90DF90CF90BF9093
:10A2F000AF909F908F907F906F905F904F903F9026
:10A300002F9008953195219531092530310524F399
:10A3100014968C9381E090E0A0E0B0E0032C04C0A0
:10A32000880F991FAA1FBB1F0A94D2F74091730A86
:10A330005091740A6091750A7091760A842B952B5E
:10A34000A62BB72B8093730A9093740AA093750A77
:10A35000B093760A3092D80ABFCF6F928F929F92B5
:10A36000AF92BF92CF92DF92EF92FF920F931F9323
:10A37000CF93DF93E0912217F0912317309719F0D4
:10A3800082E097E109952FB7F8948091EB179091AF
:10A39000EA17891708F009C10091EC17080F091B8B
:10A3A0002FBF10E00115110509F476C0C0E0D0E020
:10A3B0002091EC17EE24E394F12CE3E09E2EF4E0E0
:10A3C0008F2EA2E0AA2EBB24B394892F622F90E097
:10A3D00070E00E94CC6AE091ED17F091EE17E80F63
:10A3E000F91FF081F83F08F065C0F7FF71C0809158
:10A3F0002717843031F0F0932417F0922917E09258
:10A4000028178F2F807F803B79F198F4803961F194
:10A41000803A51F1803841F1F03F09F4B1C0F73F83
:10A4200009F4C6C010922717109229171092281706
:10A430001DC0803D09F4A1C008F49CC0803EA1F07D
:10A44000803F51F7EF2FE15FEF3030F7AE2FB0E0F4
:10A45000A15EB84F8C91813009F49BC0E8F2823044
:10A4600009F48BC08330F1F6909227173FB7F89428
:10A470009091EA17892F90E001962091EC17622FB6
:10A4800070E00E94CC6A982F8093EA173FBF219614
:10A49000C017D10708F499CFDF91CF911F910F9189
:10A4A000FF90EF90DF90CF90BF90AF909F908F90F4
:10A4B0006F900895D0902717B092271720E040E0C2
:10A4C0006F2F81E090E00E94C914D0922717CECF61
:10A4D00060902717662051F2409128175091291754
:10A4E0009A01ABEABAEA0E94796F6C01D694C794DC
:10A4F000C601880F991F8C0D9D1D6A01C81AD90AC3
:10A50000D601AE5FB84E9296FC93CA010196909325
:10A5100029178093281721E0C216D104B9F022E050
:10A52000C216D10409F0A2CF209126174091251719
:10A53000609124170E94C91480912717843009F470
:10A5400095CFF0922917E092281790CF22E062125F
:10A550008DCF20E040912517609124170E94C914E7
:10A5600080912717843009F481CFD0922917C092A7
:10A5700028177CCF803C09F04FCFA092271776CFC9
:10A5800080922717F0932417F0922917E09228174A
:10A590006DCF8093271720E040E06F2F81E090E09F
:10A5A0000E94C9141092271761CF082F091BF8CEFB
:10A5B00040912817509129179A01ABEABAEA0E94F4
:10A5C000796F969587959C01220F331F280F391FAD
:10A5D000DA01A21BB30BAE5FB84E9296FC93CA0190
:10A5E0000196909329178093281720912617409160
:10A5F0002517609124170E94C9141092271736CF8F
:10A6000026EC90EE87E0F0E8E7E477EE67EF52EEB5
:10A610004FB7F89421BB469A97B98AB99DB915B836
:10A62000F8B98BB91EB8E1BB32E03A95F1F700C03A
:10A6300036B1A9B1ACB121BB479A77B96AB95DB956
:10A640004FBF45E04A95F1F7000032FFE1CF8FB7E9
:10A65000F89496EC91BB469A15B890E898B993E0B7
:10A660009BB990E29EB997E891BB95E09A95F1F776
:10A6700000008FBF089526EC90EE87E0F0E8E7E455
:10A6800077EE67EF52EE4FB7F89421BB469A97B931
:10A690008AB99DB915B8F8B98BB91EB8E1BB32E0DB
:10A6A0003A95F1F700C036B1A9B1ACB121BB479AD8
:10A6B00077B96AB95DB94FBF45E04A95F1F7000037
:10A6C00032FFE1CF8FB7F89496EC91BB469A15B85C
:10A6D00092E898B993EC9BB990E29EB997E891BB48
:10A6E00095E09A95F1F700008FBF089526EC90EE63
:10A6F00087E0F0E8E7E477EE67EF52EE4FB7F894C3
:10A7000021BB469A97B98AB99DB915B8F8B98BB9E2
:10A710001EB8E1BB32E03A95F1F700C036B1A9B1FD
:10A72000ACB121BB479A77B96AB95DB94FBF45E073
:10A730004A95F1F7000032FFE1CF8FB7F89496EC1D
:10A7400091BB469A15B894E898B993E19BB992E207
:10A750009EB997E891BB95E09A95F1F700008FBFFD
:10A76000089526EC90EE87E0F0E8E7E477EE67EFF7
:10A7700052EE4FB7F89421BB469A97B98AB99DB962
:10A7800015B8F8B98BB91EB8E1BB32E03A95F1F7CC
:10A7900000C036B1A9B1ACB121BB479A77B96AB94B
:10A7A0005DB94FBF45E04A95F1F7000032FFE1CFB8
:10A7B0008FB7F89496EC91BB469A15B892E898B981
:10A7C00093E09BB990E29EB997E891BB95E09A958A
:10A7D000F1F700008FBF08952F923F924F925F9242
:10A7E0006F927F928F929F92AF92BF92CF92DF92A1
:10A7F000EF92FF920F931F93CF93DF93CDB7DEB706
:10A800006B970FB6F894DEBF0FBECDBF262F8823FF
:10A8100009F491C0E091760EF091770E4091780E98
:10A820005091790E40906A0E50906B0E2090700EF1
:10A830003090710E8091A20E9091A30E6091B50A96
:10A840007091B60A80905D0E3091670E7093F2128F
:10A850006093F112F093F412E093F3125093F61216
:10A860004093F5125092F8124092F7123092FA1279
:10A870002092F9129093FC128093FB128092FD12A9
:10A880003093FE12660F672F661F770B71958B0151
:10A890001A951A870987EE0FEF2FEE1FFF0BF19520
:10A8A0008F011A951E870D8760E070E06A017B01B9
:10A8B000CC0CDD1CEE1CFF1CCC0CDD1CEE1CFF1CAC
:10A8C000C40ED51EE61EF71E03E0F694E794D79457
:10A8D000C7940A95D1F75694479456944794369462
:10A8E0002794369427946D2C752C932CDD24EE241C
:10A8F000FF24332309F444C0323008F4D9C63BEABC
:10A90000539E412D1124469546954695742E770CFD
:10A91000740E770C770C339E312D112436953695B5
:10A920003695932E990C930E990C990C212C312C61
:10A93000412C512C27C06091B50A7091B60A8091C4
:10A94000F1129091F212E091760EF091770E861747
:10A95000970709F488C64091780E5091790E40907F
:10A960006A0E50906B0E2090700E3090710E809198
:10A97000A20E9091A30E80905D0E3091670E66CF6F
:10A98000552433241091620E1F873091E20F3E8BC5
:10A99000092F1127198B088BA090490E27FD26C17E
:10A9A000222309F423C127FD53C5213009F450C5E2
:10A9B00027FD44C4223009F441C427FD2FC32330AE
:10A9C00009F42CC327FD19C2243009F416C227FD4F
:10A9D0001BC02530C9F06B960FB6F894DEBF0FBED2
:10A9E000CDBFDF91CF911F910F91FF90EF90DF903E
:10A9F000CF90BF90AF909F908F907F906F905F901F
:10AA00004F903F902F9008958091670A882319F303
:10AA10005090660A20912B0E30912C0E3A83298398
:10AA200045E0642D872D850D0E94CF158C01209166
:10AA3000370E3091380E3E832D834BE0622D892DE9
:10AA4000850D0E94CF15811054C6B62C29853A85F4
:10AA5000A901662757FD6095762F29813A81290142
:10AA6000662457FC6094762C440E551E661E771E95
:10AA7000400E511E611C711C77FC96C74114510495
:10AA800031E0630671042CF044244A94542C612C68
:10AA9000712C0D811E81222717FD2095322F040F66
:10AAA000151F261F371F09871A872B873C872D857F
:10AAB0003E85A901662757FD6095762F09851A8581
:10AAC0002B853C85040F151F261F371F080F191FE4
:10AAD000211D311D09871A872B873C8737FD5FC7EA
:10AAE00029853A854B855C85211531054140510505
:10AAF00044F02FEF3FEF40E050E029873A874B8743
:10AB00005C870091430E1091440E41E16C2D8B2D1A
:10AB10000E94CF15A801662757FD6095762F480F34
:10AB2000591F611D711D77FD31C74115510531E078
:10AB30006307710524F04FEF5FEF60E070E00F8571
:10AB4000011104C01E89112309F4E3C6088919897B
:10AB5000000F111F28893989020F131F11950195C4
:10AB60001109222717FD2095322F400E511E621E1B
:10AB7000731E77FC5CC74114510481E068067104C0
:10AB80000CF09DC689859A85AB85BC85800F911F89
:10AB9000A21FB31FB7FD47C70097E1E0AE07B1059D
:10ABA0000CF088C6DC01040F151F261F371F37FD68
:10ABB00036C701151105F1E02F0731050CF075C6F8
:10ABC000AA2009F4F4C55092040E4092030EB093EB
:10ABD000100EA0930F0E10931C0E00931B0E8110ED
:10ABE000FACE1093F80D0093F70DF5CE80913A0A46
:10ABF000882309F4D8CEB090390A0091210E109123
:10AC0000220E1E830D8340E0642D872D8B0D2F8B2C
:10AC10000E94CF158C0140912D0E50912E0E5A831B
:10AC2000498346E0622D892D8B0D0E94CF15FC01D2
:10AC30002F8981106CC5B62C89859A85AC01662751
:10AC400057FD6095762F8D819E81AA2797FDA0954F
:10AC5000BA2F840F951FA61FB71F800F911FA11D2C
:10AC6000B11D8D839E83AF83B887B7FD78C60097EB
:10AC7000A140B10544F08FEF9FEFA0E0B0E08D83DD
:10AC80009E83AF83B88789819A81AA2797FDA09573
:10AC9000BA2F840F951FA61FB71F0D851E85A8010B
:10ACA000662757FD6095762F840F951FA61FB71F47
:10ACB0008E0F9F1FA11DB11D89839A83AB83BC8317
:10ACC000B7FD48C649815A816B817C814115510588
:10ACD0006140710544F04FEF5FEF60E070E0498341
:10ACE0005A836B837C830091390E10913A0E4CE0AD
:10ACF0006C2D8B2D2F8B0E94CF15A801662757FD39
:10AD00006095762F480F591F611D711D488F598F0F
:10AD10006A8F7B8F2F8977FD18C6688D798D8A8D14
:10AD20009B8D611571058140910544F04FEF5FEFF8
:10AD300060E070E0488F598F6A8F7B8F5F8551117B
:10AD400004C00E89002309F4DDC568897989882744
:10AD500077FD8095982F6A8B7B8B8C8B9D8B8D815B
:10AD60009E81AF81B8854A895B896C897D89840F12
:10AD7000951FA61FB71FB7FD76C6009751E0A50720
:10AD8000B1050CF06FC58C0189819A81AB81BC81C2
:10AD90004A895B896C897D89840F951FA61FB71F1F
:10ADA000B7FD5DC6009751E0A507B1050CF055C58C
:10ADB000FC01488D598D6A8D7B8D8A899B89AC8970
:10ADC000BD89480F591F6A1F7B1F77FD64C6411557
:10ADD000510591E0690771050CF03AC5A11016C53F
:10ADE0001093D60D0093D50DF093E20DE093E10D95
:10ADF0005093EE0D4093ED0DD6CD80915E0A8823E1
:10AE000009F4E5CDB0905D0A0091290E10912A0E4B
:10AE100044E0642D872D8B0D2F8B0E94CF159B8BCB
:10AE20008A8B4091350E5091360E5A8349834AE001
:10AE3000622D892D8B0D0E94CF15998F888F2F89B8
:10AE4000811081C4B62C89859A85AC01662757FD8F
:10AE50006095762FC801AA2797FDA095BA2F840F79
:10AE6000951FA61FB71F0A891B89800F911FA11D5F
:10AE7000B11D8D839E83AF83B887B7FD7EC50097D4
:10AE8000A140B10544F08FEF9FEFA0E0B0E08D83CB
:10AE90009E83AF83B88789819A81AA2797FDA09561
:10AEA000BA2F840F951FA61FB71F0D851E85A801F9
:10AEB000662757FD6095762F840F951FA61FB71F35
:10AEC000488D598D840F951FA11DB11D89839A83CB
:10AED000AB83BC83B7FD4CC569817A818B819C8132
:10AEE000611571058140910544F04FEF5FEF60E01F
:10AEF00070E049835A836B837C830091410E1091EB
:10AF0000420E40E16C2D8B2D2F8B0E94CF15A80196
:10AF1000662757FD6095762F480F591F611D711DDB
:10AF2000488F598F6A8F7B8F2F8977FD33C5688D46
:10AF3000798D8A8D9B8D611571058140910544F055
:10AF40004FEF5FEF60E070E0488F598F6A8F7B8F23
:10AF50005F85511104C00E89002309F4DEC44889BD
:10AF60005989440F551F08891989400F511FBA018B
:10AF7000882777FD8095982F6A8B7B8B8C8B9D8B98
:10AF80008D819E81AF81B8854A895B896C897D8975
:10AF9000840F951FA61FB71FB7FD51C5009751E03D
:10AFA000A507B1050CF06DC48C0189819A81AB8134
:10AFB000BC814A895B896C897D89840F951FA61F96
:10AFC000B71FB7FD58C5009751E0A507B1050CF0B4
:10AFD00053C4FC01488D598D6A8D7B8D8A899B896C
:10AFE000AC89BD89480F591F6A1F7B1F77FD3FC57C
:10AFF0004115510591E0690771050CF038C4A110A5
:10B00000F2C31093DE0D0093DD0DF093EA0DE09393
:10B01000E90D5093F60D4093F50DD9CC8091550A6A
:10B02000882309F4CFCCB090540A0091270E1091D8
:10B03000280E43E0642D872D8B0D2F8B0E94CF159A
:10B040009B8B8A8B4091330E5091340E5A834983E7
:10B0500049E0622D892D8B0D0E94CF15998F888F25
:10B060002F89811062C3B62C89859A85AC01662729
:10B0700057FD6095762FC801AA2797FDA095BA2F96
:10B08000840F951FA61FB71F0A891B89800F911F68
:10B09000A11DB11D8D839E83AF83B887B7FD9BC46F
:10B0A0000097A140B10544F08FEF9FEFA0E0B0E022
:10B0B0008D839E83AF83B88789819A81AA2797FD64
:10B0C000A095BA2F840F951FA61FB71F0D851E854B
:10B0D000A801662757FD6095762F840F951FA61F40
:10B0E000B71F488D598D840F951FA11DB11D8983F0
:10B0F0009A83AB83BC83B7FD69C469817A818B81F4
:10B100009C81611571058140910544F04FEF5FEF1F
:10B1100060E070E049835A836B837C8300913F0E2B
:10B120001091400E4FE06C2D8B2D2F8B0E94CF1570
:10B13000A801662757FD6095762F480F591F611D9E
:10B14000711D488F598F6A8F7B8F2F8977FD4CC473
:10B15000688D798D8A8D9B8D611571058140910572
:10B1600044F04FEF5FEF60E070E0488F598F6A8FD7
:10B170007B8F5F85511104C00E89002309F4B4C38D
:10B1800048895989519541955109440F551FBA0174
:10B19000882777FD8095982F6A8B7B8B8C8B9D8B76
:10B1A0008D819E81AF81B8854A895B896C897D8953
:10B1B000840F951FA61FB71FB7FD4DC4009751E020
:10B1C000A507B1050CF06CC38C0189819A81AB8114
:10B1D000BC814A895B896C897D89840F951FA61F74
:10B1E000B71FB7FD34C4009751E0A507B1050CF0B7
:10B1F00052C3FC01488D598D6A8D7B8D8A899B894C
:10B20000AC89BD89480F591F6A1F7B1F77FD1BC47E
:10B210004115510591E0690771050CF037C3A11084
:10B22000A0C21093DC0D0093DB0DF093E80DE093CA
:10B23000E70D5093F40D4093F30DC4CB80914C0A6D
:10B24000882309F4BACBB0904B0A0091250E1091D7
:10B25000260E1E830D8342E0642D872D8B0D2F8BD0
:10B260000E94CF158C014091310E5091320E5A83BD
:10B27000498348E0622D892D8B0D0E94CF15FC017A
:10B280002F89811028C2B62C89859A85AC01662742
:10B2900057FD6095762F8D819E81AA2797FDA095F9
:10B2A000BA2F840F951FA61FB71F800F911FA11DD6
:10B2B000B11D8D839E83AF83B887B7FD7EC3009792
:10B2C000A140B10544F08FEF9FEFA0E0B0E08D8387
:10B2D0009E83AF83B88789819A81AA2797FDA0951D
:10B2E000BA2F840F951FA61FB71F0D851E85A801B5
:10B2F000662757FD6095762F840F951FA61FB71FF1
:10B300008E0F9F1FA11DB11D89839A83AB83BC83C0
:10B31000B7FD4EC349815A816B817C81411551052E
:10B320006140710544F04FEF5FEF60E070E04983EA
:10B330005A836B837C8300913D0E10913E0E4EE04C
:10B340006C2D8B2D2F8B0E94CF15A801662757FDE2
:10B350006095762F480F591F611D711D488F598FB9
:10B360006A8F7B8F2F8977FDEBC2688D798D8A8DEF
:10B370009B8D611571058140910544F04FEF5FEFA2
:10B3800060E070E0488F598F6A8F7B8F5F85511125
:10B3900004C00E89002309F4AEC208891989000F80
:10B3A000111FB801882777FD8095982F6A8B7B8BBA
:10B3B0008C8B9D8B8D819E81AF81B8854A895B89FD
:10B3C0006C897D89840F951FA61FB71FB7FD5FC3CA
:10B3D000009751E0A507B1050CF035C28C018981B9
:10B3E0009A81AB81BC814A895B896C897D89840F94
:10B3F000951FA61FB71FB7FD46C3009751E0A507CD
:10B40000B1050CF01BC2FC01488D598D6A8D7B8DF6
:10B410008A899B89AC89BD89480F591F6A1F7B1F88
:10B4200077FD2DC34115510591E0690771050CF0B9
:10B4300000C2A110A9C11093DA0D0093D90DF093A9
:10B44000E60DE093E50D5093F20D4093F10DB5CA72
:10B450008091430A882309F4ABCAB090420A009154
:10B46000230E1091240E1E830D8341E0642D872D41
:10B470008B0D2F8B0E94CF158C0140912F0E509178
:10B48000300E5A83498347E0622D892D8B0D0E942F
:10B49000CF15FC012F89811010C1B62C89859A85A2
:10B4A000AC01662757FD6095762F8D819E81AA2776
:10B4B00097FDA095BA2F840F951FA61FB71F800F69
:10B4C000911FA11DB11D8D839E83AF83B887B7FDEA
:10B4D00095C20097A140B10544F08FEF9FEFA0E027
:10B4E000B0E08D839E83AF83B88789819A81AA2734
:10B4F00097FDA095BA2F840F951FA61FB71F0D8526
:10B500001E85A801662757FD6095762F840F951F2D
:10B51000A61FB71F8E0F9F1FA11DB11D89839A8380
:10B52000AB83BC83B7FD65C249815A816B817C8145
:10B53000411551056140710544F04FEF5FEF60E048
:10B5400070E049835A836B837C8300913B0E10919A
:10B550003C0E4DE06C2D8B2D2F8B0E94CF15A8013A
:10B56000662757FD6095762F480F591F611D711D85
:10B57000488F598F6A8F7B8F2F8977FDDCC1688D4B
:10B58000798D8A8D9B8D611571058140910544F0FF
:10B590004FEF5FEF60E070E0488F598F6A8F7B8FCD
:10B5A0005F85511104C00E89002309F4BDC10889CB
:10B5B0001989119501951109B801882777FD8095A2
:10B5C000982F6A8B7B8B8C8B9D8B8D819E81AF811D
:10B5D000B8854A895B896C897D89840F951FA61F70
:10B5E000B71FB7FD18C2009751E0A507B1050CF0D1
:10B5F00076C18C0189819A81AB81BC814A895B8942
:10B600006C897D89840F951FA61FB71FB7FDFFC1E9
:10B61000009751E0A507B1050CF05CC1FC01488D15
:10B62000598D6A8D7B8D8A899B89AC89BD89480F2C
:10B63000591F6A1F7B1F77FDFEC14115510591E01F
:10B64000690771050CF041C1A110BAC01093D80D63
:10B650000093D70DF093E40DE093E30D5093F00DBC
:10B660004093EF0DA5C98091F3129091F41240918F
:10B67000780E5091790EE817F90709F070C980919A
:10B68000F5129091F61240906A0E50906B0E48178A
:10B69000590709F404C22090700E3090710E809109
:10B6A000A20E9091A30E80905D0E3091670ECEC8D1
:10B6B000212C312C412C512C65C94B2D50E062E0DE
:10B6C00070E06819710902C0559547956A95E2F7CF
:10B6D000B62CB40EE3CE4B2D50E062E070E068195A
:10B6E000710902C0559547956A95E2F7B62CB40EDC
:10B6F000CBCD252D30E042E050E04819510902C081
:10B70000359527954A95E2F7B22EB60C9FC94B2D79
:10B7100050E062E070E06819710902C055954795E4
:10B720006A95E2F7B62CB40E87CA4B2D50E062E062
:10B7300070E06819710902C0559547956A95E2F75E
:10B74000B62CB40E91CC4B2D50E062E070E068193D
:10B75000710902C0559547956A95E2F7B62CB40E6B
:10B7600072CB1093000E0093FF0DF0930C0EE0933C
:10B770000B0E5093180E4093170E811023C950934F
:10B78000F40D4093F30D1EC91093FE0D0093FD0DB3
:10B79000F0930A0EE093090E5093160E4093150E87
:10B7A00081100BC95093F20D4093F10D06C95092D0
:10B7B000E00D4092DF0DB093EC0DA093EB0D11CA9C
:10B7C0001093FC0D0093FB0DF093080EE093070E11
:10B7D0005093140E4093130E8110EAC85093F00D4D
:10B7E0004093EF0DE5C81093020E0093010EF09305
:10B7F0000E0EE0930D0E50931A0E4093190E811009
:10B80000E6C85093F60D4093F50DE1C81093FA0D7C
:10B810000093F90DF093060EE093050E5093120E6F
:10B820004093110E8110BFC85093EE0D4093ED0D63
:10B83000BAC84FEF5FEF60E070E0FBCD8FEF9FEF96
:10B84000A0E0B0E0E0CD8FEF9FEFA0E0B0E0C6CD8C
:10B850004FEF5FEF60E070E0C1CA8FEF9FEFA0E0B5
:10B86000B0E0A6CA8FEF9FEFA0E0B0E08CCA4FEF28
:10B870005FEF60E070E0C3CB8FEF9FEFA0E0B0E040
:10B88000A8CB8FEF9FEFA0E0B0E08ECB4FEF5FEF44
:10B8900060E070E0C4CC8FEF9FEFA0E0B0E0A9CCF7
:10B8A0008FEF9FEFA0E0B0E08FCC0FEF1FEF20E015
:10B8B00030E086C98FEF9FEFA0E0B0E073C9442469
:10B8C0004A94542C612C712C5DC94FEF5FEF60E0FE
:10B8D00070E0BACE8FEF9FEFA0E0B0E09FCE8FEF89
:10B8E0009FEFA0E0B0E085CE0D811E81E981FA8155
:10B8F000488D598D94CC0D811E81E981FA81488D46
:10B90000598D97CD0D811E81E981FA81488D598D20
:10B9100065CAA985BA858A0153C90D811E81E9814D
:10B92000FA81488D598D6BCB0D811E81E981FA8199
:10B93000488D598D89CE188E198E1A8E1B8E1FCE6A
:10B94000188E198E1A8E1B8E10CD188E198E1A8E87
:10B950001B8EE3C919821A821B821C82B3C91D8205
:10B960001E821F8218868D819E81AF81B8857FC916
:10B9700019821A821B821C82AFCA1D821E821F82FC
:10B9800018868D819E81AF81B88579CA40E050E0EC
:10B99000BA01CBC8188E198E1A8E1B8EC8CA19868A
:10B9A0001A861B861C869CC8412C512C320166C805
:10B9B00019821A821B821C82ADCC1D821E821F82BC
:10B9C00018868D819E81AF81B88579CC19821A82C3
:10B9D0001B821C8292CB1D821E821F8218868D8143
:10B9E0009E81AF81B8855CCB188E198E1A8E1B8E06
:10B9F000AFCB19821A821B821C8296CD1D821E82B9
:10BA00001F8218868D819E81AF81B88562CD80E0CE
:10BA100090E0DC01FDCD80E090E0DC01E4CD00E0D1
:10BA200010E09801C6C880E090E0DC01B5C8412C68
:10BA3000512C3201A0C840E050E0BA01FECD80E0B8
:10BA400090E0DC01ABCA40E050E0BA01E1CB80E01D
:10BA500090E0DC01C8CB80E090E0DC01AFCB80E07F
:10BA600090E0DC019FC980E090E0DC0186C940E005
:10BA700050E0BA01BDCA80E090E0DC01A4CA40E019
:10BA800050E0BA01CFCC80E090E0DC01B6CC80E0A1
:10BA900090E0DC019DCC40E050E0BA0198C9809173
:10BAA000F7129091F8122090700E3090710E481697
:10BAB000590651F08091A20E9091A30E80905D0ED8
:10BAC0003091670E0C9426548091F9129091FA12DD
:10BAD0002816390679F78091A20E9091A30EA091B5
:10BAE000FB12B091FC1280905D0E8A179B0721F02B
:10BAF0003091670E0C9426543091FD128312F8CFCA
:10BB00003091670EA091FE123A130C9426540C94B7
:10BB1000EB547F928F929F92AF92BF92CF92DF921F
:10BB2000EF92FF920F931F93CF93DF9300D0CDB787
:10BB3000DEB71A821982C12CD12C08C08FEFC81A27
:10BB4000D80A84E6C816D10409F468C0C6010E9468
:10BB50003D1D882399F3BE016F5F7F4FC6010E9490
:10BB6000011DE980FA807FB6F89481E0E81AF108B7
:10BB7000F594E794F594E7948FEFE81AF80A0E9499
:10BB800094210E9400530E943B530E9476530E94CE
:10BB9000B1531E141F04BCF500E010E0F801EE0FD5
:10BBA000FF1FEE0FFF1FEE5FFA4E8080A180928094
:10BBB000B380882D8F770E94951F8A2D8F770E94E2
:10BBC000951F892D8F770E94951F8B2D8F770E944F
:10BBD000951F992D9295969594703A2D329536959C
:10BBE00036953270932B2B2D22952870922B882D11
:10BBF000881F8827881F892B0E94951F0F5F1F4F62
:10BC00000E151F055CF20E940C207FBE8FEFC81A34
:10BC1000D80A84E6C816D10409F098CF0F900F9087
:10BC2000DF91CF911F910F91FF90EF90DF90CF9018
:10BC3000BF90AF909F908F907F900895CF92DF92AA
:10BC4000FF920F931F93CF93DF9300D0CDB7DEB752
:10BC50008C01FFB67A8369830E94FE1C5A81698138
:10BC60008823E1F0EFEFF2E120E032E0DF01C901EB
:10BC70001D920197E9F7C62ED52E27E035E1462F14
:10BC8000B901CF010E94C46EC60181509D4E9093B0
:10BC900000158093FF14C8010E94A1488F2D0F90BA
:10BCA0000F90DF91CF911F910F91FF90DF90CF9078
:10BCB0000C94C21C2F923F924F925F926F927F9290
:10BCC0008F929F92AF92BF92CF92DF92EF92FF92AC
:10BCD0000F931F93CF93DF93CDB7DEB7C858D10929
:10BCE0000FB6F894DEBF0FBECDBF839709F0F3C245
:10BCF00080910215813009F0EEC2809103158230E7
:10BD000009F0E9C220910415AD962FAFAD97243606
:10BD100008F0E1C2DE01A45ABF4F80E090E09C0130
:10BD20002E5F3A4EF9014481F0E14F9FA0011124AA
:10BD3000F90123812F70242B2D93029680329105D7
:10BD400071F7A2962FADA297922F92959695969500
:10BD50009370A3964FADA397842F8F70880F880F91
:10BD6000892B982E990C990C812CB40160957095B3
:10BD7000AF967FAF6EAFAF97A1968FADA197A82E6C
:10BD8000A694AA0CAA0CA0963FADA097932F9695C7
:10BD900096959695FF24F394F822F294FF0CB0EE5A
:10BDA000FB22F92AFF0CFF0C582F551F5527551F52
:10BDB0002F73220F922F952B80E0BC0161507048A9
:10BDC000E1967FAF6EAFE1976D968FAD6D97782F4F
:10BDD000770FC058DF4F7883C058D040AA962FAD58
:10BDE000AA97922F9E7FCF57DF4F9883C158D0409C
:10BDF00042954F70A4969FADA49717E0D12ED922FB
:10BE0000D29400EFD022D42A492F469546954695E4
:10BE1000A5969FADA597092F01700295000F007E92
:10BE2000042B000F000F692F660F660F562F5877EF
:10BE300040E0BA017058E3967FAF6EAFE397492FA9
:10BE4000429546954770A6969FADA697A92FA170DB
:10BE5000AA0FAA0FAA0FA42BB0E0A25DB84F7C9145
:10BE6000EB967FAFEB97B92EB694B29440EFB42225
:10BE7000492F429546954770A7969FADA797A92F42
:10BE8000A170AA0FAA0FAA0FA42BB0E0A25DB84F11
:10BE90004C91EC964FAFEC97A92FA695AF70B0E000
:10BEA000A25DB84F6C91ED966FAFED97492F42951B
:10BEB00046954770A8969FADA897A92FA170AA0F85
:10BEC000AA0FAA0FA42BB0E0A25DB84F7C91EE960A
:10BED0007FAFEE97C92EC694C29450EFC5229295BB
:10BEE00096959770A9964FADA997A42FA170AA0F08
:10BEF000AA0FAA0FA92BB0E0A25DB84F9C91EF96B4
:10BF00009FAFEF97A42FA695AF70B0E0A25DB84F9A
:10BF10006C91C158DF4F6883CF57D040881F882766
:10BF2000881F6E965FAD6E97652F6770660F682BE2
:10BF3000962F990F990F990F80E0BC017058E596E4
:10BF40007FAF6EAFE597952F991F9927991F6F9631
:10BF50008FAD6F97182F1F73110F192B110F952F7E
:10BF600096959C7382958695869583703770330F6E
:10BF7000330F382B80E1389FB0011124E7967FAF53
:10BF80006EAFE7974295469547702170220F220FBA
:10BF9000220F242B40E050E029F0522F550F550F6F
:10BFA00040E05054AC964FACAC97742D717041FA90
:10BFB000662760F9AB968FADAB97282F2170E89676
:10BFC0002FAFE89743FA332730F9E9963FAFE99767
:10BFD00044FA332730F981FB222720F942FA222440
:10BFE00020F845FA332430F846FA442440F884FB1C
:10BFF000552450F886FBEE27E0F9F0E0EE0FFF1F26
:10C0000087FBEE24E0F8EE0CEE0CEE2A85FBEE2723
:10C01000E0F9EE2A83FB662460F882FF02C082E02A
:10C0200001C080E0680EAC967FACAC9777FA7724BD
:10C0300070F88FB7EA968FAFEA97CB57DF4F288318
:10C04000C558D040CC57DF4F3883C458D040CA576A
:10C05000DF4F4883C658D040C957DF4F5883C75871
:10C06000D040CD57DF4F6883C358D040CE57DF4F05
:10C070007883C258D040C857DF4F9883C858D04003
:10C080000E94BF1CCB57DF4F2881C558D040CC57EA
:10C09000DF4F3881C458D040CA57DF4F4881C65857
:10C0A000D040C957DF4F5881C758D040CD57DF4FD8
:10C0B0006881C358D040CE57DF4F7881C258D040F6
:10C0C000C857DF4F9881C858D040882309F4E5C08D
:10C0D0008BE5E1E5FEE0DE01119601900D928A9577
:10C0E000E1F77093510E6093520EE8966FADE897AA
:10C0F0006093530EE9967FADE9977093540E309399
:10C10000550E2093560E2092570E3092580E4092A4
:10C11000590E50925A0E10925B0EE0925C0E609295
:10C120005D0E10925E0E81E080935F0E1092600EA5
:10C130008093610E7092620E1092630E23E0209342
:10C14000640E8093650E22E02093660E8093670E46
:10C1500010926A0EA0926B0EAF962EAD3FADAF97C8
:10C1600030936D0E20936C0E10926E0EC058DF4F00
:10C170003881C058D04030936F0E1092700EF092FC
:10C18000710E9092730E8092720E1092740ECF57B1
:10C19000DF4F6881C158D0406093750EE1962EAD97
:10C1A0003FADE1973093770E2093760E1092780E84
:10C1B000D092790E10927A0E00937B0EE3966EADBC
:10C1C0007FADE39770937D0E60937C0E10927E0E90
:10C1D000EB967FADEB9770937F0E1092800EB0922E
:10C1E000810E1092820EEC962FADEC972093830E69
:10C1F0001092840EED963FADED973093850E109220
:10C20000860EEE966FADEE976093870E1092880EB5
:10C21000C092890E10928A0EEF967FADEF977093C1
:10C220008B0E10928C0EC158DF4F2881CF57D04013
:10C2300020938D0EE5966EAD7FADE59770938F0ED2
:10C2400060938E0E1092900E1093910E1092920E9B
:10C250009093930EE7962EAD3FADE7973093950EF2
:10C260002093940E5093970E4093960E1092990E31
:10C270001092980E10929B0E10929A0EAD968FAD62
:10C28000AD9790E00E94B2488BE5FE013196A1E5A2
:10C29000BEE001900D928A95E1F7EA968FADEA979C
:10C2A000C857DF4F0FB6F894DEBF0FBECDBFDF918A
:10C2B000CF911F910F91FF90EF90DF90CF90BF90A3
:10C2C000AF909F908F907F906F905F904F903F9036
:10C2D0002F900C94BD1CC857DF4F0FB6F894DEBFEB
:10C2E0000FBECDBFDF91CF911F910F91FF90EF90C7
:10C2F000DF90CF90BF90AF909F908F907F906F9086
:10C300005F904F903F902F9008952F923F924F92C1
:10C310005F926F927F928F929F92AF92BF92CF92D5
:10C32000DF92EF92FF920F931F93CF93DF93803FA3
:10C3300009F440C0873FB1F02091710A3091720A30
:10C34000211592E039070CF456C041E050E020E09E
:10C3500030E0F901EE5FFA4E80835093720A409309
:10C36000710A36C080910215813009F448C08111EC
:10C3700009C080910315813629F480910415863116
:10C3800009F448C01092720A1092710ADF91CF919D
:10C390001F910F91FF90EF90DF90CF90BF90AF90E3
:10C3A0009F908F907F906F905F904F903F902F90D5
:10C3B0000C9462351092720A1092710A80E092E039
:10C3C000E2E0F5E1DF019C011D9221503040E1F7F0
:10C3D000DF91CF911F910F91FF90EF90DF90CF9061
:10C3E000BF90AF909F908F907F906F905F904F9095
:10C3F0003F902F900895A9014F5F5F4FAACF809182
:10C400000315823009F0BECF8091710A9091720AB3
:10C4100051DCB8CF80910515813009F0B3CF809100
:10C42000710A9091720A049765E070E00E94CC6AEC
:10C430001B0177FD72C0E6E0AE2EE5E1BE2EF7E00F
:10C44000CF2EF5E1DF2EA8E0EA2EA5E1FA2E09E0D5
:10C4500015E12B01440C551C440C551C460E571E6F
:10C4600039E0430E511CC4E0D0E084E0682E712C0A
:10C4700072E0872E75E1972E8C0E9D1E44E050E0F1
:10C48000B401C3018E5F9A4E0E94CD6ED401149602
:10C490002C91B0E82B9FC0011124F5019081982BBD
:10C4A0009083922F92709295990F990F907CD6015C
:10C4B0008C91982B9C93922F94709295990F907ECB
:10C4C000F7018081982B9083822F88708295807FDE
:10C4D000D8019C91892B8C93B4E06B0E711C25962E
:10C4E000E4E0AE0EB11CF4E0CF0ED11C24E0E20E6D
:10C4F000F11C0C5F1F4FC415D50509F0B9CFC10160
:10C500000296880F991F880F991FBC016550710909
:10C510008091061590E092DB35CF84E090E0F5CF76
:10C52000EF92FF920F93CF93DF931F92CDB7DEB7B9
:10C530007B016091710A7091720A6115710529F091
:10C54000E61AF70A81E0E81AF108E114F10439F477
:10C550000F90DF91CF910F91FF90EF900895842F6E
:10C560002983D3DE2981E2E0EE16F10488F3822FDD
:10C57000CCDEF2E0EF16F10459F3802F0F90DF913B
:10C58000CF910F91FF90EF90C0CE1F920F920FB6F8
:10C590000F9211240F900FBE0F901F9018951F92AD
:10C5A0000F920FB60F9211240F900FBE0F901F9095
:10C5B00018951F920F920FB60F9211240BB60F927F
:10C5C0001F932F933F934F935F936F937F938F931B
:10C5D0009F93AF93BF93CF93DF93EF93FF933499E0
:10C5E0009BC0CFB7F89456EC51BB469A70EE77B922
:10C5F00067E06AB97DB915B8D0E8D8B96BB91EB88B
:10C60000B7E4B1BB82E08A95F1F700C026B199B1D9
:10C610008CB151BB479A422F46954370E0E82E9F5C
:10C6200090011124422B292F2071422B292F26956E
:10C6300026952870422B96959076492B90E0880F8E
:10C64000991F84709927482BA7EEA7B9F7EFFAB97D
:10C65000E2EEEDB985E08A95F1F7000047FF5BC097
:10C6600040FF59C051BB469A77B96AB97DB915B830
:10C67000D8B96BB980E28EB9B1BB82E08A95F1F787
:10C6800000C026B199B18CB151BB479AD22FD69533
:10C69000D37050E8259F90011124D22B292F2071AF
:10C6A000D22B292F269526952870D22B96959076F9
:10C6B000D92B90E0880F991F84709927D82BA7B9A0
:10C6C000FAB9EDB985E08A95F1F7000044FD3AC06A
:10C6D0001FB7F8942091EB1730E0C90101966091E3
:10C6E000EC1770E059D74091EA1750E0841795078E
:10C6F00089F0E091ED17F091EE17E20FF31FD08370
:10C700008091EB1790E001966091EC1770E044D7B0
:10C710008093EB171FBFCFBFFF91EF91DF91CF91B8
:10C72000BF91AF919F918F917F916F915F914F9149
:10C730003F912F911F910F900BBE0F900FBE0F9046
:10C740001F9018950E945321E6CF1F920F920FB6AB
:10C750000F9211240BB60F922F933F934F935F9339
:10C760006F937F938F939F93AF93BF93CF93DF93F9
:10C77000EF93FF93CEE6D0E088818D7F888385B3E9
:10C78000876085BB78940E944602F8948881826015
:10C790008883FF91EF91DF91CF91BF91AF919F91EE
:10C7A0008F917F916F915F914F913F912F910F905A
:10C7B0000BBE0F900FBE0F901F901895CF93DF9375
:10C7C000CDB7DEB764970FB6F894DEBF0FBECDBF0E
:10C7D00020E82093610010926100F89414B817B813
:10C7E0001AB81DB810BA15B880EE88B91BB81EB8B3
:10C7F00093EE91BB3FEF34B987B947E04AB98DB9A1
:10C8000090BB9CE797BD94B5926094BD95B593603D
:10C8100095BD90916E00926090936E00EC9A96ECAC
:10C8200091BB469A87B94AB98DB915B828B91BB8D2
:10C830001EB887E481BB42E04A95F1F700C086B19B
:10C8400089B18CB191BB479A87EE87B987EF8AB9D6
:10C8500082EE8DB907EA1BE08AEA92E0D801FC017A
:10C860001D923197E9F7E1E6F9E0DF011D922A9583
:10C87000E9F781E4E1EEF9E0DF011D928A95E9F73D
:10C8800080E28093F00985E4E9EDFAE0DF011D9292
:10C890008A95E9F786E6E3E7FAE0DF011D928A95DB
:10C8A000E9F73093D80A0E94791E8FE4E2E2FAE0B9
:10C8B000DF011D928A95E9F78FE380936F0A46E0C6
:10C8C00050E06FEF70E088E69AE00E94DE6E109212
:10C8D000680A0E94532189E8EEE1FBE0DF011D9226
:10C8E0008A95E9F78FEF2FEF8193BBE0EE39FB07D5
:10C8F000D1F78FEF9FEF90939F0B80939E0B209328
:10C90000A00B8DE0ECEAFEE0DF011D928A95E9F7CD
:10C910002093AD0E2093AF0E8FEF9FEFDC0180933D
:10C92000B00E9093B10EA093B20EB093B30E81E00F
:10C930008093AE0E2093B80E1092271710922917ED
:10C940001092281780EC8093EC178AE297E190937D
:10C95000EE178093ED171092EB171092EA171092D2
:10C960000B1710920A1710920F1710920E171092B1
:10C970001317109212171092151710921417109285
:10C9800017171092161710921B1710921A17109261
:10C990001F1710921E171092211710922017109235
:10C9A00023171092221783EE9FE190930317809331
:10C9B00002178DE194E2909307178093061784E0A5
:10C9C00094E2909309178093081782EF97E490936D
:10C9D00005178093041782EC97E4909311178093C6
:10C9E00010178EE995E490930D1780930C1780E94A
:10C9F00092E690931D1780931C1784EE91E190931B
:10CA00001917809318171092720A1092710A8AE20D
:10CA1000E3EAFCE0DF01282F1D922A95E9F7D8010F
:10CA2000E82F1D92EA95E9F7EDECFCE0DF01282FF5
:10CA30001D922A95E9F7E1EDFBE0DF01282F1D9219
:10CA40002A95E9F7E7EFFCE0DF01282F1D922A95F0
:10CA5000E9F7EBEFFBE0DF01282F1D922A95E9F7BC
:10CA6000E1E2FDE0DF01282F1D922A95E9F7E5E2DA
:10CA7000FCE0DF01282F1D922A95E9F7EBE4FDE0A9
:10CA8000DF01282F1D922A95E9F7EFE4FCE0DF0192
:10CA9000282F1D922A95E9F7E5E7FDE0DF01282F11
:10CAA0001D922A95E9F7E9E7FCE0DF011D928A95DE
:10CAB000E9F78FE99DE00E941F1F8AEB9DE00E942D
:10CAC0001F1F61E08AEB9DE00E94FA1E64E08AEB82
:10CAD0009DE00E94601C8BED90E00E943D1D811145
:10CAE00006C00E94A81D8BED90E00E94B2480E94F3
:10CAF000011E811104C00E94D11E0E94384981E0AC
:10CB00000E94F34A8091D70A00E210E046E1D42E59
:10CB10000E944A502091D70A203109F407C13327D7
:10CB200027FD30952F5F3F4F2F71307837FF06C0BC
:10CB300021503109206E3F6F2F5F3F4F822F20938E
:10CB4000D70A0150110921F781E00E944A5080E183
:10CB50000E944A508EE10E944A508DE10E944A5044
:10CB60000E9420370E9462358EE397E00E943D19B3
:10CB7000789406ECC02EBB24B39487E8D82E93E4B7
:10CB8000892E20EF922E30EAA32E9FB7F894809141
:10CB9000E30F8F5F8093E30FC1BA469A80FBEE24C8
:10CBA000E0F8F12CEE0CFF1CEE0CFF1CB1E3EB2ABD
:10CBB0008E2D86958270806CB5B8E2E4E8B9F0E518
:10CBC000FBB98EB9D1BA9FBF1092730A1092740A42
:10CBD0001092750A1092760A2FEF2093D80A80914E
:10CBE000D70A0E944A502091D70A203109F44CC13B
:10CBF000332727FD30952F5F3F4F2F71307837FD5A
:10CC0000FFC3822F2093D70A0E944A502091D70A4F
:10CC1000203109F434C1332727FD30952F5F3F4F72
:10CC20002F71307837FDE5C3822F2093D70A0E94F9
:10CC30004A502091D70A203109F41DC1332727FD1E
:10CC400030952F5F3F4F2F71307837FDCBC3822F48
:10CC50002093D70A0E944A508091D70A803109F464
:10CC600006C1992787FD909501968F71907897FD61
:10CC7000CEC38093D70A81E00E944A5080E10E948F
:10CC80004A508EE10E944A508DE10E944A50109114
:10CC9000D80A1F3F11F41091AF0E1093AF0E173149
:10CCA00009F4A2C08091730A9091740AA091750A48
:10CCB000B091760A0091AE0E2091DD0FE4E7F6E028
:10CCC0002223C1F12AE63EE0212E332427FC3094B2
:10CCD000898B9A8BAB8BBC8B22C0462F552747FD87
:10CCE000509549885A886B887C8804C076946794EC
:10CCF000579447946A95D2F740FE0BC0440F551FD6
:10CD00004956554FDA014D915C91D9014D935C9391
:10CD100001E02E5F3F4FB6E0E239FB0711F1619170
:10CD20006F3FB9F36113D9CFA101E8CFD092D70AF1
:10CD300086E107CFAAE6BEE09D0181918F3F59F0C1
:10CD4000880F990B8956954FDC018D919C91D901E3
:10CD50008D939C9301E02E5F3F4FB6E0E239FB07D5
:10CD600061F70093AE0E1F3F61F1E12FEE0FFF0B55
:10CD7000E956F54F80819181A0E0B0E04091B00E7E
:10CD80005091B10E6091B20E7091B30E8417950759
:10CD9000A607B707B1F08093B00E9093B10EA093A1
:10CDA000B20EB093B30E0E946F4F8091AF0E8631DA
:10CDB00009F4A3C3803109F4B7C38450883008F460
:10CDC00086C34091E30F4370423009F4ACC0433056
:10CDD00009F45FC0413009F4FAC10E94A1446FEF29
:10CDE00080E00E94EC53D1CEE091B80EE7FD5ACF1F
:10CDF0002091C50A3091C60AA90160E070E08091D7
:10CE0000B00E9091B10EA091B20EB091B30E481732
:10CE100059076A077B0709F445CFFF27E7FDF0951F
:10CE2000CF01880F991F8E0F9F1F880F991F880FA2
:10CE3000991F8C579A4FFC01DE0111961CE001905E
:10CE40000D921A95E1F7DC010C9111961C910111DC
:10CE5000E3C2E12FEE0FFF0BEF5AF14F328F218F1C
:10CE6000B092AE0E0E9462351091AF0E1BCF96E1CC
:10CE70009093D70A00CF86E18093D70AEBCE56E194
:10CE80005093D70A86E1D3CE46E14093D70A86E194
:10CE9000BBCE0E941F3400E010E423E035E440E004
:10CEA00050EE6BE276E48091960E9091970E0E9480
:10CEB0008E1B9C019093480E8093470E81E0203D8D
:10CEC00037400CF080E08093490E8091A40E909141
:10CED000A50E2091E10F222309F400C3AC0160E00C
:10CEE00070E0DB01CA01880F991FAA1FBB1F880FC2
:10CEF000991FAA1FBB1F880F991FAA1FBB1F840F52
:10CF0000951FA61FB71F880F991FAA1FBB1FFD01E2
:10CF1000EE0FFF1FEE56F94F808191819093A40B85
:10CF20008093A30B5CCF80916C0E90916D0E6FB7C8
:10CF3000F8949C01232F332726952695722FC1BA8A
:10CF4000469A522F550F452F46704068207133275F
:10CF50002260352F330F3072322B507C352B272F28
:10CF600026952270206215B848B93BB92EB9D1BABE
:10CF70009695879596958795282FC1BA469A482FFA
:10CF8000440F382F3695221F2227221F542F567008
:10CF9000252B2068807199278260942F990F9072B9
:10CFA000982B407C942B327015B828B99BB93EB9A8
:10CFB000D1BAC1BA469AB5B888B89BB8AEB8D1BA9A
:10CFC00095E09A95F1F70000C1BA469AB5B888B8CD
:10CFD00050E75BB9AEB8D1BAAAE0AA95F1F700C0A4
:10CFE000C1BA469AB5B888B89BB8AEB8D1BABAE05B
:10CFF000BA95F1F700C06FBF8091720E9091730ED9
:10D000006FB7F8949C01232F332726952695E22F9E
:10D01000C1BA469A722F770F472F46704068207129
:10D0200033272260372F330F3072322B707C372B2F
:10D030002E2F26952270206215B848B93BB92EB91B
:10D04000D1BA9695879596958795282FC1BA469A15
:10D05000482F440F382F3695221F2227221F742F66
:10D060007670272B2068807199278260942F990F02
:10D070009072982B407C942B327015B828B99BB9CC
:10D080003EB9D1BAC1BA469AB5B885E488B99BB859
:10D09000AEB8D1BAE5E0EA95F1F70000C1BA469A18
:10D0A000B5B888B95BB9AEB8D1BAFAE0FA95F1F77C
:10D0B00000C0C1BA469AB5B888B99BB8AEB8D1BA63
:10D0C0002AE02A95F1F700C06FBF2091B30A309192
:10D0D000B40A8091450E9091460EAA2797FDA0951F
:10D0E000BA2F820F931FA11DB11DB7FDF3C1009789
:10D0F00041E0A407B10524F08FEF9FEFA0E0B0E07E
:10D100005FB7F8949C01232F332726952695722F1D
:10D11000C1BA469A622F660F462F4670406820714A
:10D1200033272260362F330F3072322B607C362B40
:10D13000272F26952270206215B848B93BB92EB921
:10D14000D1BA9695879596958795282FC1BA469A14
:10D15000482F440F382F3695221F2227221F642F75
:10D160006670262B2068807199278260942F990F12
:10D170009072982B407C942B327015B828B99BB9CB
:10D180003EB9D1BAC1BA469AB5B887E488B99BB856
:10D19000AEB8D1BA95E09A95F1F70000C1BA469AB7
:10D1A000B5B888B990E79BB9AEB8D1BAAAE0AA954C
:10D1B000F1F700C0C1BA469AB5B888B99BB8AEB805
:10D1C000D1BABAE0BA95F1F700C05FBF08CE80913E
:10D1D000900E9091910E6FB7F8949C01232F3327F6
:10D1E00026952695E22FC1BA469A722F770F572FB0
:10D1F00056705068207133272260372F330F3072FA
:10D20000322B707C372B2E2F26952270206215B87A
:10D2100058B93BB92EB9D1BA969587959695879509
:10D22000282FC1BA469A582F550F382F3695221FEE
:10D230002227221F752F7670272B2068807199274F
:10D240008260952F990F9072982B507C952B32709D
:10D2500015B828B99BB93EB9D1BAC1BA469A45B9F1
:10D2600081E488B99BB8AEB8D1BAE5E0EA95F1F7A8
:10D270000000C1BA469A45B988B950E75BB9AEB863
:10D28000D1BAFAE0FA95F1F700C0C1BA469A45B9A9
:10D2900088B99BB8AEB8D1BA2AE02A95F1F700C098
:10D2A0006FBF80917A0E90917B0E6FB7F8949C01BE
:10D2B000232F332726952695F22FC1BA469AE22FBF
:10D2C000EE0F7E2F767070682071332722603E2F1C
:10D2D000330F3072322BE07C3E2B2F2F269522709D
:10D2E000206215B878B93BB92EB9D1BA9695879511
:10D2F00096958795282FC1BA469A782F770F382FA1
:10D300003695221F2227221FE72FE6702E2B20683A
:10D31000807199278260972F990F9072982B707C5B
:10D32000972B327015B828B99BB93EB9D1BAC1BA9A
:10D33000469A45B995E498B99BB882EA8EB9D1BAB4
:10D34000A5E0AA95F1F70000C1BA469A45B998B987
:10D350005BB98EB9D1BABAE0BA95F1F700C0C1BADB
:10D36000469A45B998B99BB88EB9D1BAEAE0EA9520
:10D37000F1F700C06FBF2FB7F894C1BA469A15B83D
:10D3800090E898B932E33BB930E23EB9D1BAC1BABC
:10D39000469A15B898B992E09BB91EB8D1BAC1BAED
:10D3A000469A45B988B89BB88EB9D1BAF5E0FA95D6
:10D3B000F1F70000C1BA469A45B988B85BB98EB991
:10D3C000D1BA5AE05A95F1F700C0C1BA469A45B9A8
:10D3D00088B89BB88EB9D1BA8AE08A95F1F700C0B7
:10D3E0002FBFFDCC21503109206E3F6F2F5F3F4F83
:10D3F0002ECC21503109206E3F6F2F5F3F4F14CC50
:10D4000021503109206E3F6F2F5F3F4FFACB0197BC
:10D41000806E9F6F01962DCC033008F021CD2D87B3
:10D420005E876F87788B0E944E1A8D819E814D8515
:10D430005E856F857889892B09F4A4C08F819885D2
:10D44000892B09F489C089859A85892B09F480C0C4
:10D450008B859C85892B09F485C0440F551F661F59
:10D46000771F440F551F661F771F2B01772457FC2A
:10D470007094672C8091B40E9091B50EA091B60E69
:10D48000B091B70E481659066A067B0671F0F20194
:10D490003296EE0FFF1F41E050E04C0F5D1FE40F8E
:10D4A000F51F808191810E943D190130B9F5E12F6E
:10D4B000FF27E7FDF095EF5AF14F40824092B40EFE
:10D4C0005092B50E6092B60E7092B70EC9CC0E9403
:10D4D000E63B77CC80E090E0DC0109CE00E010E094
:10D4E0002AEF33E440E050EE6BEA76E40E948E1BB4
:10D4F0009093A40B8093A30B72CC0091C30A10915C
:10D50000C40A10931E0E00931D0E0E94A14442E017
:10D51000B80180E090E00E943E1453CCB301A20118
:10D52000812F0E94671ACACF0E94CF218C0190934D
:10D53000200E80931F0E0E944F176FEF81E00E9414
:10D54000EC5341E060E070E0C8010E943E1439CC29
:10D55000440F551F661F771F2B01772457FC7094CB
:10D56000672C88CF2A013B01440C551C661C771C94
:10D57000440E551E661E771E2301772457FC7094B7
:10D58000672C78CF412C512C320174CFB2D4B7FF25
:10D590000895821B930B089597FB072E16F40094B1
:10D5A00006D077FD08D00BD007FC05D03EF490954F
:10D5B00081959F4F0895709561957F4F0895AA1B9F
:10D5C000BB1B51E107C0AA1FBB1FA617B70710F06E
:10D5D000A61BB70B881F991F5A95A9F780959095A0
:10D5E000BC01CD0108955058BB27AA270ED0C9C150
:10D5F00092D130F097D120F031F49F3F11F41EF416
:10D6000062C10EF4E095E7FB58C1E92FDCD180F34D
:10D61000BA17620773078407950718F071F49EF52F
:10D62000F4C10EF4E0950B2EBA2FA02D0B01B90119
:10D6300090010C01CA01A0011124FF27591B99F088
:10D64000593F50F4503E68F11A16F040A22F232F94
:10D65000342F4427585FF3CF469537952795A795E4
:10D66000F0405395C9F77EF41F16BA0B620B730B8B
:10D67000840BBAF09150A1F0FF0FBB1F661F771FFC
:10D68000881FC2F70EC0BA0F621F731F841F48F4B1
:10D69000879577956795B795F7959E3F08F0B3CF37
:10D6A0009395880F08F09927EE0F97958795089521
:10D6B00041D1E39577C10CD064C134D140F02BD176
:10D6C00030F021F45F3F19F0F8C051119FC1FBC049
:10D6D0007AD198F39923C9F35523B1F3951B550BD0
:10D6E000BB27AA2762177307840738F09F5F5F4F35
:10D6F000220F331F441FAA1FA9F333D00E2E3AF076
:10D70000E0E830D091505040E695001CCAF729D08F
:10D71000FE2F27D0660F771F881FBB1F26173707DE
:10D720004807AB07B0E809F0BB0B802DBF01FF270E
:10D7300093585F4F2AF09E3F510568F0BEC066C106
:10D740005F3FECF3983EDCF3869577956795B79548
:10D75000F7959F5FC9F7880F911D9695879597F963
:10D760000895E1E0660F771F881FBB1F62177307DC
:10D770008407BA0720F0621B730B840BBA0BEE1FF1
:10D7800088F7E095089519F40EF097C03EC19BC04C
:10D7900022D1C8F39638C0F707F80F92E8942BE32C
:10D7A0003AEA48EB5FE7BAD10F920F920F924DB76A
:10D7B0005EB70F9272D1ECEAF0E088D04F915F91A2
:10D7C000EF91FF91E595EE1FFF1F49F0FE57E068CE
:10D7D0004427EE0F441FFA95E1F74195550B29D1E7
:10D7E0000F9007FE1DC10895F6D088F09F5790F066
:10D7F000B92F9927B751A0F0D1F0660F771F881F76
:10D80000991F1AF0BA95C9F712C0B13081F0FDD056
:10D81000B1E00895FAC0672F782F8827B85F39F0F4
:10D82000B93FCCF3869577956795B395D9F73EF4D4
:10D8300090958095709561957F4F8F4F9F4F08957C
:10D84000E89409C097FB3EF490958095709561959A
:10D850007F4F8F4F9F4F9923A9F0F92F96E9BB2750
:10D860009395F695879577956795B795F111F8CFCC
:10D87000FAF4BB0F11F460FF1BC06F5F7F4F8F4F37
:10D880009F4F16C0882311F096E911C0772321F02D
:10D890009EE8872F762F05C0662371F096E8862FC5
:10D8A00070E060E02AF09A95660F771F881FDAF71C
:10D8B000880F9695879597F9089597F99F6780E85F
:10D8C00070E060E008959FEF80EC0895DF93CF93C0
:10D8D0001F930F93FF92EF92DF927B018C0168946C
:10D8E00005C0DA2EEF0118D1FE01E894A59125912B
:10D8F000359145915591AEF3EF0187DEFE01970119
:10D90000A801DA9479F7DF90EF90FF900F911F91C3
:10D91000CF91DF91089500240A9416161706180671
:10D920000906089500240A94121613061406050623
:10D930000895C9CF50D0E8F3E894E0E0BB279F57A3
:10D94000F0F02AED3FE049EC06C0EE0FBB0F661F7A
:10D95000771F881F28F0B23A62077307840728F000
:10D96000B25A620B730B840BE3959A9572F7803869
:10D9700030F49A95BB0F661F771F881FD2F7904827
:10D9800094C1092E0394000C11F4882352F0BB0FAC
:10D9900040F4BF2B11F460FF04C06F5F7F4F8F4FC7
:10D9A0009F4F0895EF93E0FF06C0A2EA2AED3FE003
:10D9B00049EC5FEB2ADEE5DF0F90039401FC905801
:10D9C000E4EDF0E07EC157FD9058440F551F59F02B
:10D9D0005F3F71F04795880F97FB991F61F09F3F5C
:10D9E00079F087950895121613061406551FF2CF85
:10D9F0004695F1DF08C0161617061806991FF1CFD5
:10DA000086957105610508940895E894BB276627FB
:10DA10007727CB0197F9089522D108F48FEF089565
:10DA20009B01AC0160E070E080E89FE344CE45CF0D
:10DA30003AC1D1DFE8F39923D9F3940F511DBBF319
:10DA40009150504094F059F0882332F0660F771FC0
:10DA5000881F91505040C1F79E3F510544F7880FF1
:10DA6000911D9695879597F908955F3FACF0983E84
:10DA70009CF0BB27869577956795B79508F4B160BC
:10DA80009395C1F7BB0F58F711F460FFE8CF6F5FB4
:10DA90007F4F8F4F9F4FE3CFB9CFFA01DC01AA0F21
:10DAA000BB1F9B01AC01BF5728F422273327442713
:10DAB00050781FC0B75188F4AB2F00244695379596
:10DAC0002795011CA395D2F3002069F0220F331F84
:10DAD000441FB395DAF30DD086CD61307105A0E80F
:10DAE0008A07B94630F49B01AC016627772788275F
:10DAF0009078309621F020833183428353830895B8
:10DB00000BD03FCF08DF28F00DDF18F0952309F088
:10DB1000D4CED9CE11247ACF56DFA0F3959FD1F37E
:10DB2000950F50E0551F629FF001729FBB27F00DCB
:10DB3000B11D639FAA27F00DB11DAA1F649F662720
:10DB4000B00DA11D661F829F2227B00DA11D621F6F
:10DB5000739FB00DA11D621F839FA00D611D221F29
:10DB6000749F3327A00D611D231F849F600D211D0D
:10DB7000822F762F6A2F11249F5750408AF0E1F0B0
:10DB800088234AF0EE0FFF1FBB1F661F771F881FF9
:10DB900091505040A9F79E3F510570F08ECE36CF80
:10DBA0005F3FECF3983EDCF3869577956795B795E4
:10DBB000F795E7959F5FC1F7FE2B880F911D96950E
:10DBC000879597F90895FA01EE0FFF1F309621050A
:10DBD000310599F16115710561F48038BFE39B0748
:10DBE00049F168949038810561F08038BFEF9B0758
:10DBF00041F0992342F5FF3FE1053105210511F17F
:10DC0000E8940894E795D901AA2329F4AB2FBE2FF5
:10DC1000F85FD0F310C0FF5F70F4A695E0F7F73916
:10DC200050F019F0FF3A38F49F779F930CD00F9083
:10DC300007FC905808953EF046CE60E070E080E822
:10DC40009FE308954FE79F775F934F933F932F9301
:10DC50004ED02F913F914F915F9152DF99CD990F07
:10DC60000008550FAA0BE0E8FEEF16161706E807A6
:10DC7000F907C0F012161306E407F50798F0621BC7
:10DC8000730B840B950B39F40A2661F0232B242B9C
:10DC9000252B21F408950A2609F4A140A6958FEFBB
:10DCA000811D811D08959F3F31F0915020F487958B
:10DCB00077956795B795880F911D9695879597F9F4
:10DCC00008959F938F937F936F93FF93EF939B019F
:10DCD000AC0116DFEF91FF91F9DD2F913F914F914C
:10DCE0005F910ECF0EF0DFCFEECD6894E6CD73DE00
:10DCF000C8F39923D1F3C6F3DF93CF931F930F9308
:10DD0000FF92C92FDD2788232AF02197660F771FFE
:10DD1000881FDAF720E030E040E85FEB9FE38839C6
:10DD200020F0803E30F021968F775EDCE2EFF0E06D
:10DD300003C05ADCEFE1F1E0C9DD8B01BE01EC016B
:10DD4000FB2E6F5771097595771F880B990B7ADD3C
:10DD500028E132E741E35FE3DFDEAF2D9801AE015A
:10DD6000FF900F911F91CF91DF914FDC0ACEFB0105
:10DD7000DC0104C08D910190801921F44150504084
:10DD8000C8F7881B990B0895FB01DC0102C00190C4
:10DD90000D9241505040D8F708956817790768F4FC
:10DDA000FB01DC01E40FF51FA40FB51F02C00290B8
:10DDB0000E9241505040D8F70895E6CFDC0101C0E3
:10DDC0006D9341505040E0F70895FB01DC010D9048
:10DDD0000020E9F7119701900D920020E1F70895D6
:10DDE000FB01DC0101900D920020E1F708958F9274
:10DDF0009F92AF92BF92CF92DF92EF92FF92CF931A
:10DE0000DF93EC01688179818A819B8161157105BD
:10DE10008105910521F464E279ED8BE597E02DE130
:10DE200033EF41E050E04AD049015A019B01AC0177
:10DE3000A7EAB1E433D06B017C01ACEEB4EFA501ED
:10DE4000940138D0C60ED71EE81EF91EF7FE06C094
:10DE500081E0C81AD108E10880E8F80AC882D982AE
:10DE6000EA82FB82E894F7F8B601C701DF91CF910F
:10DE7000FF90EF90DF90CF90BF90AF909F908F90EA
:10DE80000895B5CF80E891E0B2CF609380017093A0
:10DE90008101809382019093830108952AD0A59FE8
:10DEA000900DB49F900DA49F800D911D1124089595
:10DEB000B7FFF4CFF3DF821B930B0895052E97FB7A
:10DEC00016F4009406D057FD0CD01FD007FC09D0E3
:10DED0007EF490958095709561957F4F8F4F9F4F01
:10DEE000089550954095309521953F4F4F4F5F4F86
:10DEF0000895A29FB001B39FC001A39F01D0B29F1C
:10DF0000700D811D1124911D0895A1E21A2EAA1BE6
:10DF1000BB1BFD010DC0AA1FBB1FEE1FFF1FA217D9
:10DF2000B307E407F50720F0A21BB30BE40BF50BD6
:10DF3000661F771F881F991F1A9469F7609570955F
:10DF4000809590959B01AC01BD01CF010895F89497
:02DF5000FFCF01
:10DF520000000000000000000000000000000000BF
:10DF620000000000000000000000000000000000AF
:10DF7200003022366D247D20390F76461040105233
:10DF82003F065B4F666D7D077F6F484861484327B8
:10DF92007B777F393F79713D76060E763837373F8A
:10DFA200733F776D783E3E7E76665B39640F230859
:10DFB20002777C585E79716F74040C743837545C44
:10DFC2007367506D781C1C7E766E5B39300F0100D2
:10DFD2000100000000003507370E0715A51B1422AB
:10DFE2005428672E4E340B3A9E3F0A454E4A6C4FD8
:10DFF20065543A59ED5D7E62ED663D6B6E6F8073DE
:10E0020075774E7B0B7FAC823486A289F88C359073
:10E012005B936B966499489C179FD2A179A40DA734
:10E022008EA9FDAB5BAEA8B0E4B210B52CB739B97E
:10E0320037BB27BD09BFDEC0A5C25FC40DC6AFC7CF
:10E0420045C9D0CA4FCCC4CD2ECF8ED0E4D131D366
:10E0520074D4AED5DFD607D827D940DA50DB58DCE6
:10E0620059DD53DE46DF32E017E1F6E1CFE2A1E30C
:10E072006EE434E5F5E5B1E668E719E8C5E86DE96F
:10E0820010EAAEEA47EBDDEB6EECFBEC84ED09EE59
:10E092008BEE09EF83EFFAEF6DF0DEF04BF1B5F1A5
:10E0A2001CF280F2E1F240F39CF3F5F34CF4A0F49D
:10E0B200F2F442F58FF5DAF524F66BF6B0F6F3F6E4
:10E0C20034F773F7B1F7EDF727F860F897F8CCF863
:10E0D20000F932F963F993F9C1F9EEF91AFA44FA3F
:10E0E2006EFA96FABDFAE3FA08FB2BFB4EFB70FBC5
:10E0F20091FBB1FBD0FBEEFB0BFC28FC43FC5EFC6E
:10E1020078FC92FCABFCC3FCDAFCF1FC07FD1CFDC5
:10E1120031FD45FD59FD6CFD7EFD90FDA2FDB3FD77
:10E12200C3FDD4FDE3FDF2FD01FE0FFE1DFE2BFE3D
:10E1320038FE45FE51FE5DFE69FE75FE80FE8AFEDA
:10E1420095FE9FFEA9FEB3FEBCFEC5FECEFED7FE27
:10E15200DFFEE7FEEFFEF6FEFEFE05FF0CFF13FFFD
:10E162001AFF20FF26FF2CFF32FF38FF3EFF43FF3E
:10E1720048FF4EFF53FF57FF5CFF61FF65FF69FFDA
:10E182006EFF72FF76FF7AFF7DFF81FF84FF88FFBB
:10E192008BFF8EFF92FF95FF98FF9BFF9DFFA0FFD5
:10E1A200A3FFA5FFA8FFAAFFADFFAFFFB1FFB3FF1B
:10E1B200B6FFB8FFBAFFBCFFBDFFBFFFC1FFC3FF81
:10E1C200C4FFC6FFC8FFC9FFCBFFCCFFCEFFCFFF06
:10E1D200D0FFD2FF0000EE01DA03C305A9078C09C4
:10E1E2006C0B4A0D250FFD10D212A414741641189F
:10E1F2000B1AD31B981D5A1F1A21D7229124492684
:10E20200FE27B129612B0E2DB92E62300832AB33B5
:10E212004D35EB368738213AB93B4E3DE03E7140F1
:10E22200FE418A4313459A461F48A149224B9F4CFF
:10E232001B4E944F0C518152F4536455D3563F58A0
:10E24200A959115B775CDB5D3D5F9C60FA615663A7
:10E25200AF6407665C67B068016A516B9E6CEA6DD9
:10E26200346F7B70C171057347748775C576027808
:10E272003C79757AAC7BE17C147E457F7580A38105
:10E28200CF82F983218548866D879188B289D28AA7
:10E29200F18B0D8D288E418F59906F9183929693B9
:10E2A200A794B695C496D197DB98E599EC9AF29B20
:10E2B200F79CFA9DFB9EFB9FFAA0F7A1F2A2ECA3AA
:10E2C200E5A4DCA5D2A6C6A7B9A8AAA99AAA88AB32
:10E2D20076AC61AD4CAE35AF1CB003B1E7B1CBB299
:10E2E200ADB38EB46EB54CB629B705B8DFB8B8B9C0
:10E2F20090BA67BB3CBC10BDE3BDB4BE85BF54C081
:10E3020022C1EEC1BAC284C34DC415C5DCC5A2C6C2
:10E3120066C729C8ECC8ADC96DCA2BCBE9CBA5CC61
:10E3220061CD1BCED4CE8DCF44D0FAD0AFD162D244
:10E3320015D3C7D378D427D5D6D584D630D7DCD752
:10E3420086D830D9D9D980DA27DBCCDB71DC15DD70
:10E35200B7DD59DEFADE9ADF39E0D7E074E110E288
:10E36200ACE246E3DFE378E410E5A6E53CE6D1E67D
:10E3720065E7F9E78BE81CE9ADE93DEACCEA5AEB3F
:10E38200E7EB74EC00ED8AED14EE9EEE26EFAEEFB5
:10E3920035F0BBF040F1C4F148F2CBF24DF3CEF3CD
:10E3A2004FF4CFF44EF5CCF54AF6C7F643F7BEF775
:10E3B20039F8B3F82CF9A5F91DFA94FA0AFB80FB97
:10E3C200F5FB6AFCDDFC50FDC3FD34FEA5FE16FF25
:10E3D20085FFF4FF001D660700000000000000003A
:10E3E20002006C077607800789070000001A93076E
:10E3F2000000000000000000001B9B07000000005E
:10E40200000000000019A307000000000000000047
:10E412000202AD07B707C007C907D1070114D90720
:10E42200C408E207E607EA070016EE07000000004C
:10E4320000000000001CF4070000000000000000C3
:10E442000017FB070000000000000000001D660727
:10E452000000000000000000020104080C080F0880
:10E462000D080000010A11081B081F080000000027
:10E47200020524082E081B081F0832080117370856
:10E482003F0843080000000002034708B707C0071F
:10E49200C907D107020451085C08600864086808CB
:10E4A20001126C0871081B081F080000011676088B
:10E4B2007C0881088A08000000189108000000000A
:10E4C200000000001E00181D0C0D1F0102030405B0
:10E4D200060708090A0B191B1A1CFFFFFFFFFFFFA3
:10E4E200FFFF8001C000A80090008000600048008B
:10E4F20030002400180012000C000900060004007D
:10E5020003000200010000FFFFFFFFFF01020408F9
:10E51200102040801009150919091D092109250932
:10E5220029092D093109350939093E0943094809E3
:10E532004D095209570901010101010101010103BC
:10E5420002060201010101010204020302010208A2
:10E552000C080A0808080808080808080A080C0C29
:10E562000000000000080C0A0A0A0A0A0C0C080241
:10E572000302000001000101010101000101003755
:10E5820056656F7C878B8F949AA4B0B9BFD2476CC3
:10E5920069476C6927732050363030207570677276
:10E5A20061646520616C706861205365702020365B
:10E5B2002032303134007370656564006C666F2000
:10E5C20073686170650070756C73652D7472690093
:10E5D20072616E642D73696E006E6F6973652D735F
:10E5E2006177005669622073706400566962206127
:10E5F2006D74006D6F642064656C617900616D708B
:10E6020020736861706500666173742D65787000AF
:10E61200666173742D6C696E00736C6F2D65787012
:10E6220000736C6F2D6C696E0062656E6420746796
:10E63200740056636F0056636600566F6C00676C19
:10E6420069646500646574756E6500616D7020565D
:10E65200656C6F006C666F207467740061620061A4
:10E66200006C666F2072616E6765006C6F77006880
:10E67200696768006D6F642072616E6765006D691D
:10E682006E0066756C6C006D6F6420746774006C4C
:10E69200666F005669620066696C20736861706516
:10E6A2000062656E642072616E676500326E64009E
:10E6B20033726400357468004F6374007072696F5E
:10E6C200006C6173740070697463680066726565DA
:10E6D2000073656D69746F6E65006F637461566572
:10E6E2000066696C2056656C6F00203D2000207228
:10E6F200656376002073656E640062656E646572A0
:10E702002063616C696272617465640056632D00F6
:10E7120056632D206F66660056632D206F6E007063
:10E722007265736574732064756D70656400496EFB
:10E73200742073796E63004D6964692073796E6326
:10E7420000746170652073796E6300737072656125
:10E7520064206F6E00737072656164206F6666007C
:10E762006F6D6E69006368310063683200636833FD
:10E772000063683400636835006368360063683795
:10E782000063683800636839006368313000636889
:10E7920031310063683132006368313300636831BC
:0CE7A200340063683135006368313600D4
:020000021000EC
:10E000002F923F924F925F926F927F928F929F9248
:10E01000AF92BF92CF92DF92EF92FF920F931F9336
:10E02000CF93DF93CDB7DEB72A970FB6F894DEBF54
:10E030000FBECDBF2FEF31EE44E0215030404040C5
:10E04000E1F700C00000F89414B817B81AB81DB86A
:10E0500010BA15B890EE98B91BB81EB883EE81BB04
:10E060002FEF24B997B947E04AB99DB980BB36EC88
:10E0700031BB469A97B94AB99DB915B880E888B9B5
:10E080001BB81EB8F7E4F1BB52E05A95F1F700C097
:10E0900086B189B18CB131BB479AE7EEE7B977EF2A
:10E0A0007AB962EE6DB931BB469AA1E0A5B982E4B6
:10E0B00088B91BB81EB887E881BB8DE08A95F1F757
:10E0C000000031BB469A97B94AB99DB9A5B920E479
:10E0D00028B91BB82EB9F1BBB2E0BA95F1F700C070
:10E0E00086B159B1BCB131BB479AE7B97AB96DB9BC
:10E0F000BDE0BA95F1F7000031BB469A97B94AB92D
:10E100009DB9A5B928B91BB82EB9F1BBF2E0FA95B3
:10E11000F1F700C026B199B14CB131BB479AE7B9CC
:10E120007AB96DB93DE03A95F1F70000422F469576
:10E13000437060E8269F90011124242B392F307101
:10E14000322B292F269526952870232B969590768D
:10E15000922B907C21E0903C09F020E0382F3695FE
:10E160003370A0E88A9FC0011124832B952F9071F2
:10E17000982B852F869586958870982B852F869568
:10E180008076982B907C81E0903C09F080E082239F
:10E1900009F4B4C286EC81BB469A21E025B990E42B
:10E1A00098B99BB91EB897E891BBBAE0BA95F1F758
:10E1B00000C081BB469A25B934E438B930E73BB991
:10E1C00032E23EB991BBEAE0EA95F1F700C081BBCB
:10E1D000469A25B922E428B920E52BB920EC2EB9BE
:10E1E00091BBFAE0FA95F1F700C081BB469A15B8E9
:10E1F00026E828B923E02BB91EB891BBAFE9BFE0F0
:10E200001197F1F700C0000081BB469A15B823E8CA
:10E2100028B923E12BB922E02EB991BBBAE0BA9517
:10E22000F1F700C081BB469A20EE27B997E09AB972
:10E230002DB915B870E878B99BB91EB867E461BB11
:10E24000E2E0EA95F1F700C036B139B13CB181BBEB
:10E25000479A57EE57B947EF4AB932EE3DB9F5E064
:10E26000FA95F1F7000081BB469A27B99AB92DB902
:10E2700015B878B99BB990E29EB961BB22E02A95A6
:10E28000F1F700C096B199B19CB181BB479A57B9DB
:10E290004AB93DB935E03A95F1F7000099249394D5
:10E2A000612C712C0F2EF4EF4F2EF1E15F2EF02D2B
:10E2B0000F2EF4EF2F2EF2E13F2EF02D88248394C1
:10E2C0009FD499230CF405C2803F9105C9F798D4D7
:10E2D000892B09F0FEC194D48136910509F0F9C16A
:10E2E0008FD4469709F0F5C18BD48B36910509F090
:10E2F000F0C186D499230CF4ECC1A3015827052E54
:10E300000294202D2F702527352F3025330F307E96
:10E310002327302D3527307F3695052E000C331FEF
:10E320005695569556955F7153275427422F7A017B
:10E330008F7799278C011695102F00271795079531
:10E340005FD499230CF4C5C1D701B8270B2E0294D2
:10E35000202D2F702B273B2F3025330F307E232786
:10E36000302D3B27307F36950B2E000C331FB69592
:10E37000B695B695BF71B327BA27A22F7D018F77C7
:10E380009927082B192B0115B1E01B0721F0012B50
:10E3900009F4A1C19EC134D46C0199230CF499C134
:10E3A00087011827012E0294802D8F708127912FCD
:10E3B0009025990F907E8927902D9127907F969593
:10E3C000012E000C991F1695169516951F71192789
:10E3D0001027082F15D45C0199230CF47AC1F80199
:10E3E000F8270F2E0294802D8F708F279F2F902556
:10E3F000990F907E8927902D9F27907F96950F2EBD
:10E40000000C991FF695F695F695FF71F927FE27F2
:10E41000E82FFA87E9878201F3D399230CF4F4C03B
:10E42000E984FA84A7015827052E0294202D2F7025
:10E430002527352F3025330F307E2327302D3527E4
:10E44000307F3695052E000C331F56955695569500
:10E450005F7153275427422F7A015A874987DC017D
:10E46000AF77BB27BA83A983CBD399230CF4CCC055
:10E47000F701F8270F2E0294202D2F702F273F2F02
:10E480003025330F307E2327302D3F27307F3695C0
:10E490000F2E000C331FF695F695F695FF71F327B6
:10E4A000FE27E22F7F01FA87E9879C012F77332728
:10E4B0003C832B83A5D399230CF4A6C0A70158272E
:10E4C000052E0294202D2F702527352F3025330F50
:10E4D000307E2327302D3527307F3695052E000CD2
:10E4E000331F5695569556955F7153275427422FE3
:10E4F0007A015A874987DC01AF77BB27BE83AD839A
:10E500007FD399230CF480C0F701F8270F2E0294D3
:10E51000202D2F702F273F2F3025330F307E2327BC
:10E52000302D3F27307F36950F2E000C331FF69588
:10E53000F695F695FF71F327FE27E22F7F01FA8704
:10E54000E9879C012F77332738872F8359D3992365
:10E550000CF45AC0A7015827052E0294202D2F70C5
:10E560002527352F3025330F307E2327302D3527B3
:10E57000307F3695052E000C331F569556955695CF
:10E580005F7153275427422F5A874987F8013397E1
:10E590009C013695322F2227379527955981252BB7
:10E5A0002083F80132979C0122703327002436958E
:10E5B00027950794369527950794322F202D6B8148
:10E5C000262B2083F80131979C0124703327220FDA
:10E5D000331F22953295307F3227207F3227AD813D
:10E5E0002A2B20838870992782959295907F98276F
:10E5F000807F9827BF818B2BF80180830C5F1F4F92
:10E600000215130509F008CFFBD299230CF461C061
:10E610008C01102F0027110FF3D299230CF459C04D
:10E620008F779927880F991F880F991F082B192B0F
:10E63000E7D299230CF44DC083709927082B192B2E
:10E6400029853A850217130709F043C0D9D2873FBD
:10E65000910509F03EC0990C3FE3391508F4982C58
:10E6600046EC41BB469A892D880F392D3695282FC7
:10E6700026702064992D991F9927991F292B992D70
:10E680009071482F440F4072942B807C982B832FDD
:10E690008270806285B828B99BB98EB957E851BBA2
:10E6A0006AE06A95F1F700C0B5016F777727C60178
:10E6B0008F7799279695982F882797958795682B18
:10E6C000792B762F662780E090E041EF51E198D4D6
:10E6D000F7CD89E701C08DE696EC91BB469A982F5D
:10E6E0009071906E86958270806221E025B922E457
:10E6F00028B99BB98EB987E881BBFFCF2A960FB6A0
:10E70000F894DEBF0FBECDBFDF91CF911F910F9167
:10E71000FF90EF90DF90CF90BF90AF909F908F9041
:0EE720007F906F905F904F903F902F900895E4
:10EC000045E04A95F1F70000349B04C000C000C005
:10EC10003499FCCF86EC81BB469A20EE27B997E069
:10EC20009AB92DB915B820E828B99BB91EB897E450
:10EC300091BB52E05A95F1F700C096B129B13CB1B1
:10EC400081BB479A87EE87B987EF8AB982EE8DB983
:10EC500085E08A95F1F70000392F3695337040E84A
:10EC6000949FC0011124832B922F9071892B922F96
:10EC7000969596959870892B26952076282B217B42
:10EC8000213809F040C026EC21BB469A90EE97B996
:10EC900087E08AB99DB915B890E898B98BB980E238
:10ECA0008EB987E481BB52E05A95F1F700C036B1C6
:10ECB00099B14CB121BB479A87EE87B987EF8AB9E2
:10ECC00082EE8DB985E08A95F1F70000832F869555
:10ECD000837050E8359F90011124282B892F807173
:10ECE000282B892F869586958870282B9695907667
:10ECF000292B50E0CA01880F991F84709927822B15
:10ED0000282F30E002C02FEF3FEF822F932F08957E
:10F000008F929F92AF92BF92CF92EF92FF92CF9347
:10F01000DF93EA01CFB6F894F999FECF23E0FB0124
:10F0200080935B002093570010D707B600FCFDCFFC
:10F03000DE01B3954B015C0121E04881F980E12CB0
:10F04000F701E40FF11DAF0122960A01F401A0922D
:10F050005B0020935700F9D61124F2E08F0E911C2B
:10F06000A11CB11CAC17BD0741F725E0FB01809343
:10F070005B0020935700E9D607B600FCFDCF81E185
:10F0800080935700E2D6CFBEDF91CF91FF90EF90F3
:0CF09000CF90BF90AF909F908F9008959C
:00000001FF
